:020000040000FA
:107800005469616E59696E673130300000000000C4
:1078100054593230302E303830303030625F747925
:10782000424154333247313339474B3634464200B4
:1078300043414E5F5354440000000000000000002C
:1078400043414E5F43485F300000000000000000ED
:1078500043414E5F3530304B6270730000000000D2
:107860009407000014070000DF070000000000007C
:020000040000FA
:1080000080330020E9800000F1800000F380000050
:108010000000000000000000000000000000000060
:10802000000000000000000000000000FB800000D5
:108030000000000000000000FF8000008DCA010069
:108040003514010079140100A9140100D9140100AC
:108050000915010039150100691501009915010084
:10806000C9150100F91501002D1601004116010086
:10807000511601008516010095160100A516010094
:10808000D91601001D17010065170100AD17010089
:10809000F51701003D1801004D180100811801007D
:1080A000B5180100E5180100191901004D1901006A
:1080B0005D1901006D190100A1190100D519010018
:1080C000EF72E8FF03B40148019001BD017F002079
:1080D0000448854600F02CFA00480047390F02009A
:1080E000C046C046803300201648804716480047E7
:1080F000FEE7FEE7FEE7FEE7FEE7FEE7FEE7FEE758
:10810000FEE7FEE7FEE7FEE7FEE7FEE7FEE7FEE747
:10811000FEE7FEE7FEE7FEE7FEE7FEE7FEE7FEE737
:10812000FEE7FEE7FEE7FEE7FEE7FEE7FEE7FEE727
:10813000FEE7FEE7FEE7FEE7FEE7FEE7FEE7FEE717
:10814000FEE7000091D00100D180000030B50B4661
:10815000014600202022012409E00D46D5409D4221
:1081600005D31D469540491B2546954040191546A7
:10817000521E002DF1DC30BD70B5002425460028CC
:1081800001DA01244042002901DA01254942FFF7C2
:10819000DDFFAC4200D04042002C00D0494270BD0F
:1081A000F0B51FB40646002082B005464024019178
:1081B00000901BE0019922460F46304600F066F918
:1081C000049A059B801A994110D3104619462246FD
:1081D00000F04CF9361A8F41019722460120002108
:1081E000009F00F043F938184D4100902046641E6E
:1081F0000028DFDC019B00982946324607B0F0BD1D
:10820000F0B51FB486B0002000900190029006984F
:10821000069980B204900798090C020400141143D7
:1082200007900027089D099806913E463C4603901A
:108230000398A9B20204000C039004982D0C154376
:1082400048430021224600F011F9C719714110344A
:108250000E46402CECDB3846029A00F007F9009AF3
:10826000019B8018009059410298019110300290B2
:108270004028CCDB00980BB0F0BD03460B439B07B6
:1082800003D009E008C9121F08C0042AFAD203E08B
:108290000B780370401C491C521EF9D27047D2B2B1
:1082A00001E00270401C491EFBD270470022F6E735
:1082B00010B513460A4604461946FFF7F0FF20465C
:1082C00010BD30B504460020034600E05B1C93421D
:1082D00003D2E05CCD5C401BF8D030BD0321001D13
:1082E000401E037812021A43491EF9D51046704702
:1082F000034603220870000A491C521EFAD518468C
:108300007047024670B54A40D30FDB0740002DD0BE
:108310004A002AD0010E140E000212020919400A66
:10832000520A8418E50104465443000A120A2E0436
:108330005043A4194219200CC543AA18120C012558
:10834000AD03521C521912047F39240400D0521C70
:10835000104301D44000491EC2B20C06C0092018C7
:10836000401C4008802A02D003E0002070BD400875
:108370004000002900DA0020184370BD70B50246A5
:108380004A40D50F40004A00ED0740085208002837
:1083900014D0002A12D0C40DD30D41020120C00513
:1083A0005202490A520AE41A091812187D349142FD
:1083B00001D3641C00E04900002C01DA002070BDEC
:1083C0000023914201D3891A034340084900002841
:1083D000F7D100290AD0914202D10121C90705E055
:1083E000914201D2012101E00121C943E005C018F9
:1083F000401900F05CF870BD10B5002296231146BC
:1084000000F05DF810BDC20FD207400040080BD04D
:10841000C10D0723DB01C91840020905400A1143B9
:10842000C208400711437047002001467047000012
:1084300010B5002904DB0124E40740428C412146A9
:10844000002B04DB1C460123DB075242A341994267
:1084500000D1904210BD00000122D207002800DBAD
:10846000101A002900DB511A8842704710B5202AE3
:1084700004DB0146203A9140002010BD91402023AA
:108480009C1A0346E3401943904010BD10B5202AC2
:1084900004DB0846203AD040002110BD0B46D340F3
:1084A000D0402024A21A91400843194610BD00294B
:1084B00004DA401C490001D140084000704770B404
:1084C0000024050C05D11024000402D1002921D07C
:1084D0001124050E01D100020834050F01D100015D
:1084E000241D850F01D18000A41C002801DB400061
:1084F000641C002908D020252E1B0D46F540A14004
:1085000000D001212943084301061B1B000ADB1D83
:1085100002D5002070BC7047DB05181880180029B0
:10852000F8DA401C4900F5D170BC400840007047A3
:10853000064C0125064E05E0E36807CC2B430C3CB6
:1085400098471034B442F7D3FFF7C6FD74230200F6
:10855000A423020070B58C180578401C6B075B0FD4
:1085600001D10378401C2A1106D10278401C03E097
:1085700006780E70401C491C5B1EF9D12B0705D4F0
:108580000023521E0DD40B70491CFAE70378401CDF
:10859000CB1A921C03E01D780D70491C5B1C521E07
:1085A000F9D5A142D8D3002070BD70B507F0A6F868
:1085B0000524204618F07AFC0025284607F092F89A
:1085C000204618F073FC0126304607F067F8204675
:1085D00018F06CFC284607F061F8204618F066FC9D
:1085E000304607F07FF8204618F060FC70BDB0B54B
:1085F00007F084F80524204618F058FC0125284689
:1086000007F070F8204618F051FC284607F046F8AD
:10861000204618F04BFC002007F040F8204618F0E8
:1086200045FCB0BDF0B581B007F054F8052018F056
:108630003DFC08270026012007F030F805242046DD
:1086400018F034FC204618F031FC07F039F80546E4
:10865000204618F02BFC002007F020F8204618F0E8
:1086600025FC76002E437F1E3806E4D1F0B201B01F
:10867000F0BD70B50446002007F010F807F03EF892
:10868000052018F013FC0826E0B2C00907F02AF80C
:108690000525284618F00AFC012006F0FFFF2846B1
:1086A00018F004FC002006F0F9FF284618F0FEFB45
:1086B000284618F0FBFB6400761E3006E4D1052046
:1086C00018F0F4FB012070BDF0B583B0019314469F
:1086D0000E460746012038430290032504E000F0CF
:1086E0008EF86D1E280631D000F067F83846FFF787
:1086F000C0FF00F0A7F80028F1D13046FFF7B9FF1E
:1087000000F0A0F80028EAD100F057F80298FFF72F
:10871000B0FF00F097F80028E1D1019802280BD3B0
:10872000451E0026FFF77EFF2070FFF73EFF641C0A
:10873000761CF0B28542F5DCFFF774FF2070FFF77E
:1087400056FF00F05CF8202003B0F0BD102003B00D
:10875000F0BDF0B583B01C46009201910290032554
:1087600004E000F04CF86D1E280623D000F025F838
:108770000298FFF77EFF00F065F80028F1D101981C
:10878000FFF777FF00F05EF80028EAD1002C0CD04C
:108790000026009F3878FFF76CFF00F053F80028A0
:1087A000DFD1761C7F1CA642F4D300F028F8082005
:1087B00003B0F0BD102003B0F0BDB0B506F09EFFD1
:1087C0000524204618F072FB0125284606F066FFB6
:1087D000204618F06BFB284606F084FF204618F070
:1087E00065FB0025284606F07DFF204618F05EFB5D
:1087F000284606F053FF642018F058FBB0BDB0B512
:1088000006F07CFF0524204618F050FB0025284682
:1088100006F044FF204618F049FB284606F062FFA8
:10882000204618F043FB0125284606F037FF204676
:1088300018F03CFB284606F055FF642018F036FB84
:10884000B0BD0000B0B506F045FF0524204618F085
:108850002DFB012006F022FF204618F027FB0B4DD0
:1088600006F02EFF044606F013FF002C02D06D1E0A
:108870002804F5D10525284618F018FB002006F03D
:108880000DFF284618F012FB2046B0BD3321000032
:10889000034801780B2901D8491C01707047C04674
:1088A0006B2F002070B584B00025039502950195CB
:1088B000009506F0EDFE0F20C6430E4C1036F1B2C7
:1088C000A0206A461023FFF744FF204618F0EEFA76
:1088D000204618F0EBFA912EF0D3A020B0216A4682
:1088E0001023FFF736FF204618F0E0FA0248058013
:1088F00004B070BD581B00005E2F002070B5022927
:1089000002D2EB24E0B270BD891EEB250022134693
:1089100005E0401C5B1CDDB2A94225460EDB047855
:108920006C40154604E034466E1C072D3546F0D2E7
:108930006608E407F7D09A246640F4E7E0B270BD19
:10894000F0B591B00C91417810AA117083781B0298
:108950005918C37804792402E3181B0459180B0E24
:10896000D3700C0C94700D0A55700B910895691812
:10897000099409190A93C9180278D24389184279CF
:1089800083791B029A18C379047A2402E3181B0422
:108990009A188918130A0693C918130C0593C91855
:1089A0000792120E04928918827AC37A1B029A18CF
:1089B000037B0F90447B2402E3181B0498180918CA
:1089C000020A02928918020C019289180D910390F3
:1089D000000E0E9000200346014606E032409A4009
:1089E000D2B211435B1C082B0ED0012635469D40A8
:1089F0000746024602E07F1C042FEFD010ACE45D76
:108A00002542F8D0521CF6E70E9C0D980019C3B20F
:108A10000F98827B934205D0427A914202D1002086
:108A200011B0F0BD1021FFF769FF0C99CC72019ACB
:108A30008A72029A4A72039A0A72049ACA71059A51
:108A40008A71069A4A71079A0A710A9ACA70099A33
:108A50008A70089A4A700B9A0A7011B0F0BDF0B58E
:108A60008DB055220270002747720B784370CA7987
:108A7000059202728A790492C2714A7903928271D4
:108A80000A7902924271CA7A089242738A7A0192F2
:108A900002734E7AC6720C7A84720CAA13704D78E7
:108AA0002D02EB188D78C978090249190904CB18F1
:108AB000190E01711D0CC57009931B0A0B90837070
:108AC00038460A91D170079595700693537031021C
:108AD0000919089A1202019BD21812045118089120
:108AE00003990902029A8918059A1202049BD21866
:108AF0001204511805913D463A4605E02640AE4025
:108B000032436D1C082D0ED001242146A940034696
:108B1000064602E05B1C042BF0D00CAFFF5C394230
:108B2000F8D0761CF6E70B9B5A7209980699401804
:108B3000079940180A994018059A8018110A401898
:108B4000110C4018110E4018089A8018110A40188C
:108B5000110C4018110E4018563898731021184601
:108B6000FFF7CCFE0DB0F0BDF0B58FB00446FF208E
:108B7000E070A07060700F20C04302900F30207032
:108B8000704818F093F970490868632801D8642088
:108B900008606E4F002038806D4E0190308008E0F4
:108BA0000B99814222D338881030388080B2A128B6
:108BB0006DD206F06DFD3978A02003AA1023FFF7CF
:108BC00083FD30802028EED103AD0BA92846FFF7A6
:108BD000B7FEE97B8842E6D128785528E3D15D4885
:108BE000017800290298DBD10846D9E73888A02807
:108BF0004DD8C0B20021019105E006F049FD398849
:108C0000C8B2A12943D2C1B2A02003AA1023FFF702
:108C10005BFD3080398810313980202837D103AD91
:108C200007A92846FFF78CFEE97B8842E5D1287822
:108C30005528E2D1474800780028029900D1014622
:108C400007988842D9D240490A68962151430B9A25
:108C5000824208D90818904219D30BA90E22204647
:108C6000FFF70BFBC9E78918814210D307A90E2231
:108C70002046FFF702FB0BA80A99818107980B9009
:108C800008980C9009980D9038880190B5E72078E5
:108C9000617809020818A178E278120251180904D3
:108CA0000818401C24D1002001903880A020B02159
:108CB00003AA1023FFF708FD3080202818D103AD48
:108CC0000BA92846FFF73CFEE97B884210D12878A3
:108CD00055280DD11F480078002800D102900B982C
:108CE0000299884204D20BA90E222046FFF7C5FA4A
:108CF0002078617809020818A178E27812025118E8
:108D000009040818401C0CD10020E072A0726072A7
:108D10002072E071A07160712071E070A0706070CD
:108D20002070019838802078617809020818A178AD
:108D3000E2781202511809040818074908603088BF
:108D40000FB0F0BD70110100582F00205E2F0020E1
:108D5000542F0020572F0020642F0020F0B581B041
:108D600000910646214800250570002A2ED01446A1
:108D7000C036631B71190F2008401022101A83425D
:108D800000D303461A480278102A01D0042A1AD1C7
:108D9000C809FE2707405F2F13D80127B843603862
:108DA000C0B29E3282420CD3009A5219C9B2DFB2CD
:108DB0003B46FFF789FC0F490880ED19A542D8D33F
:108DC00004E0082000E004200A49088009480188DE
:108DD0000020042902D0082900D00120034908708E
:108DE000411E8841400001B0F0BDC0466A2F0020FE
:108DF000562F0020682F00200A4A012313700A4AC8
:108E000010700A4A11600A4A00211160042801D139
:108E100005218901102801D11D208101054801800B
:108E20007047C046572F0020562F0020582F002093
:108E3000642F00205C2F0020F0B587B0994D0026EC
:108E40002E80994B1B688B4224D1994C2188202974
:108E500025D1029000920196964C00272760964DEE
:108E6000964E2878062809D806F012FC2068401C87
:108E70002060B042F5D38D48042101802F70904CC2
:108E800020880107029B31D0884820210180854D30
:108E9000019E0BE0012040028449088006E003A8FF
:108EA000FFF762FE20808148802101807F48008892
:108EB0003F2807DD874988420BDC402812D08028F4
:108EC00010D010E004280DD008280AD0202809D09E
:108ED00009E001214A02904204D0C902884201D02F
:108EE00001E002262E80288807B0F0BDA128019E4F
:108EF00000D32780009A012A6A4D1ED1187B0128D1
:108F000056D1DF719F715F711F711F73587B0128EC
:108F100004D1DF729F725F721F725F7303AF3846B6
:108F20001946FFF79CFDF8732088002846D01038BA
:108F3000C1B2A02003AA102344E0002AB6D16148A0
:108F400001780029B2D002701878597809020818FF
:108F50009978DA7812025118090408185A490978E0
:108F6000002901D00F21C943884233D2274603ACE0
:108F700020461946FFF773FDE0733978A0201023CF
:108F80002246FFF7E6FB029A4849088008288DD15F
:108F90003888103038801078517809020818917894
:108FA000D2781202511809040818484908607DE770
:108FB000597B012911D10128A3D0A7E7A02003AA3A
:108FC00010230146FFF7C5FB384908803D4800994A
:108FD00001706BE70120C0025EE73D480078012880
:108FE00012D103AC20461946FFF739FDE073A020EB
:108FF000B02110232246FFF7ACFB2C49088008283B
:10900000E4D133480770E1E7187859780902081865
:109010009978DA7812025118090408182B4909685E
:10902000214A12685118884203D220484021018009
:10903000CCE725490978002901D00F21C94388428E
:109040002DD203AF384619461C46FFF708FDF873CA
:109050001B480178A02010233A46FFF77AFB1349FA
:1090600008800828B2D11649088810300880207876
:10907000617809020818A178E278120251180904EF
:1090800008181249086008490A6815215143FFF77A
:109090005DF800299AD101200D49087096E701205A
:1090A000C00291E7702F0020582F00206E2F002063
:1090B000542F0020742F00206B2F0020818D5B0027
:1090C0005E2F0020602F0020572F0020642F0020EB
:1090D0006C2F0020FF010000F0B585B00646434C20
:1090E0000027278004921018414A1288904241D2EA
:1090F00001910397404F0020029038603F4C404D53
:109100002078052809D806F0C3FA3868401C386072
:10911000A842F5D3374804210180029820703948CD
:10912000018839480278102A01D0042A32D18819DE
:109130000346C033049C651A0F2404401020001B12
:10914000854200DB0546DC09603C01263002E7B2BF
:109150007F09052F12D3B443E6B29E32B242234CAC
:10916000039F0DD301984218D9B2EBB23046FFF7F6
:10917000F0FA05E01F482021018011E01B4C039FFD
:109180001C49088008280BD1E8B21E4A118808182B
:10919000108005E00120800216490880134C039FCF
:1091A000144800881F2809DD202813D001210A0255
:1091B00090420FD0890288420CD00CE0042809D0DC
:1091C000082808D10F4800880499884201D3022753
:1091D00000E001272780208802210143022902D1D3
:1091E000084900220A8005B0F0BDC046702F00205B
:1091F0005C2F00206E2F0020742F00206B2F00208A
:10920000818D5B00782F0020562F0020F0B585B0AF
:10921000044600200190042C6FD20CF09BF800282B
:1092200001D10CF017F90020009000BF0098401CFD
:1092300000900CF08FF803900398002803D0484961
:1092400000988842F2D30398002856D1042145485B
:109250000CF062F84448454908802101444A515CB9
:109260004900404A505A41490A880121090300F047
:1092700055F902900120049020013D4940184078A2
:10928000002801D100264BE02001394940184078E0
:10929000012802D13548068842E0200134494018AF
:1092A000407802282AD12001401805792901304A46
:1092B000515C49002B4A505A2C490A880121090364
:1092C00000F02CF9064628012A49431828012849AC
:1092D00040180289280140180021C7683046B84765
:1092E00006462801224BC018C2882801C018817880
:1092F000304600F087F8064612E02DE020011C49B8
:1093000040184078032804D02001401840781328E2
:1093100004D1200116494018868801E000200490FD
:109320000498002818D02001124943182001104940
:1093300040180289200140183146C7680298B84792
:10934000019020010A4BC018C2882001C018817802
:10935000019800F057F80190019805B0F0BD0000A9
:1093600050C30000F200002088130000EC00002031
:10937000101A0200501A0200F8B505460E461446AF
:109380000020009001211C4801751C48007888438A
:109390001A490870084680780821084317498870E0
:1093A000002088710846007801210843134908709D
:1093B00008460572002717E010480078802108430E
:1093C0000E49087000BF0E48007D0028FBD0002029
:1093D0000B4908750948C0892080A41C0748C18929
:1093E0000098081800907F1CB742E5D331460098DA
:1093F000FEF7ACFE80B2F8BD406100400050044072
:109400004060004010B50346012908D1094CA41A58
:109410009C4202D99C18A0B20BE0064809E0022940
:1094200006D1934202DD9C1AA0B202E0002000E0C7
:10943000184610BDFFFF000010B504460121202092
:1094400002F012F8002032490870012131480175FC
:10945000002031490875152017F010FA2C48807843
:10946000E17808432A4988700846807821780843C3
:10947000274988702078802806D108460079E1794C
:10948000490008432249087121488078E17A08435D
:109490001F498870A078002803D108460079087118
:1094A0000FE0A078012806D119480079602108430F
:1094B0001749087105E016480079802108431449CE
:1094C0000871134880792179084311498871084649
:1094D0008079617908430E498871207AC872607A70
:1094E0008872084600783821884309490870084680
:1094F00000786178C900084305490870A07A0873AC
:1095000008460078012108430149087010BD000099
:10951000005004404061004040600040F8B50446FF
:109520000E461746002E01D100250FE0A64201DCB1
:109530003D460BE00094009C204678430090314665
:109540000098FEF703FE0090009885B22846F8BD0B
:109550000146042904D28A00024BD218508800E048
:1095600000207047282900200146042903D28A00E0
:10957000024B985C00E00020704700002829002082
:10958000FFB587B004460898844203DA0A988068D9
:10959000002802D12448019042E00898001B82B2C2
:1095A0000292002625460A98806800212F463A46F6
:1095B0003346049605910690FEF722FE05460E46B8
:1095C000002328463146029AFEF7EAFD05460E467C
:1095D000304600210A4649405040014302D012481B
:1095E00001901DE003950A98C068039DA84202D32C
:1095F0000020019014E00A98C1680398401A039073
:1096000009990398FEF7A2FD03900398000C00044B
:10961000002802D00448019002E0039880B2019033
:1096200001980BB0F0BD0000FFFF000010B5084826
:10963000007880218843064908700121054801759A
:10964000002005490875152017F018F910BD000015
:10965000005004404061004040600040F8B50546BD
:109660000E4614461F4621462846FEF785FD80B269
:10967000F8BD0000FFB587B006460A98406800288C
:1096800001D1029035E00A980168406808180390FB
:10969000002534460021274603980695049105903D
:1096A00038462946049B059AFEF7AAFD04460D4656
:1096B0000A98406802460023019020462946FEF79A
:1096C0006FFD04460D46002320462946099AFEF701
:1096D00067FD04460D4628460749214000235940AE
:1096E0005840014303D00448C043029001E0A0B2B7
:1096F000029002980BB0F0BD0000FFFF10B5FE48CD
:1097000000688079030017F09FF807059ED8F5F4EC
:10971000F3F2F100F84800684079030017F094F87C
:109720000805138A2A8A468A638A13F0E7F800201C
:10973000F1490968C873F04800684079401CEE4957
:10974000096848717DE0ED494969EB4A1268D27AAF
:10975000885C13F04BF9E84800684079401CE64902
:1097600009684871E44800684079401CE24909688A
:10977000487166E00AF0A8F8002810D113F036F915
:10978000DD4800684079401CDB4909684871DA48C7
:1097900000684079401CD8490968487105E013F019
:1097A000D7F80020D449096848714AE00AF08CF8DB
:1097B000002811D1112013F019F9CF480068407921
:1097C000401CCD4909684871CB4800684079401C6D
:1097D000C9490968487105E013F0BAF80020C64984
:1097E000096848712DE00AF06FF800281BD1C248C3
:1097F0000068C07A401CC0490968C872BE48006849
:10980000C07ABE49097888420DDB0020BA49096850
:10981000C872B94909684862B74800688079401C35
:10982000B5490968887113F093F80020B2490968B6
:10983000487106E013F08CF80020AF4909684871C0
:1098400000BF00BF32E3AC480068407C002817D05E
:10985000AA48C068002803D0A848C16819208847D2
:109860000020A54909684862A34800688079401C27
:10987000A1490968887100209F49096848711BE067
:109880009D480068406A282807D29B480068406AC3
:10989000401C9949096848620EE000209649096811
:1098A0004862954800688079401C9349096888712E
:1098B0000020914909684871F8E28F4800684079B2
:1098C000030016F0C1FF080518A42FA44CA480A41F
:1098D00013F014F8002088490968C87386480068A6
:1098E0004079401C84490968487197E0D4E2C7E296
:1098F00030E25DE194E0814949697F4A1268D27A99
:10990000885C13F073F87C4800684079401C7A4901
:1099100009684871784800684079401C76490968B0
:1099200048717BE009F0D0FF002811D1012013F02D
:109930005DF8714800684079401C6F4909684871BA
:109940006D4800684079401C6B490968487105E022
:1099500012F0FEFF00206849096848715EE009F0D6
:10996000B3FF002828D164490968C97A24225143E9
:10997000634A12688918604A1268D27B885C13F0C7
:1099800035F85D480068C07B401C5B490968C873B6
:1099900059480068C07B242814D357480068407990
:1099A000401C554909684871534800684079401C7B
:1099B00051490968487105E012F0CAFF00204E497C
:1099C000096848712AE009F07FFF002818D14A4849
:1099D0000068C07A401C48490968C8724648006857
:1099E000C07A4649097888420ADB00204249096862
:1099F000C872414800688079401C3F4909688871F5
:109A000012F0A6FF00203C490968487106E012F0F8
:109A10009FFF002038490968487100BF00BF45E238
:109A2000354800684079030016F00EFF0A0614B9A5
:109A30002BB948B978B995B912F060FF00202E49CA
:109A40000968C8732C4800684079401C2A49096895
:109A50004871ABE029494969274A1268D27A885C83
:109A600012F0C4FF244800684079401C224909686C
:109A70004871214800684079401C1F4909684871B5
:109A800094E009F021FF002811D14A2012F0AEFF26
:109A9000194800684079401C174909684871164800
:109AA00000684079401C14490968487105E012F0CB
:109AB0004FFF002010490968487177E009F004FF62
:109AC000002824D1FF2012F091FF0B480068C07BD2
:109AD000401C09490968C87307480068C07B2428EE
:109AE0001BD3054800684079401C03490968487148
:109AF00001480068407905E0D40700203C2F002091
:109B0000D0070020401CEA490968487105E012F0BE
:109B10001FFF0020E6490968487147E009F0D4FEBC
:109B2000002811D1FF2012F061FFE1480068407960
:109B3000401CDF4909684871DD4800684079401CD5
:109B4000DB490968487105E012F002FF0020D8499E
:109B5000096848712AE009F0B7FE002818D1D448F6
:109B60000068C07A401CD2490968C872D0480068B1
:109B7000C07AD049097888420ADB0020CC490968BC
:109B8000C872CB4800688079401CC949096888714F
:109B900012F0DEFE0020C6490968487106E012F0A6
:109BA000D7FE0020C2490968487100BF00BF7DE1AF
:109BB000BF4800684079030016F046FE0C0715C345
:109BC0002CC349C366C382C39FC312F097FE002013
:109BD000B7490968C873B64800684079401CB44961
:109BE00009684871B4E0B3494969B14A1268D27A48
:109BF000885C12F0FBFEAE4800684079401CAC491E
:109C000009684871AA4800684079401CA849096859
:109C100048719DE009F058FE002811D1772012F01C
:109C2000E5FEA34800684079401CA14909684871D5
:109C30009F4800684079401C9D490968487105E0CB
:109C400012F086FE00209A490968487180E009F008
:109C50003BFE002811D10C2012F0C8FE9448006889
:109C60004079401C924909684871914800684079E0
:109C7000401C8F490968487105E012F069FE002018
:109C80008B490968487163E009F01EFE002810D175
:109C900012F0ACFE864800684079401C844909688F
:109CA0004871834800684079401C814909684871BF
:109CB00005E012F04DFE00207D490968487147E03B
:109CC00009F002FE002811D1132012F08FFE78480F
:109CD00000684079401C76490968487174480068FA
:109CE0004079401C72490968487105E012F030FE65
:109CF00000206F49096848712AE009F0E5FD002855
:109D000018D16B480068C07A401C69490968C8725C
:109D100067480068C07A6749097888420ADB0020F2
:109D200063490968C872624800688079401C6049CC
:109D30000968887112F00CFE00205D4909684871BD
:109D400006E012F005FE002059490968487100BF7D
:109D500000BFABE0564800684079030016F074FD80
:109D6000080513872A874787638712F0C7FD0020FD
:109D70004F490968C8734E4800684079401C4C49F7
:109D8000096848717AE04B494969494A1268D27AB0
:109D9000885C12F02BFE464800684079401C44491C
:109DA00009684871424800684079401C4049096888
:109DB000487163E009F088FD002811D1492012F0B4
:109DC00015FE3B4800684079401C394909684871D4
:109DD000374800684079401C35490968487105E0FA
:109DE00012F0B6FD002032490968487146E009F0DA
:109DF0006BFD002810D112F0F9FD2D480068407964
:109E0000401C2B4909684871294800684079401C6A
:109E100027490968487105E012F09AFD002024499D
:109E2000096848712AE009F04FFD002818D1204840
:109E30000068C07A401C1E490968C8721C48006846
:109E4000C07A1C49097888420ADB00201849096851
:109E5000C872174800688079401C154909688871E4
:109E600012F076FD002012490968487106E012F0F0
:109E70006FFD00200E490968487100BF00BF15E062
:109E800000200B4909688871094909684871062052
:109E900007490968C87009E012F05AFD002004491A
:109EA0000968487102490968887100BF00BF10BD88
:109EB000D40700203C2F002010B56A480068407984
:109EC000030016F0C1FC090610C627C644C6608E02
:109ED000C60012F013FD634800684079401C6149D8
:109EE00009684871BCE0604949695E4A1268D27AE3
:109EF000885C12F07BFD5B4800684079401C594942
:109F000009684871574800684079401C55490968FC
:109F10004871A5E009F0D8FC002811D17F2012F08B
:109F200065FD504800684079401C4E4909684871F9
:109F30004C4800684079401C4A490968487105E06E
:109F400012F006FD002047490968487188E009F0D1
:109F5000BBFC002810D112F049FD4248006840794E
:109F6000401C4049096848713E4800684079401CDF
:109F70003C490968487105E012F0EAFC00203949C3
:109F8000096848716CE009F09FFC002822D135482F
:109F90000068C07A401C33490968C87231480068BB
:109FA000C07A3149097888420FDB00202D490968C1
:109FB000C8722C4800684079401C2A4909684871D9
:109FC000002028490968486208E0002025490968FE
:109FD000487103E0002023490968487112F0B8FC79
:109FE0003EE020480068407C002816D01E48C0682B
:109FF000002803D01C48C16819208847002019494F
:10A0000009684862174909684871164909688871E2
:10A01000052014490968C8701AE012480068406AAF
:10A02000282807D20F480068406A401C0D4909687B
:10A0300048620DE000200B49096848620949096837
:10A040004871084909688871052006490968C8707F
:10A0500006E012F07DFC002002490968487100BF4B
:10A0600000BF10BDD40700203C2F002010B50024F5
:10A07000F7480068807A01287ED1F5480068C079E9
:10A0800000287AD0F24800688079002804D001289E
:10A0900074D0022873D191E1ED480068007B242838
:10A0A0006ED2EB480068C07901287AD1002475E0AF
:10A0B000E7480068C07A24214843E6490968401807
:10A0C000E3490968097B415CE1480068C07A2422C1
:10A0D0005043E14A12688018DD4A1268127B805CA6
:10A0E000814229D0DA480068C07A24214843DA49FD
:10A0F00009684018D6490968097B415CD448006862
:10A10000C07A24225043D34A12688018D04A126879
:10A11000127B8154CE480068407B242805D3CC486C
:10A120000068007BCA4909684873C9480068007B19
:10A13000C7490968887308E0C5480068407B24283F
:10A1400003D20120C24909688871C1480068007BB8
:10A15000401CBF4909680873BD480068007B24287B
:10A1600008D3BB480068407B242803D20120B849AB
:10A1700009688871B64805E0D3E1CDE169E0BAE14C
:10A1800038E00EE00068007B242804D2B048006864
:10A190008079012800D103E0601CC4B2242C87D34D
:10A1A00056E0002413E0AA480068C07A24214843FE
:10A1B000A94909684018015DA5480068C07A2422B1
:10A1C0005043A44A126880180155601CC4B2242C64
:10A1D000E9D300209E490968487323209C490968F7
:10A1E000887301209A490968887124209849096870
:10A1F00008732DE0002096490968087394480068A8
:10A20000C07A401C92490968C87291480068C07AB7
:10A2100092490978884217DB8D480068007C012844
:10A2200004D102208A490968887106E00020884923
:10A230000968887186490968C871002084490968DD
:10A24000C872834909680874002081490968487107
:10A2500061E17F4800684079030016F0F5FA0805CF
:10A2600013A62AA651A68EA601207949096808746A
:10A2700012F044FB764800684079401C7449096834
:10A28000487199E075494969714A1268D27A885CC7
:10A2900012F0ACFB6E4800684079401C6C490968BC
:10A2A00048716B4800684079401C694909684871E9
:10A2B00082E009F009FB00281BD165490968497B48
:10A2C000491CC8B212F092FB61480068407B6049AB
:10A2D0000968C8735E4800684079401C5C49096899
:10A2E00048715B4800684079401C594909684871C9
:10A2F00005E012F02DFB00205549096848715BE02C
:10A3000009F0E2FA00282BD151490968C97A2422C0
:10A310005143504A126889184D4A1268D27B885CB2
:10A3200012F064FB4A480068C07B401C4849096839
:10A33000C87347480068C07B45490968897B8842E3
:10A340001ADD434800684079401C4149096848715A
:10A350003F4800684079401C3D49096848710BE05E
:10A3600012F0F6FA3A480068407B39490968C87328
:10A3700000203749096848711EE009F0A5FA002855
:10A380000CD1334909688871242031490968C873A0
:10A390002F49096848732E490968887312F0D8FA62
:10A3A00000202B490968487106E012F0D1FA00201C
:10A3B00027490968487100BF00BFACE02448006825
:10A3C0004079030016F040FA08050F8E268E4C8E59
:10A3D000688E12F093FA1E4800684079401C1C49B0
:10A3E0000968487185E01D494969194A1268D27A9D
:10A3F000885C12F0FBFA164800684079401C14494A
:10A4000009684871124800684079401C1049096881
:10A4100048716EE009F058FA002811D1492012F075
:10A42000E5FA0B4800684079401C09490968487101
:10A43000074800684079401C05490968487105E0F3
:10A4400012F086FA002002490968487151E00000C4
:10A45000D4070020D0070020CC0700203C2F00208C
:10A4600009F032FA002810D112F0C0FA9C480068B6
:10A470004079401C9A4909684871994800684079B8
:10A48000401C97490968487105E012F061FA002004
:10A490009349096848712CE009F016FA00281AD18E
:10A4A0008F480068C07A401C8D490968C8728C4882
:10A4B0000068C07A8B49097888420CDB0020884903
:10A4C0000968C872864909688871854909684871B0
:10A4D00083490968C87112F03BFA00208049096875
:10A4E000487106E012F034FA00207D49096848718D
:10A4F00000BF00BF0FE012F02BFA00207849096876
:10A500004871774909688871754909680873744901
:10A510000968C87200BFE2E00020714909688872CA
:10A52000DDE06F480068807A0228F4D16C4800684A
:10A53000007A002879D06A4800684079030016F054
:10A5400083F90B0711BB25BB41545EBB7590BB0063
:10A5500012F0D4F9624800684079401C60490968EB
:10A560004871B7E05F494969087812F03FFA5C48E2
:10A5700000684079401C5A49096848715848006889
:10A580004079401C564909684871A3E009F09CF9DC
:10A59000002810D112F02AFA514800684079401C76
:10A5A0004F49096848714E4800684079401C4C4941
:10A5B0000968487105E012F0CBF9002048490968A4
:10A5C000487187E009F080F9002807D14448006805
:10A5D0004079401C42490968487103E00020404925
:10A5E0000968487112F0B4F974E012F087F93C4838
:10A5F00000684079401C3A49096848716AE0394965
:10A6000049690978491CC8B212F0F0F93448006869
:10A610004079401C324909684871314800684079E6
:10A62000401C2F490968487154E054E009F04CF986
:10A6300000280FD112F034F92949096888700120E7
:10A6400012F0A8F9264800684079401C244909689E
:10A65000487105E012F07CF9002021490968487131
:10A6600038E01F480068807811280CD100201C4970
:10A6700009680872AA201A490968887000201849D8
:10A680000968487011E0164800684078401C144979
:10A6900009684870124800684078032805D309F01B
:10A6A000B3F900200E490968487012F051F90020F2
:10A6B0000B49096848710DE012F04AF90020084979
:10A6C00009684871064909684870AA200449096860
:10A6D000887000BF03E0002001490968887210BD3E
:10A6E000D40700203C2F0020F0B505460C46164646
:10A6F0001F462088482806DA3A462946304605F0A3
:10A7000005F8012800D0F0BD2088C0002E50208818
:10A71000401C208000BFF6E710B502469000074BB2
:10A72000C018405C002802D00320C04310BD0120A7
:10A730009300024C1B1958540020F7E7BC2A002054
:10A7400070B5002508E06D1C1B48854202D20AF056
:10A75000ADFE01E0002503E00AF0FCFD0028F2D187
:10A7600000BF022100200AF003FE032100200AF0AE
:10A77000FFFD052100200AF0FBFD072100200AF063
:10A78000F7FD002408E00020A1000C4A5054A1006D
:10A7900089184880601CC4B2042CF4D301200849F5
:10A7A000087000204870052088700020C870054897
:10A7B0000549088070BD000050C300002829002012
:10A7C000EE00002088130000EC000020F8B58D4852
:10A7D0000078030016F038F8060405163D5EFDFC0F
:10A7E0000EE10AF037FE00208649C870487008461E
:10A7F0008078002802D10320087002E002208149FD
:10A800000870FDE07F488078002804D07D4880787B
:10A81000401E7C4988700AF09DFD00280BD10AF08B
:10A8200019FE00207749C8700846807800280FD1AB
:10A83000032008700CE07348C078401C7149C87050
:10A840000846C078052803D3052008700AF02EFEBC
:10A85000D6E00AF07FFD00280ED104216A480AF0F4
:10A860005BFD00206749C8704870684868490880E7
:10A870000420644908700CE06248C078401C6149BB
:10A88000C8700846C078052803D3052008700AF070
:10A890000DFEB5E05B49497809015E4A515C49000B
:10A8A000594A505A5A490A8801210903FEF736FECF
:10A8B00000900125534840780001564940184078DF
:10A8C000002801D100243CE04E4840780001514965
:10A8D00040184078012802D14D48048831E04948A9
:10A8E000407800014B4940184078022812D1454970
:10A8F00049780901474A89180879FEF729FE044674
:10A90000404949780901434A89180879FEF72CFE25
:10A91000054616E03B48407800013E494018407823
:10A92000032806D0374840780001401840781328A3
:10A9300006D134484078000136494018848800E048
:10A940000025002D2FD02F484078000132494318B0
:10A950002C48407800012F49401802892948407846
:10A96000000140182146C7680098B84706462548A8
:10A9700040780001274BC018C28822484078000167
:10A98000C01881783046FEF73DFD06461D484078E8
:10A99000800022494018468001201A4949788900E0
:10A9A0001E4A50540AE000201649497889001B4A83
:10A9B00089184880134949788900505411484078D3
:10A9C000401C1049487008464078042809D301E02B
:10A9D00013E007E00AF03EFD00200A49487003201A
:10A9E00008700DE00AF0B6FC002803D101200549EB
:10A9F000087001E00AF05AFD02E0FFF7A1FE00BF77
:10AA000000BFF8BDEE000020F20000208813000017
:10AA1000EC000020101A0200501A02002829002021
:10AA200010B50AF061FC002405E00020A100074AEF
:10AA30005054601CC4B2042CF7D3002004490870A1
:10AA40000520887003480449088010BD282900208B
:10AA5000EE00002088130000EC00002070B50446D2
:10AA6000002000F0AFF8002000F0DAF8002000F03D
:10AA70009BF8002000F0C4F8002000F087F80020C8
:10AA800000F0AEF800BF012000F08EF8012000F0C9
:10AA9000B7F8002521E0002000F086F8002000F043
:10AAA000AFF880202040002806D0012000F08AF86E
:10AAB000012000F0B5F805E0002000F083F8002048
:10AAC00000F0AEF800BF012000F06EF8012000F0A9
:10AAD00097F86006040E681CC5B2082DDBDB012068
:10AAE00000F054F8012000F07BF870BD70B504460A
:10AAF0000D46012000F066F8012000F091F80020DA
:10AB000000F052F8002000F07BF8002000F03EF842
:10AB1000002000F065F800BF012000F045F801209A
:10AB200000F06EF8002628E0002000F03DF800203C
:10AB300000F066F880202040002803D0012000F0BB
:10AB400041F802E0002000F03DF880202840002875
:10AB500003D0012000F064F802E0002000F060F86B
:10AB600000BF012000F020F8012000F049F8600645
:10AB7000040E6806050E701CC6B2082ED4DB012038
:10AB800000F004F8012000F02BF870BD10B5044669
:10AB9000002C04D0812103200AF01AFD03E080215B
:10ABA00003200AF015FD10BD10B50446002C04D09A
:10ABB000812104200AF00CFD03E0802104200AF02A
:10ABC00007FD10BD10B50446002C04D081210220E1
:10ABD0000AF0FEFC03E0802102200AF0F9FC10BD1F
:10ABE00010B50446002C04D0812104480AF0F0FC82
:10ABF00003E0802101480AF0EBFC10BD01070000D2
:10AC000010B50446002C05D08121072000020AF06F
:10AC1000DFFC04E08021072000020AF0D9FC10BD0F
:10AC200010B50446002C04D0812104480AF0D0FC61
:10AC300003E0802101480AF0CBFC10BD02070000B0
:10AC400010B5F920FFF70AFF3221424805F09CFDBC
:10AC50008820FFF703FF9020FFF700FF9820FFF701
:10AC6000FDFE08210846FFF741FFE820FFF7F6FE4A
:10AC700012210846FFF73AFFA020FFF7EFFE7021F0
:10AC80000846FFF733FFA820FFF7E8FE70210846CB
:10AC9000FFF72CFFB020FFF7E1FE70210846FFF719
:10ACA00025FFB820FFF7DAFE00210846FFF71EFF58
:10ACB000C020FFF7D3FE00210846FFF717FFC8208A
:10ACC000FFF7CCFE00210846FFF710FFD020FFF76A
:10ACD000C5FE2F210846FFF709FFD820FFF7BEFE6B
:10ACE0002F210846FFF702FFE020FFF7B7FE2F21D4
:10ACF0000846FFF7FBFE4020FFF7B0FE00210846A4
:10AD0000FFF7F4FE0A20FFF7A9FE002405E000216A
:10AD10000846FFF7EBFE601CC4B25A2CF7DB002498
:10AD20000AE000200C4908550C4908550C49085503
:10AD30000C490855601CC4B25A2CF2DB8120FFF785
:10AD40008DFE0020084908708870C870087148702E
:10AD500010BD0000204E000050260020AA26002032
:10AD6000042700205E270020C300002010B58020AB
:10AD7000FFF774FE10BD0000002004490870012098
:10AD8000034908700020487070470000C800002088
:10AD9000C300002010B54848007800287AD0464803
:10ADA0008078030015F050FD0604434A535A687E2C
:10ADB000414800794149085C3F490979404A515C62
:10ADC000884209D13C4800793E49085C3A490979F2
:10ADD0003D4A515C88421BD0374800793749085CAE
:10ADE00035490979364A5054334800793549085C69
:10ADF00031490979344A50542F48C078002803D08B
:10AE000004202D49887011E001202B4988700DE045
:10AE100000202949C87008460079401C087108467E
:10AE200000795A2802DB00200871087041E04020B8
:10AE3000FFF714FE0220204988703AE01E4A11797B
:10AE40001079FFF753FE03201B49887031E00A2078
:10AE5000FFF704FE0420184988702AE0164A127988
:10AE6000194B995C144A1279154B985CFFF73EFE1A
:10AE70000520114988701CE00F480079401C0E49DC
:10AE80000871084600795A2805DB0020087108700F
:10AE9000C87003E00EE001200749C8700020064991
:10AEA000887006E00020044908708870C870087136
:10AEB00000BF00BF10BD0000C300002050260020CE
:10AEC000AA260020042700205E27002010B512F0DB
:10AED0004DF9012837D1072009F0CCFA002810D00D
:10AEE0001C480078052805DA1A480078401C1949E2
:10AEF000087016E0052017490870002016490870F0
:10AF00000FE015480078052805DA13480078401C42
:10AF10001149087005E005200F49087000200D490F
:10AF200008700C480078052806D14B22D200002179
:10AF3000012013F049FE0BE07D22D2000021012008
:10AF400013F042FE04E000221146012013F03CFE03
:10AF500010BD00001D0000201C000020002003493F
:10AF6000087248708870486070470000600A0020CE
:10AF700058221152704710B504460121022000F0FA
:10AF800073FA0021022000F06FFA10BD0146002084
:10AF90005322525C10231A40002A08D05322525CDC
:10AFA0000C231A409210032A18D1032016E05422D1
:10AFB000525A0123DB031A40002A0ED05322525C5E
:10AFC0000C231A409210032A05D05322525C920798
:10AFD000920F032A01D1022000E0012070470246AF
:10AFE000002058239B5A0B40002B01D0012000E089
:10AFF00000207047014600226020405AFF231B02B8
:10B0000018400005020F1001014BC01870470000E6
:10B010000055044010B5002A0AD056231B5A0C02D2
:10B0200023435624235256231B5A8B43235209E0B1
:10B0300056231B5A0C02A3435624235256231B5A51
:10B040000B43235210BD0000F8B504460D460127FE
:10B0500000263448844203D10121022000F004FA82
:10B060002878401EA0702088FF21013108432080ED
:10B070002088400840002080A878401EC1B25A2095
:10B08000015568790007000CE97909020843A9799C
:10B0900008435C210853288981B240200153A868E5
:10B0A000C000C10C42200153A88981B24420015341
:10B0B000E868C000C10C46200153288A81B24820AC
:10B0C00001532869C000C10C4A200153A88A81B2EB
:10B0D0004C2001536869C000C10C4E200153502020
:10B0E000005B297909020843502108535020005B76
:10B0F000297988435021085300E0761C5020005BDA
:10B100004007400F2979884202D007488642F4D18F
:10B110005020005B4007400F2979884200D000276B
:10B120003846F8BD00540440FFFF000030B5034628
:10B1300000201C898C4209DD082A05D218244C43C2
:10B140001D682C19A05C02E0002000E0002030BD4A
:10B1500010B5024613898B4205DD18234B43146852
:10B16000E318987C00E0002010BD0146FF22C8894A
:10B17000C007C00F00280AD00120C88100E0521E7D
:10B18000C889C007C00F002801D0002AF7D1C8899C
:10B19000C007C00F00280FD10220C8810420C88139
:10B1A000487A400840004872487A382398434872E9
:10B1B00000204872012070470020FCE70246507AC8
:10B1C000012318435072507A0B78DB0018435072F9
:10B1D000087A012808D1888850814868000C01232A
:10B1E000DB031843908108E0087A002805D15081DC
:10B1F000486880001A4B18409081487A012804D191
:10B20000507A40231843507206E0487A002803D150
:10B21000507A4023984350720878002811D1C87A98
:10B220001072087B1070487B5070887B9070CB7BCD
:10B23000D370087C10714B7C5371887C9071CB7CEF
:10B24000D371887A002803D00120C002D08101E0A8
:10B250000820D081FF200130D081012070470000FC
:10B26000FC1F0000002904D0427A80231A43427256
:10B2700003E0427A80239A434272704730B5024617
:10B2800000200F4B5024A45A0D022C435025AC52E1
:10B290005024A45A8C43AC5200E05B1E5024A45AA4
:10B2A0006407640F8C4201D0002BF6D15024A45ABD
:10B2B0006407640F002C01D0002000E0012030BDA5
:10B2C000FFFF0000827A80231A40802A00D081721A
:10B2D0007047000070B5044600250023002D02D001
:10B2E0000126602006530420C88188890126F603C0
:10B2F0003040002808D0012010728889C004C0089E
:10B300004E893043506006E00020107288890F4E4D
:10B31000304080105060087AD072002304E0CE5C88
:10B3200010460C30C6545B1CD07A9842F7DCC889B2
:10B3300004263040002804D1C889F6023040002895
:10B3400001D0002070BDD07AFCE70000FC1F000097
:10B350000020024908800249088070477A000020D6
:10B360007C000020027C80231A40802A00D00174D7
:10B37000704710B50246FF23D089C007C00F0028D0
:10B3800002D00120D0815B1ED089C007C00F0028E9
:10B3900001D0002010BD507A012420435072507A11
:10B3A0003824A0435072C87A1072487A00280FD10E
:10B3B000087B1070487B5070887B9070CC7BD47079
:10B3C000087C10714C7C5471887C9071CC7CD47159
:10B3D000FF200130D0814000D081107ADAE70000F0
:10B3E000F8B504460D460020002C00D100BF002A0D
:10B3F00000D100BF012C01D141263043012A01D1E7
:10B4000012263043022C01D1C0263043022A01D13A
:10B4100030263043134E307076788027BE43114F6C
:10B420007E70012C08D1FF2100BF0E4EB3781E465E
:10B430000E4033468B42F8D10A4E76784027BE4301
:10B44000084F7E70012A0BD10026009603E000BF52
:10B45000009E761C0096FF276937009EBE42F6D9F3
:10B46000F8BD000000040240002905D0054A12780A
:10B470000243044B1A7004E0024A12788243014BE3
:10B480001A70704720040240002905D0054A927EB8
:10B490000243044B9A7604E0024A927E8243014BB7
:10B4A0009A7670470008024070B5034614460020A3
:10B4B000002B01D1C0B202E005468035E8B2012977
:10B4C00002D1051DE8B206E0022903D10546083580
:10B4D000E8B200E0C0B2012C02D1851CE8B200E065
:10B4E000C0B2084DA870AD7801263543054EB57041
:10B4F000002201E000BF521C7D252D01AA42F9D98E
:10B5000070BD0000000C024070B500242448007992
:10B5100020210840002801D0224D3FE000F046F8ED
:10B5200005462148007880210840002836D01E4872
:10B5300080780840002801D01A4D02E000F036F86B
:10B540000546194880780007840F022C01DBAD08FE
:10B5500004E0012C01D16D0800E000BF12488078A2
:10B560008007C00F002801D02D0101E00C204543C9
:10B570000D4800784007840F002C02D1601CC4B233
:10B5800007E0032C03D1601C4006040E01E06006B6
:10B59000040E21462846FCF7D9FD0546284670BD15
:10B5A0000004024000127A00000C024000B5C022E4
:10B5B0009178F82211401C4A12781143EA2923D0CD
:10B5C0000ADC0A46E03A130015F03EF90A181C207E
:10B5D000242A2A2A2A161A2AED291FD004DCEB294C
:10B5E00016D0EC291CD117E0F02903D0F82917D187
:10B5F0000E4817E00E4815E00E4813E00E4811E023
:10B600000E480FE00E480DE00E480BE00E4809E032
:10B610000E4807E00E4805E00E4803E00E4801E042
:10B620000D4800BF00BF00BD201C02400090D003A9
:10B63000006CDC020048E80100366E010024F400D2
:10B64000001BB70000127A00808D5B0000093D00EE
:10B65000C0C62D0080841E0040420F0070B586B029
:10B6600004460025002620680290A1796846C1732F
:10B670006179417300210173017100BF05E020462B
:10B680000830415D04A841556D1C6846C07BA84246
:10B69000F5D80B22D2010299881A914237D007DCE3
:10B6A0002548081A1FD023210901401A3AD113E076
:10B6B000FF386F38002802D0012833D105E001A9F6
:10B6C0001E48FFF756FE06462DE001A91B484030F4
:10B6D000FFF74FFE064626E001A918485030FFF755
:10B6E00048FE06461FE001A914482030FFF741FE3E
:10B6F000064613480088072805DA11480088401CD0
:10B700000F49088002E000200D4908800BE005F099
:10B71000C1FC002805D001A908486030FFF729FEC8
:10B72000064600E000BF00BF002E02D1012006B097
:10B7300070BD0020FBE7000020020000805504409F
:10B740007C00002010B5A8211348FCF7AFFD12487B
:10B75000124908601248486007200881002088725A
:10B7600007220F490D4800F0A9FA00210B48FFF706
:10B77000A9FDA0210B48FCF799FD0A480A49486039
:10B780000A4B05220A49084800F037FC0021064808
:10B79000FFF7E8FD10BD00007408002054080020E9
:10B7A000481602001C090020600800205DB6000059
:10B7B000BC1502000C4A127812060B4B5B781B0476
:10B7C0001A43094B9B781B021A43074BDB781A4339
:10B7D000104642084240D20083085A401146034AAC
:10B7E0005140034A116070471B070020010200000E
:10B7F00020070020F8B504460F46A07A4006400E08
:10B80000002874D10025ACE018206843216808188E
:10B81000407C01283CD1012118206843226810187F
:10B82000017400260CE018206843216808180830CD
:10B83000815D18206843226810188155701CC6B2BB
:10B84000082EF0D3002118206843226810180174D4
:10B850001820684322681018417418206843226831
:10B8600010184161182068432268101881742C2038
:10B87000684361680818406A002809D018236B43A0
:10B880002268D0182C236B436268D218516A88470B
:10B8900018206843216808184069FF21C94388427D
:10B8A0005DD818206843216808184069C11918201C
:10B8B00068432268101841611820684321680818FD
:10B8C00041692C206843626810188069814246D320
:10B8D0001820684321680818807C55283FD05521DE
:10B8E00018206843226810188174002624E03CE088
:10B8F0001820684321680818805D2C21694362681C
:10B9000051181031895D0840182169432268511887
:10B9100088551820684321680818805D2C216943E8
:10B92000626851180831895D08431821694322680B
:10B9300051188855701CC6B2082ED9D32C206843E4
:10B9400061680818806A002809D018236B432268B0
:10B95000D0182C236B436268D218916A8847681C00
:10B9600085B22089A84200DD4EE7F8BD01200149DB
:10B97000087070479400002010B50446002015F0B0
:10B98000C7FA02284DD1FFF7E3FC2D4800780028C4
:10B9900002D101202A49087029480078012823D1C2
:10B9A00027484078401C2649487021465A20FCF719
:10B9B000CDFB23494978884241D80020204948706E
:10B9C00008468078401C8870084680780A2803D38F
:10B9D0000020887002200870FFF7BAFC00F068F8B9
:10B9E000002015F0C5FA2AE015480078022826D173
:10B9F00013484078401C1249487021467D20C00001
:10BA0000FCF7A4FB0E494978884218D800200C495D
:10BA10004870FFF79DFC00F04BF8002015F0A8FAE5
:10BA20000DE00748C078401C0549C8700846C0783A
:10BA3000042804DB0020C87008704870887010BDAE
:10BA40007600002000B587B000216846017104210E
:10BA500041710C480290411003910B4904910591EA
:10BA60000A480690FFF76EFE01A815F0E5FA00F00F
:10BA70007BFB00F033F80021054809F015FE07B004
:10BA800000BD0000FFFF1F00FFFFFF1F45BD0000BE
:10BA90000205000030B5034600201C898C4204D901
:10BAA0004D015C686419626000E0022030BD000056
:10BAB00010B5002400BF09E01C2060430549401870
:10BAC000214682680448FFF7E5FF641C052CF3D388
:10BAD00010BD0000BC1502006008002010B5FF205A
:10BAE000023072494860002008720120087000206E
:10BAF0004872012088726E48FFF737FB6B496C482B
:10BB0000FFF75CFB01216A48FFF7ACFB6948674916
:10BB1000486000200872012008700020487201204F
:10BB2000887263481030FFF720FB6049604810308E
:10BB3000FFF744FB01215E481030FFF793FB5D489F
:10BB4000401E5A49486000200872012008700020F9
:10BB500048720120887256485030FFF706FB53495F
:10BB600053485030FFF72AFB012151485030FFF76E
:10BB700079FB5048C1384D494860002008720120C7
:10BB80000870002048720120887249484030FFF751
:10BB9000ECFA464946484030FFF710FB0121444883
:10BBA0004030FFF75FFBFF20123040494860002023
:10BBB00008720120087000204872012088723C48F9
:10BBC0006030FFF7D2FA394939486030FFF7F6FAAA
:10BBD000012137486030FFF745FBFF202130334912
:10BBE000486000200872012008700020487201207F
:10BBF00088722F48A030FFF7B8FA2C492C48A030A3
:10BC0000FFF7DCFA01212A48A030FFF72BFB294877
:10BC10008F382649486000200872012008700020F3
:10BC20004872012088722248E030FFF79EFA1F49CF
:10BC30001F48E030FFF7C2FA01211D48E030FFF74E
:10BC400011FB1D4819494860002008720120087046
:10BC5000002048720120887215482030FFF785FACD
:10BC6000124913482030FFF7A9FA0121104820306B
:10BC7000FFF7F8FA1048CB300C49486000200872F2
:10BC80000120087000204872012088720848303076
:10BC9000FFF76BFA054906483030FFF78FFA0121AC
:10BCA00003483030FFF7DEFA10BD0000802A002084
:10BCB000105504400204000014070000F0B50B46C4
:10BCC000144643600481002136E0002216E02C2552
:10BCD0004D4346687519AD5C18274F430668F61941
:10BCE000B5542C254D4346687519AD5C18274F4354
:10BCF0000668F6190836B554551CEAB2082AE6D388
:10BD0000002518274F430668F619357418274F4346
:10BD10000668F619757418274F430668F619B57446
:10BD200018274F430668F619F57418274F4306681D
:10BD3000F61975614D1CA9B205898D42C5DC002537
:10BD40008572F0BD70B50446606800F013FE0546CC
:10BD5000E27A23460C332946094800F0D3FD09490D
:10BD60006068884204D00749CB396068884206D1B0
:10BD7000E17AA28890B222460C3203F003F870BD3B
:10BD800054080020DF070000F8B5054600262C46C1
:10BD9000002C29D000BF03E00020A055701CC6B2C3
:10BDA000082EF9D304F024FFC000082108400746FC
:10BDB0002078884338432070E079E02188430B499C
:10BDC00009884901E02211400843E07104F010FFA6
:10BDD000012801D1082000E00020C706FF0EE0790D
:10BDE000400940013843E071F8BD00007C000020AC
:10BDF000F8B5054600260027002000902C46002CB0
:10BE00005BD000BF03E00020A055701CC6B2082E16
:10BE1000F9D304F0EBFF00280DD005F02FF902282C
:10BE200009D106212548FFF793F9552803D004F0DE
:10BE3000D7FF002803D100202070607011E004F0CB
:10BE4000EBFF92307D21C900884204D804F0E4FF62
:10BE5000923087B201E07D27FF003804000E207089
:10BE6000677005F0C7F800280DD005F00DF902281D
:10BE700009D106211148FFF76BF9552803D005F0C9
:10BE8000B3F8002803D10020A070E07015E005F0A1
:10BE9000C7F892307D21C900884205D805F0C0F866
:10BEA000923080B2009002E07D20C00000900098A7
:10BEB0000004000EA0700098E070F8BD5408002047
:10BEC00070B5054600262C46002C42D000BF03E08A
:10BED0000020A055701CC6B2082EF9D305F0DAF880
:10BEE000012817D11B480088401C80B219490880DE
:10BEF000032804DD00201849087016490880312005
:10BF00002070012060705920A0700820E07000208F
:10BF100020711EE005F0BEF8022817D10D480088F8
:10BF2000401C80B20B490880032804DD00200A4928
:10BF30000870084908803120207001206070592065
:10BF4000A0700820E0700120207102E0002001496B
:10BF5000088070BD7A000020E0000020FEB5054694
:10BF600000260020019001F06BFC074604F070FEF3
:10BF70000A210090FCF700F980B201902C46002CB9
:10BF800018D000BF03E00020A055701CC6B2082ED8
:10BF9000F9D33802000E60713804000EA071E77109
:10BFA00004F050FFFF2802DDFF20A07002E004F043
:10BFB00049FFA070FEBDFEB5054600260020019099
:10BFC000002704F03FFC64210090FCF7D5F880B214
:10BFD0000190002001F056FC87B22C46002C0BD0BB
:10BFE00000BF03E00020A055701CC6B2082EF9D394
:10BFF0003804000EA070E770FEBDFFB581B00446A6
:10C000000F4600250026002000902760039820811D
:10C010000498E0600020207400BF9DE01C2068436D
:10C02000216808586A01616888501C2068432168AB
:10C03000081880686A016168891848601C20684394
:10C040002168081840686A016168891888601C20A6
:10C05000684321680818C0686A0161688918C86067
:10C060001C20684321680818007C6A0161688918EF
:10C0700008741C20684321680818407C6A016168C4
:10C08000891848741C20684321680818807C6A015C
:10C090006168891888831C20684321680818C07C5F
:10C0A0006A0161688918887400206A0161688918CA
:10C0B000C8741C206843216808184068002813D001
:10C0C0001C20684321680818C07C002805D1401E48
:10C0D0006A0161688918C8831AE00020C0436A01B8
:10C0E00061688918C88313E01C2068432168081818
:10C0F000C07C002805D000206A0161688918C883C7
:10C1000006E000206A0161688918C8830120009058
:10C11000002607E000216A0160688018143081550C
:10C12000701CC6B2690160684018808BB042F1DCB7
:10C130001C20684321680818406900280AD06B0158
:10C140006268D218104614301C236B432268D21840
:10C1500051698847681CC5B22089A84200DD5DE7A7
:10C16000009805B0F0BD000000B58BB0684807909E
:10C17000002108A801706846017608A841700020D7
:10C1800064498872082108A8C170002004E00022D8
:10C1900009A90A54411CC8B208A9C9788142F6DC31
:10C1A0005D48FEF7E2FF06A95B48FFF707F858482D
:10C1B000401C0790002108A801706846017608A875
:10C1C0004170002053498872082108A8C1700020DE
:10C1D00004E0002209A90A54411CC8B208A9C97880
:10C1E0008142F6DC4C484030FEF7BFFF06A94A48C2
:10C1F0004030FEF7E3FF452000010790002108A82A
:10C2000001706846017608A8417000204149887293
:10C21000082108A8C170002004E0002209A90A54DE
:10C22000411CC8B208A9C9788142F6DC3A485030AE
:10C23000FEF79BFF06A938485030FEF7BFFF1120DC
:10C2400040010790002108A801706846017608A8FF
:10C25000417000202F498872082108A8C170002071
:10C2600004E0002209A90A54411CC8B208A9C978EF
:10C270008142F6DC28482030FEF777FF06A92648E1
:10C280002030FEF79BFF0B20C0010790002108A87B
:10C2900001706846017608A8417000201D49887227
:10C2A000082108A8C170002004E0002209A90A544E
:10C2B000411CC8B208A9C9788142F6DC1648603032
:10C2C000FEF753FF06A914486030FEF777FF1048C9
:10C2D000A630029000216846017301714173817399
:10C2E0000821C173002004E0002204A90A54411C63
:10C2F000C8B26946C97B8142F6DC07481030FEF7B8
:10C3000034FF01A904481030FEF758FF0BB000BD00
:10C31000EE060000802A002080550440F0B585B06C
:10C3200004460F4600250026207C4006400E552876
:10C330007ED100BF76E1690160684018807C0028EA
:10C3400077D169016068401840686A01616889189E
:10C350008968884209D26901606840184068C0193C
:10C360006A016168891848605AE16901606840188B
:10C37000C068AF49884208D8690160684018C06841
:10C38000401C6A0161688918C860690160684018CA
:10C39000C07C002821D1002607E000216A016068E6
:10C3A000801814308155701CC6B26901606840184D
:10C3B000808BB042F1DC1C2068432168081840697A
:10C3C00000280AD06B016268D218104614301C2372
:10C3D0006B432268D21851698847690160684058E8
:10C3E0000090690160684018017C68460171002175
:10C3F0004171690160684018017F68468171690177
:10C4000060684018417C6846C171002608E06901F7
:10C41000606840181430815D02A88155701CC6B256
:10C42000690160684018808BB042F0DCE06801E090
:10C43000FCE01DE0002806D06846E16888476A01F4
:10C4400061688918C874690160684018C07C002858
:10C4500004D16A01616889184860E1E06901606897
:10C4600040184068C01B6A01616889184860D7E0BD
:10C4700069016068401880680028EED06901606832
:10C480004018C08B0028E8D0690160684018C08B54
:10C490006A0161688918C968884207D169016068C2
:10C4A0004018C08B6249C94388427DD169016068E8
:10C4B000401840686A01616889188968884209D211
:10C4C0006901606840184068C0196A01616889188C
:10C4D0004860A5E000206A01616889184860690128
:10C4E00060684018C0685249884208D8690160688D
:10C4F0004018C068401C6A0161688918C86000263D
:10C5000007E000216A016068801814308155701CB2
:10C51000C6B2690160684018808BB042F1DC1C2013
:10C52000684321680818406900280AD06B016268D6
:10C53000D218104614301C236B432268D21851695C
:10C540008847690160684058009069016068401838
:10C55000017C6846017100214171690160684018E1
:10C56000017F68468171690160684018417C6846B6
:10C57000C171002608E06901606840181430815DCF
:10C5800002A88155701CC6B2690160684018808B92
:10C59000B042F0DCE068002808D06846E1688847CF
:10C5A0006A016168891800E015E0C8746901606873
:10C5B0004018C07C002804D16A016168891848606D
:10C5C0002EE06901606840184068C01B6A0161681C
:10C5D0008918486024E01C206843216808184068D6
:10C5E00000280FD00020C0436A0161688918C88301
:10C5F0001C2068432168081840686A01616889182E
:10C60000886008E000206A0161688918C8836A01AF
:10C6100061688918886000206A0161688918C860AB
:10C62000681CC5B22089A84200DD84E605B0F0BDD3
:10C630000000FFFF7CB500BF19212C480078FBF7F4
:10C6400085FD04462A4860432A4A811800220120B9
:10C650000DF088F820460A2250436430001981B258
:10C66000002201200FF0F0F801200A226243121983
:10C67000D1B20A22624312190090D0B201231A46A5
:10C6800009F026FBFF220721002006F0B5FF01205C
:10C69000009001900B20604382B20B20604381B276
:10C6A000002301200EF0ECFD6F20604381B20120D9
:10C6B0000FF070FB104860430246032101200BF08D
:10C6C000CBFD002505E0012128460BF0FFFC681C8E
:10C6D000C5B20F2DF7DB21460B2251436431C8B29E
:10C6E0000FF0C2FD0FF0AAFD7CBD0000730000201A
:10C6F000672B0000A0860100FCB101000020054965
:10C700000870054908700549087005490870054911
:10C71000087070477400002075000020730000202E
:10C720007200002071000020F0B589B000BF00BF8A
:10C7300000BF00BF00BF00BF00BF00BF00BF00BF01
:10C740005D4800783C2805DA5B480078401C5A496F
:10C75000087002E03C2058490870574800781D28AE
:10C7600005DC56480078401C544908700BE05348DB
:10C770000078002802D15149087004E04F48007841
:10C78000401E4E49087003214C480078FBF7F4FC2A
:10C790004B4948430390052148480078FBF7D6FCF5
:10C7A0000446032145480078FBF7E6FC0B2148438B
:10C7B000643080B20690414909788A0088180621C1
:10C7C000FBF7DAFCFF21F531484380B207900321E3
:10C7D0003A480078FBF7D0FC0B214843643080B224
:10C7E0000890032135480078FBF7C6FC35494843DB
:10C7F000354940180490032130480078FBF7BCFC11
:10C800000B2106464E4303212C480078FBF7B4FC6D
:10C810000B2107464F43032128480078FBF7ACFC67
:10C820006F21484380B2059003210120039A0BF049
:10C8300013FDE1B201200BF0DBFAE1B2012318464F
:10C84000069A09F01FFDFF21F5310798FBF794FCCC
:10C85000C0B20146029001200AF0F6F90022012040
:10C8600008990EF0F1FF0022012004990CF07AFFE4
:10C87000012005990FF08EFA0120F9B20090F0B274
:10C8800001231A46029009F023FAFF220721002013
:10C8900006F0B2FE032109480078FBF76DFC0B217E
:10C8A000484385B20120009000232A462946019082
:10C8B0000EF0E6FC09B0F0BD750000207400002009
:10C8C000FCB10100672B0000A0860100002000BF22
:10C8D00006E00021044A1154044A1154411CC8B214
:10C8E0005A28F6DB7047000050260020042700205D
:10C8F0000348007A002801D10149487070470000C0
:10C90000600A0020FFB581B004460F463D462089ED
:10C91000A8422DDD1820684321680818007C0028F3
:10C9200026D1002609E00498815D1820684322681A
:10C93000101808308155701CC6B2082EF3D301219F
:10C94000182068432268101841742C2068436168DD
:10C950000818006A00280BD018236B432268D218ED
:10C96000104608302C236B436268D218116A88473E
:10C9700005B0F0BD01460720124BCA1A994211D0EA
:10C9800008DCCA1FFA3A002A14D0102A0CD01F2A39
:10C9900014D10DE0322A0FD0C02A07D0C12A0DD100
:10C9A00000200DE001200BE0022009E0032007E059
:10C9B000042005E0052003E0062001E0072000BF79
:10C9C00000BF70474103000010B504467D21C90037
:10C9D00061430846322103F0D7FE10BDFF200B490A
:10C9E00008700020C0430A4908800A490880FF20D7
:10C9F0000949087009490870094908700020094967
:10CA0000086009490860094908607047580000201B
:10CA10005A0000205C0000205E0000205F00002023
:10CA2000600000204C000020500000205400002036
:10CA3000014800687047000050000020014800686D
:10CA4000704700004C00002010B505490988652298
:10CA5000514308466421FBF78FFB80B210BD0000F4
:10CA60005A00002001480078704700005F00002055
:10CA700001480078704700005800002010B510F001
:10CA800075FB01282CD100F063F8012000F066F856
:10CA900003F0DEFE044600F043F804F0B7F8044665
:10CAA00000F04AF804F018FB012805D100F03EF828
:10CAB000012000F047F805E0002000F037F80020E2
:10CAC00000F040F80020134908601348006813493B
:10CAD00088421ED210480068801C0F49086018E088
:10CAE00000200D4908600B4800680C49884204D2B8
:10CAF00008480068801C07490860002000F028F8FA
:10CB0000012000F02BF8002000F00AF8002000F0CF
:10CB100013F810BD500000204C000020FFFFFF7FE5
:10CB200001490880704700005A0000200149087040
:10CB3000704700005F000020014908807047000036
:10CB40005C00002001490870704700006000002070
:10CB50000149087070470000580000200149087022
:10CB6000704700005E0000200021014A11717047EB
:10CB700000600040002201494A7570470060004093
:10CB8000002201494A767047006000400021014AB6
:10CB900011727047006000400021014A1173704714
:10CBA000006000400021014A11747047006000409D
:10CBB0000021014A11757047006000400021014AC0
:10CBC0001176704700600040002201494A737047A7
:10CBD00000600040002201494A7470470060004034
:10CBE00010B51C4C1C49206888421ED106221B49E6
:10CBF000201DFBF766FB002817D11122184920469B
:10CC00000A30FBF75EFB00280FD1062215492046AB
:10CC10001B30FBF756FB002807D10622124920469D
:10CC20002130FBF74EFB00280DD000F04FFE0A48E4
:10CC30000E490860074814F0CCFA0C4A2821054830
:10CC400014F0F2FA04E0282221460848FBF715FB0D
:10CC500010BD0000000250007AA7A55A310700203D
:10CC6000370700202B070020250700208C2E0020EE
:10CC70000020084908700849087001200749087019
:10CC80000020074908700748074908600020074945
:10CC900008707047130700201207002015070020B6
:10CCA0001A0700202506000048070020240700205E
:10CCB00070B5044600BF9120604305460A2128460E
:10CCC000FBF744FA0546284670BD000070B5A8B0D1
:10CCD000054600240026A0216846FBF7E7FA00F08D
:10CCE00065FC1E490A6814216943505000211B4805
:10CCF0000268142068431018416018480268142024
:10CD000068431018816015484068002824D000BF8F
:10CD100017E06006060E282E00D316E00F480168C3
:10CD2000142060430858B1006A4650500B4801680F
:10CD30001420604308184168701C80001150601C6A
:10CD4000C4B20648007AA042E3DC00BF6200034898
:10CD5000694643680220984728B070BD042F002020
:10CD600030B5A9B000240025A02101A8FBF79EFA48
:10CD700000BF25E06006050E00F018FC1F490A6898
:10CD800014216143505000211C4802681420604364
:10CD9000101841601948026814206043101881601F
:10CDA000282D0BD215480168142060430858A900AB
:10CDB00001AA50500021681C80001150601CC4B2B0
:10CDC0000E48007AA042D5DC0C484068002813D0F9
:10CDD0000A48007A4000282806D30848282201A9DA
:10CDE00043680220984707E00448007A420003485D
:10CDF00001A943680220984729B030BD042F0020C4
:10CE000010B510F0B3F901287ED1FFF717FE554990
:10CE1000884216D20F20544948718871084680789C
:10CE2000002801D1052048704F488078052802D19C
:10CE300000204D49487000204B4908724872087024
:10CE400035E0FA204849487188714849088803F05C
:10CE500027FE4648807800280CD1434908700846D0
:10CE60004079C87008468079087100208870487041
:10CE700048721CE001203C4908700846407A0228AC
:10CE800005D1012048720020C87008710FE03648B3
:10CE9000407A00280BD10220334948720846407876
:10CEA000887008464079C8700846807908712E4815
:10CEB00080782D494978884213DD00202A49C870BE
:10CEC00008460079401C0871084600798979884233
:10CED00022DB00202449087108468078401E8870B3
:10CEE0001AE02148807820494978884214DA0020E5
:10CEF0001D4908710846C078401CC8700846C078B3
:10CF00004979884208DB00E01EE000201649C8701D
:10CF100008468078401C887014488078002803D127
:10CF20000120114908721BE010480088732803DBB8
:10CF300002200D49087213E00C48008870280FDCAD
:10CF40000020094908720BE00020074908700846D4
:10CF50004079C870084680790871002008724872CC
:10CF600010BD0000B80B0000BC09002080000020AC
:10CF70000020044988704870C870087108724872AF
:10CF800070470000BC090020002006490880887016
:10CF9000054988704870FA20C8700871002008722E
:10CFA0004872704780000020BC090020F8B50024BA
:10CFB00000250026002703F07BFC044603F08AFCD2
:10CFC000054610F0D3F801282ED105211A48FEF7A6
:10CFD000BFF8552804D1002018498870088027E040
:10CFE000012D04D1002015498870088020E001201F
:10CFF000124988701248844202DB201A84B200E091
:10D0000000240A212046FBF7B7F8052901DB601D43
:10D0100084B20C48844200DD04460A212046FBF716
:10D02000ABF80649088003E00020044988700880B6
:10D03000FFF7E6FEF8BD0000540800208000002045
:10D04000AA0A0000C60700001CB50020009001904D
:10D0500000F0ACFA0B49086000200B490968086031
:10D060000A48006800280CD00749096808680A21A6
:10D07000FBF76CF80090012269460520034B1B6802
:10D0800098471CBDE4070020D8070020E0070020D7
:10D090000020084948800849088008490880084954
:10D0A0000870084988720849088048800120087182
:10D0B00070470000300000202000002022000020E7
:10D0C000240000203808002028000020F8B503F0D4
:10D0D000D1FB074603F0E0FB0090FFF7C9FC0128F5
:10D0E00060D10521C548FEF733F8552802D00098D5
:10D0F000012807D10020C2490870C2490880C249EE
:10D10000887256E0BE480078002810D10120BC4942
:10D1100008703D462846E917890F091889030D0C48
:10D12000BA48854200DD0546B648058041E0B6486C
:10D13000807A4000B4490F520846867A0EE07000AB
:10D14000B1490D5A701E4000085A7100AE4A505243
:10D15000701E400011460D52701EC6B2002E08DD32
:10D160007000A949095A701E4000A74A105A81420E
:10D17000E5DBA548807A401CA34988720846807A7E
:10D18000052816DB002088720846C5882846E9175E
:10D19000890F09188D109D48854200DD0546994884
:10D1A000058006E000209649087096490880964957
:10D1B00088729448058896480088A84257DA9448AF
:10D1C0000088281A84B292480079012827D1904813
:10D1D0004088A0420BDA8E4840880A308C4948804B
:10D1E00008464088A04204DD0846448001E08848A3
:10D1F00044808748448803212046FAF7BDFF84B263
:10D20000192C00DA19248248008800198049088006
:10D2100008460088A84201DD08460580CDE07C482C
:10D220004088142805DD7A484088143878494880B9
:10D2300002E0002076494880754844880321204652
:10D24000FAF79AFF84B2192C03DA012070490871A9
:10D25000B3E06F480088A04205DD6D480088001BE0
:10D260006B490880A9E0002069490880A5E068486A
:10D270000088A84259DD66480088401B84B2644893
:10D280000079012827D162484088142805DD6048CC
:10D29000408814385E49488002E000205C4948809C
:10D2A0005B48448803212046FAF766FF84B2192CB4
:10D2B00003DA0220564908717FE0554800880019BA
:10D2C00053490880084600885049884275DD084661
:10D2D0004F49088071E04E484088A0420BDA4C4824
:10D2E00040880A304A49488008464088A04204DD08
:10D2F0000846448001E0464844804548448803216C
:10D300002046FAF739FF84B2192C00DA1924404874
:10D3100000882919884202DA3D4805804DE03C48E2
:10D320000088001B3A49088047E0394844880321B7
:10D330002046FAF721FF84B2192C3EDD344840889C
:10D34000142805DD3248408814383149488002E00D
:10D3500000202F4948802E48448803212046FAF7B0
:10D360000BFF84B22A480079012813D1192C03DA63
:10D3700002202749087120E0254800880019244927
:10D380000880084600882149884216DD0846204961
:10D39000088012E0192C03DA01201D4908710CE005
:10D3A0001B480088A04205DD19480088001B184969
:10D3B000088002E00020164908801648008850289E
:10D3C00004DC134800881349088016E010480088E0
:10D3D00010490988884204DD0D4800880D490880FD
:10D3E0000BE00B4800880B490988081A84B2502CBE
:10D3F00003DB0748008807490880F8BD540800206F
:10D40000240000202000002038080020E02E00002A
:10D41000280000202200002010B504466420444368
:10D42000A1212046FAF792FE0446204610BD0000D6
:10D4300010B501200F49087000200F4909680860E5
:10D440000D49096848600C490968886000F07EF958
:10D45000FFF7FAFDFFF784FC08480068002807D0B2
:10D4600001220548016808310020044B1B689847D9
:10D4700010BD0000B1070020AC070020A807002065
:10D4800010B5184800681849884229D11748006823
:10D49000002804D0154800688047154908701548D1
:10D4A0000068002804D013480068804712490870BB
:10D4B00012480068002804D01048006880471049CE
:10D4C000088010480068002805D00E480068804792
:10D4D0000D49088002E00D480B49088000F078F8FB
:10D4E00010BD0000BC0700207856341298070020B9
:10D4F000B00700209C070020B2070020A0070020F2
:10D50000B4070020A4070020B60700201027000061
:10D5100010B50023174C2360174C2370174C237051
:10D52000174C2370174C2380174C2380174C237003
:10D53000174C13682360174C53682360164C93688C
:10D540002360164CD3682360154C136923600028B0
:10D550000CD0144B1860134C0B682468A360002394
:10D56000104C246823600F4C246863600E4B014C00
:10D57000236010BDBC070020B8070020B0070020C2
:10D58000B2070020B4070020B6070020B107002032
:10D59000980700209C070020A0070020A407002077
:10D5A000A8070020AC070020785634120548006810
:10D5B0000549884203D1054800688068704700200B
:10D5C000C043FBE7BC07002078563412AC070020AC
:10D5D00070B50024002500263048007801285CD171
:10D5E0002F480078002858D12E480078012854D1BF
:10D5F0002D4805882D490988694308462C49FAF7C2
:10D60000A5FD85B2E1200001854207D819216943B3
:10D6100008460921FAF79AFD044600E0244C254803
:10D6200000680068001923490968086021480068FB
:10D630000068204909684968884207D31D48006886
:10D6400000681C4909684968461A0AE019480068D8
:10D6500040680021C943081A16490968096840183A
:10D66000461C1548864218D3344601462046FAF730
:10D670006DFD04460F48006841680F486043081874
:10D680000C490968486001200C4908700948006885
:10D690008068001907490968886070BDB0070020DC
:10D6A000B1070020B2070020B4070020B607002011
:10D6B00010270000AC070020A0860100B80700205A
:10D6C00000220C4B1A600C4B0A681A600B4B4A681C
:10D6D0001A600B4B8A681A600A4BCA681A600A4BB8
:10D6E0000A691A60002801D0084A1060084A014BF4
:10D6F0001A607047BC070020980700209C07002094
:10D70000A0070020A4070020A8070020AC070020E5
:10D710007856341210B50A48006800280ED009481F
:10D72000007801280AD10020064908700122064825
:10D73000016808310020024B1B68984710BD0000AB
:10D74000A8070020B8070020AC0700201CB5002067
:10D75000009001900024FFF729FF04460E4800685E
:10D76000046000200C49096848600B49096888601A
:10D770000A48006800280DD007480068006800903B
:10D780000548006840680190022269460120034B69
:10D790001B6898471CBD0000C0070020C40700207C
:10D7A000F8B505460C4616460027002D17D00E4842
:10D7B0000560FFF7FBFE07462068B84203D90A4818
:10D7C0000068076003E008492068096808600649A6
:10D7D0006068096848600449A0680968C86003482F
:10D7E000066000F005F8F8BDC0070020C40700205F
:10D7F00070B500240025FFF7D9FE04460F480068E5
:10D800000068A04200D903E00C4800680068251AAF
:10D810000A48006840684019084909688860074854
:10D820000068806805490968C968884205D90348C5
:10D830000068C06801490968886070BDC0070020A1
:10D840000148006880687047C0070020002801D0A8
:10D85000024A1060024A116070470000C0070020B1
:10D86000C40700200549002005E00A1D135C044A96
:10D870001354421CD0B22028F7DB7047000650003A
:10D88000B82E0020014610480268142048431018A2
:10D8900082680D480368142048431818C068824203
:10D8A0000BD909480268142048431018C26806487A
:10D8B0000368142048431818826003480268142043
:10D8C0004843101880687047042F00200021002072
:10D8D00005E01A4A135C1A4A1354421CD0B20628B7
:10D8E000F7DB1121002006E0164A135C144A921D52
:10D8F0001354421CD0B28842F6DB002006E0124AE4
:10D90000135C0F4A17321354421CD0B20628F6DBC0
:10D91000002006E00D4A135C094A1D321354421CD4
:10D92000D0B20628F6DB002005E00023044A2332AB
:10D930001354421CD0B20128F7DB70473107002096
:10D94000902E0020370700202B07002025070020FD
:10D9500038B5044600200090009401226946052055
:10D9600000F06AFC38BD000008B5002000900122DC
:10D970006946062000F020FC684600780F490873CD
:10D980006846407848730846007B0D4948730B4849
:10D99000407B88730948807BC8730848C07B087443
:10D9A00000200873074908600749086007490860B4
:10D9B000074908600749087008BD0000402800209A
:10D9C000C809002084000020880000208C0000206E
:10D9D000900000209400002008B500200090012253
:10D9E0006946062000F0E8FB684600781249087393
:10D9F0006846407848730020104908604860087203
:10DA0000487288720C48007B48730B48407B8873CF
:10DA10000948807BC8730848C07B087400200873DD
:10DA20000749086007490860074908600749086016
:10DA30000749087008BD000040280020C8090020E0
:10DA400084000020880000208C000020900000202E
:10DA50009400002038B5002400250020009001210A
:10DA6000FA48FDF775FB55280AD002F077FFF84910
:10DA7000487302F087FFF64988730120087308E0B5
:10DA8000F448007BF2494873F248407B88730020D9
:10DA900008730621ED48FDF75BFB552830D002F0F6
:10DAA000A5FF002808D002F0A1FF401C002803D0E9
:10DAB0000120E749087502E00020E549087502F0F9
:10DAC00077FF002808D002F073FF401C002803D025
:10DAD0000120DF49C87402E00020DD49C87402F06B
:10DAE00085FF002808D002F081FF401C002803D0E9
:10DAF0000120D749087507E00020D549087503E0E3
:10DB00000020D349C8740875D148407B00282BD128
:10DB1000D1490860D1480068D149884208D8CF4827
:10DB20000068401CCD4908600020C94948736CE07A
:10DB3000C848007B022812D0C648007B03280ED0BC
:10DB40000121C248FDF704FB552803D00320C0493A
:10DB500048735AE0BF48007BBD49487355E0BD4853
:10DB6000007BBB49487350E0B948407B01282CD169
:10DB70000020BA490860B8480068B949884208D806
:10DB8000B5480068401CB44908600120B04948739A
:10DB90003BE0B048007B022812D0AE48007B03284F
:10DBA0000ED00121A948FDF7D3FA552803D0032050
:10DBB000A749487329E0A748007BA549487324E09A
:10DBC000A448007BA24948731FE0A148407B02287B
:10DBD00005D10020A14908609F49086015E09C48D4
:10DBE000407B032808D100209C4908609A490860BE
:10DBF00003209749487308E0002098490860964937
:10DC000008609448007B924948739148807B0028C3
:10DC10002BD194490860944800689149884208D8FB
:10DC200091480068401C904908600020884988732A
:10DC30006CE08848407B022812D08648407B03284D
:10DC40000ED001218148FDF783FA552803D0032027
:10DC50007F4988735AE07F48407B7D49887355E04F
:10DC60007C48407B7A49887350E07948807B012862
:10DC70002CD100207C4908607A48006878498842A5
:10DC800008D878480068401C76490860012070492F
:10DC900088733BE06F48407B022812D06D48407B80
:10DCA00003280ED001216948FDF752FA552803D008
:10DCB00003206749887329E06648407B644988737C
:10DCC00024E06448407B624988731FE06048807BA1
:10DCD000022805D10020644908606249086015E007
:10DCE0005B48807B032808D100205F4908605D49BC
:10DCF000086003205649887308E000205A490860EC
:10DD0000584908605348007B514988735048407B0C
:10DD10005049097B884205D14D48807B4D49497B5C
:10DD200088424FD04A48407B4A49097B884202D00A
:10DD300001204749C8734648807B4649497B884251
:10DD400002D00120424908744148407B022803D098
:10DD50003F48407B032816D13D48407B3D49097B25
:10DD6000884210D03A48407B3A4908730846017B04
:10DD7000684601703748417B684641700122694618
:10DD8000062000F059FA3248807B022803D0304840
:10DD9000807B032816D12E48807B2E49497B884200
:10DDA00010D02B48807B2B4948730846017B68467E
:10DDB00001702848417B684641700122694606206F
:10DDC00000F03AFA02F0D4FD044602F0E7FD054601
:10DDD000FEF74EFE01287BD101211C48FDF7B8F962
:10DDE000552807D100201A49087248720860486017
:10DDF0008872BAE0FF2C01D0FF2D78D1FF2C3FD1E3
:10DE0000FF2D3DD0002012490872012048721748AA
:10DE1000086017486843486048686621FAF796F931
:10DE20000B494860084640681249884202D90846B2
:10DE30000749486003F0E4F8112803DB03F0E0F839
:10DE4000192819DD0120024988728EE0540800204B
:10DE5000C8090020402800208800002084000020FD
:10DE600070170000900000208C000020DE030000EE
:10DE7000BE0A0000AC26000000205D49887274E0F4
:10DE8000FF2C2BD0FF2D29D10120594908720020E9
:10DE900048725848486058486043086008686621DE
:10DEA000FAF754F952490860084600685349884215
:10DEB00002D908464E49086002F09EFF112803DB94
:10DEC00002F09AFF192805DD0120494988724CE0CB
:10DED00086E00CE000204649887246E04748444905
:10DEE0000860486000208872087248723DE0012096
:10DEF0003F490872487240486043086008686621DC
:10DF0000FAF724F93A490860084600683B49884214
:10DF100002D90846364908603748684334494860A2
:10DF200048686621FAF712F93149486008464068A6
:10DF30003249884202D908462D49486002F05CFF08
:10DF400011280BDB02F058FF192807DC03F058F802
:10DF5000112803DB03F054F8192803DD01202449BC
:10DF6000887202E00020224988722148407B002804
:10DF700002D11F49C87315E01D48407B012802D11A
:10DF80001B49C8730EE01A48407B022802D1184989
:10DF9000C87307E01648407B032803D11449C873AF
:10DFA000164808601248807B002802D11049087486
:10DFB0001DE00F48807B012802D10D49087416E04E
:10DFC0000B48807B022802D1094908740FE00848F9
:10DFD000807B03280BD1064908740848486006E096
:10DFE000002003490872487208604860887238BD92
:10DFF000C8090020DE030000BE0A0000AC260000B5
:10E00000FFB583B006460D46174600240020029057
:10E0100000BF1420784380190190002E57D001983A
:10E02000002854D02B4806602A49069848600846C4
:10E03000077200BF45E0FFF7B9FA029020012958A6
:10E040000298814204D820012858401C002806D19B
:10E05000204902980A6814216143505006E02001CB
:10E0600029581C48026814206043115020014019AF
:10E070004068401C002807D100211648026814207F
:10E0800060431018416008E02001401941681148C0
:10E090000268142060431018416020014019816813
:10E0A0000C480268142060431018C1602001401918
:10E0B000017B084802681420604310180161601C4D
:10E0C000C4B20448007AA042B5DC00F005F807B0FD
:10E0D000F0BD0000042F002070B5002400250026AC
:10E0E000FFF764FA054600BF4EE02A480168142095
:10E0F00060430858A84239D8264801681420604374
:10E1000008582E1A234801681420604308184068F4
:10E1100081192048026814206043101881601D484E
:10E12000016814206043081881681A4802681420A6
:10E1300060431018C068814224D916480168142031
:10E14000604308180069002803D02046FEF7BEFD92
:10E1500018E010480168142060430818C1680D4891
:10E16000026814206043101881600BE009480168C0
:10E17000142060430818406806490A681421614366
:10E1800051188860601CC4B20248007AA042ACDC1E
:10E1900070BD0000042F002010B500BF14244C43B4
:10E1A0002318002805D0002B03D0024C20606260A9
:10E1B000217210BD042F0020F8B505460E46144606
:10E1C0002B0012F041FB0705131A313121293100D0
:10E1D0001748FAF7C9FC174908701548FAF77EF88E
:10E1E00007466421F9F7B2FF30601EE0A004020C7C
:10E1F00031462020FAF7B2FD17E0A004020C3146A8
:10E200006020FAF7ABFD10E0A004020C3146FF20BD
:10E210002130FAF7A3FD08E06004020C3146FF202C
:10E220004130FAF79BFD00E000BF00BF0020F8BDC1
:10E2300032280020CD00002070B505460E46144659
:10E240002B0012F001FB07051D243A3A2B323A004D
:10E250003068002802D1FAF725FB10E0642231680B
:10E26000514308461649FAF743F80020154908704B
:10E27000012264211248FAF7DFFD124908701DE0FF
:10E28000A004020C31462020FAF726FF16E0A00475
:10E29000020C31466020FAF71FFF0FE0A2B23146B0
:10E2A000FF202130FAF718FF08E06004020C314625
:10E2B000FF204130FAF710FF00E000BF00BF70BD43
:10E2C00024280020CC00002000B5AFB050211BA8AE
:10E2D000F9F7ECFF00201A90142115A8F9F7E6FFD2
:10E2E00000201290139014901190402101A8F9F78A
:10E2F000DDFF002000904849086001221BA9FFF7BC
:10E300005BFF1B98401C002801D11A9001E01B986C
:10E310001A904248159042481690424817900020A3
:10E3200018904148199015AA1AA94048FFF7F0F82B
:10E3300002221CA90120FFF73FFF1C98401C002867
:10E3400001D1129001E01C9812901C98401C0028EA
:10E3500001D1139001E01D9813903548149012A933
:10E360003448199AFFF71CFA08221EA90220FFF769
:10E3700023FF1E98401C002801D1019001E01E9847
:10E3800001901F9802902C48039001206946087460
:10E39000801E059029490791012101A80177881E57
:10E3A000099026490B91012109A80173881E0D903F
:10E3B00022490F9101210DA80173042201A92048CF
:10E3C000199BFFF71DFE01221BA90520FFF7F4FE94
:10E3D0001B98401C002807D101201A49886001229F
:10E3E00008310520FFF728FF01221BA90620FFF7AF
:10E3F000E3FE1B98401C002808D1002168460170EC
:10E400004170012269460620FFF716FF0E480249B7
:10E4100008602FB000BD0000D000002071CA0000CD
:10E4200065CA000049CA000039E20000B827002090
:10E4300076841E00C42700200F2700009F8601005D
:10E44000D427002040280020A33AA55A00B585B063
:10E4500014216846F9F72AFF00200F4908600F4889
:10E4600000900F4801900F480290002003900E4842
:10E47000049069460D48FFF723F90D480499FFF70A
:10E48000E5F904210B48049AFFF786FE0A48024981
:10E49000086005B000BD0000D000002071CA000077
:10E4A00065CA000049CA000039E20000B827002010
:10E4B000C4270020D4270020A33AA55A00200C49E5
:10E4C00008800C4908800C49088001200B4908701D
:10E4D00000200B4908730B4908804880012008710F
:10E4E00000200749488008800749086070470000FD
:10E4F000380000203A0000204000002042000020A8
:10E5000044080020440000203C000020F8B502F040
:10E51000EBF9064602F0F2F90746FEF7A9FA0128E0
:10E5200065D10521AB48FCF713FE552807D1002023
:10E53000A9490870A9490880A94988805FE0012F8E
:10E5400007D10020A4490870A4490880A449888004
:10E5500055E0A1480078002808D101209E490870A4
:10E5600035460A2068439D49088048E09C48007B66
:10E5700042009B48801D8652801F047B11E0610091
:10E580009748801D455A601E41009548801D415A9C
:10E5900062008152601E41009148801D4552601EFC
:10E5A000C4B2002C0ADD61008D48801D415A601EF6
:10E5B00042008B48801D805A8142E0DB8848007B06
:10E5C000401C874908730846007B032807DB0020AE
:10E5D0000873084605890A206843804908807F48F7
:10E5E00000887F49888001207B49087007E000206F
:10E5F0007949087079490880794908738880774893
:10E6000000887849086074480078002815D00846CA
:10E6100000686C21484373490860642171480068B0
:10E62000F9F794FD6F490860084600686E49884212
:10E6300006D908466B49086002E000206949086075
:10E640006848006869490988884203D265480068BB
:10E650000F2804D263480088644908800AE06348B0
:10E66000008860490968401A0F2803D35D48008874
:10E670005E4908805A480088401C5949088008466D
:10E6800000880A282CDB0020088059480088574958
:10E690000988884203DA01205649087108E0544885
:10E6A000008852490988884202DD022051490871D8
:10E6B00050480079012840D14C4800884C490988CD
:10E6C00088420DDB4948018849480088FF30913075
:10E6D000814206DD46480088FF3073304449088097
:10E6E00077E042480188424800889630814205DD43
:10E6F0003F48008878303E4908806AE03B480188FE
:10E700003B4800883230814205DD394800881E30A0
:10E71000374908805DE035480188354800880A306F
:10E72000814205DD324800880A303149088050E0D6
:10E730002E4800882E4908804BE02E480079022898
:10E7400047D12A4800882A490988884239DA274867
:10E750000088FF30913026490988884206DA24482B
:10E760000088FF387338224908802AE01F48008853
:10E7700096301F490988884205DA1D480088783894
:10E780001B4908801DE01948008832301849098863
:10E79000884205DA164800881E381549088010E0BE
:10E7A000124800880A3012490988884205DA104860
:10E7B00000880A380E49088003E00C4800880C499C
:10E7C00008800B4800880849884202DB084608494F
:10E7D0000880F8BD540800204200002038000020C6
:10E7E000440800203C000020C60700004000002034
:10E7F0003A00002044000020002008490880084911
:10E8000008800849088048800120087100200649D6
:10E810004880088005490860704700003A000020E1
:10E820004000002044000020440800203C0000205C
:10E83000002004490870044908700021034801764B
:10E84000704700009500002096000020400A00203C
:10E8500070B500250024FEF70BF9012863D10321D0
:10E860003448FCF775FC552808D10020324908705F
:10E870003249087000213248017659E02F4800786B
:10E88000002807D102F0D0F82B49087001202B494D
:10E8900008704DE001202949087002F0C5F82849A8
:10E8A000097E8900264A603A50502548047E10E0CF
:10E8B000A000234960390D5C601E80000858A1004B
:10E8C0001F4A603A5050601E800011460D50601E75
:10E8D000C4B2002C0ADDA000194960390958601E35
:10E8E0008000174A603A10588142E1D31448007EF4
:10E8F000401CC1B212480176007E1E2818DB0021A0
:10E900000F48017601466039896B0246603AD26B46
:10E9100089180246603A126C88180321F9F716FC30
:10E920000549087004E00020034908700349087095
:10E9300070BD0000540800209500002096000020C3
:10E94000400A0020F0B5A9B004460E460025002775
:10E9500000202890A0216846F9F7A8FCFEF726FEC3
:10E9600026490A6814216143505024480168142044
:10E9700060430818C068B0420CD2204801681420D7
:10E9800060430818C1681D480268142060431018CD
:10E99000416005E01948016814206043081846608A
:10E9A00016484068002826D0002517E06806070EA4
:10E9B000282F00D316E01148016814206843085836
:10E9C000B9006A4650500D48016814206843081881
:10E9D0004168781C80001150681CC5B20748007A55
:10E9E000A842E3DC00BF6A0004486946436802208D
:10E9F000984701202890289829B0F0BD042F0020C6
:10EA000010B500F0F9FD00F0D7F810F03DFE00F071
:10EA10000DFB00F001F810BD70B541480078912859
:10EA200000D070BD00F0BEF8012876D13D480088C6
:10EA30003D49088008468078F021884320303A49D3
:10EA4000887008468078000900013549097A09076D
:10EA5000090F0843344988703148807A401E304994
:10EA6000887208460089401C088108460089C988C8
:10EA7000884216DA08202C49887200240EE02848C3
:10EA800041882848001D415C2748C01C0155244886
:10EA90004088401C22494880601CC4B2072CEEDB31
:10EAA0002DE01F4800891E49C98888421CD11C4896
:10EAB00000791B498978401AC5B2681C1A498872C6
:10EAC00000240EE0164841881648001D415C164897
:10EAD000C01C015512484088401C11494880601CE8
:10EAE000C4B2AC42EEDB0AE000F012FD00200C499B
:10EAF00008700C490888092100F0B8F991E7012055
:10EB000000F0C8FC084A917A1088921C00F070F955
:10EB100005490888002100F0C1F800BF81E7000026
:10EB2000402C0020DC2B00206C2B00201B49097E90
:10EB3000002932D01949897E0C225143174A515A73
:10EB4000174A118000200CE01449897E0C225143A1
:10EB5000124A8918891C0A5C1149891C0A54411CF3
:10EB6000C8B20828F0DB0D49897E0C2251430B4ABC
:10EB70008918897A0A4A91720121D1720749097E5E
:10EB8000491E064A11761146897E491C9176114626
:10EB9000897E022901DB002191767047382B002005
:10EBA000602B00200349487B012802D10021014A43
:10EBB00051737047502C002010B53348406800282E
:10EBC00061D13148007B030011F03EFE0759051268
:10EBD000212E3D4A59002D480078002807D00020FA
:10EBE0002A4908702A490888012100F03FF947E0C6
:10EBF00026480078002809D00020244908702549BB
:10EC00004A8808880123091D00F040F938E01F48B0
:10EC10000078002807D000201C4908701C4908888B
:10EC2000022100F023F92BE018480078002809D0D1
:10EC300000201649087017494A8808880923091DC9
:10EC400000F024F91CE011480078002807D00020CB
:10EC50000E4908700E490888092100F007F90FE0F5
:10EC60000A480078002809D000200849087009499E
:10EC70004A8808880323091D00F008F900E000BF56
:10EC800000BF00F045FC10BD502C0020402C00209F
:10EC9000DC2B0020782B00207047000070B5044664
:10ECA0000D4634480088A04263D1002D61D132481E
:10ECB000007822284ED004DC20283DD0212856D1CF
:10ECC00041E0902802D0912851D115E02A48C0880F
:10ECD00001280AD100202849087000F019FC2749B2
:10ECE0000888002100F0C2F805E0032000F0D2FB04
:10ECF000A020214908703BE01F4800891E49C988AF
:10ED000088420AD100201C49087000F001FC1B4910
:10ED10000888002100F0AAF80DE01748807A002842
:10ED200006D000F0F5FB1449087B00F095FB02E0EB
:10ED3000032000F0AFFB1BE0062000F0ABFB11202E
:10ED40000D49087014E0062000F0A4FB11200A49C8
:10ED500008700DE000200849087000F0D9FB084950
:10ED60004A8808880923091D00F090F800E000BFD8
:10ED700000BF70BD542B0020402C0020DC2B002055
:10ED8000782B002070B50346184C247E022C00DB43
:10ED900070BD164C647E0C256C43144D2B53002023
:10EDA0000AE0155C114C647E0C2674430F4EA419C6
:10EDB000A41C2554441CE0B28842F2D30B4C647E60
:10EDC0000C267443094EA419A1723446247E641C97
:10EDD00035462C762C46647E641C6C762C46647E0C
:10EDE000022C01DB00246C7600BFD1E7382B002019
:10EDF000F0B585B007460D4616461A480780002430
:10EE000006E031781748801C0155761C601CC4B29E
:10EE1000AC42F6DB2C4605E0AA211248801C0155C5
:10EE2000601CC4B2082CF7DB0E4800880190082152
:10EE30006846C1720021417201720170002406E02F
:10EE40000848801C015D03A80155601CC4B2082C51
:10EE5000F6DB69460448FCF78CFA01200149887208
:10EE600005B0F0BD542B00209055044070B5044609
:10EE70000D462946204610F029FB70BD70B50446AA
:10EE80000D462946204610F02FFB70BDF8B504460C
:10EE90000D4616461F463B4632462946204610F090
:10EEA00024FBF8BDF8B507460E4615465C480078C9
:10EEB000002804D009213846FFF7D8FFF8BD002DFF
:10EEC00001D0602D04DD09213846FFF7CFFFF5E7BB
:10EED000544807804580002406E031785148001DE1
:10EEE0000155761C601CC4B2AC42F6DB00204C49D4
:10EEF000487008468580FF2088727F200873084686
:10EF0000808808282EDA0120C8800846808848803A
:10EF100001200881434800884349088008468078DA
:10EF2000F021884340498870084680780009000134
:10EF30003B4909790907090F08433B49887038485C
:10EF40000079401C8872002407E03648001D015DEE
:10EF50003548C01C0155601CC4B231488088A042AD
:10EF6000F3DC4AE00721681CF9F706F9002907D00D
:10EF7000072128460830F9F7FFF82949C88005E03D
:10EF80000721681CF9F7F8F82549C88006202449AC
:10EF900048800120088123480088234908800846CA
:10EFA0008078F021884310301F49887008468078A7
:10EFB000000900011A4989880905090F08431A49FF
:10EFC000887008464088FF210902884314498988CF
:10EFD0000902FF2212021140084313494880082009
:10EFE0008872002407E00F48001D015D0E48001DD7
:10EFF0000155601CC4B2062CF5DB012000F04AFA72
:10F00000094A917A1088921CFFF7F2FE9020044979
:10F010000870054908880021FFF740FE00BF4DE752
:10F02000402C0020DC2B00206C2B002010B5FFF7BB
:10F030007DFD1448C07A002822D01248807800094B
:10F04000002806D0012807D002280AD0032810D1B2
:10F050000CE000F0A7F90FE000F09EF800F066FA6F
:10F060000AE000F011F800F061FA05E000F000F9A4
:10F0700002E0FFF711FE00BF00BF00200149C87287
:10F0800010BD0000602B002010B53F48007811280B
:10F0900000D010BD3D4800883D49884200D0F8E7C7
:10F0A0003A4880780007000F3749097A0907090FA5
:10F0B00088420CD000203449087000F029FA354904
:10F0C0004A8808880423091DFFF7E0FEE1E72E487F
:10F0D0000089401C2C4908810846807A401E8872AD
:10F0E00008460089C98888421BDA2848807A08289F
:10F0F00000D0CEE700240EE02448C01C015D224869
:10F1000042882448001D81541F484088401C1E49E5
:10F110004880601CC4B2072CEEDB062000F0BAF970
:10F1200030E01948808818494988401A1749897A77
:10F13000884203DA1548807A082800D0A9E700241D
:10F140000EE01248C01C015D0F4842881148001DA6
:10F150008154601CC4B20C484088401C0A49488055
:10F1600009484088084989888842EADB0020064926
:10F17000087000F0CDF907494A8808880023091D66
:10F18000FFF784FE00BF84E7402C0020602B0020A6
:10F1900014070000782B002070B5314800788021DA
:10F1A0000840802800D170BD2E4800882E49884232
:10F1B00000D0F8E72B48807A082800D0F3E72948E8
:10F1C000807805072D0F2D0226484088000A054348
:10F1D000082D00DAE7E70020214948700620488022
:10F1E0000846858001200881082088720020C872A6
:10F1F0008988481C0721F8F7BFFF002909D0184962
:10F200008988084608300721F8F7B6FF1449C880F6
:10F2100007E013498988481C0721F8F7ADFF10491A
:10F22000C88010480088114908800846458000249D
:10F2300007E00C48001D015D0C48001D0155601CD5
:10F24000C4B2062CF5DB042000F024F91020044998
:10F250000870064A51881088FFF710FE00BFA2E729
:10F26000402C0020602B002014070000782B002089
:10F2700010B548480078A02808D046480078912862
:10F2800004D044480078A12800D010BD424800882E
:10F29000424988420AD0424908880921FFF7E6FD21
:10F2A00000F036F900203B490870EEE73A48807AD2
:10F2B00008280AD03A4908880921FFF7D7FD00F04D
:10F2C00027F9002033490870DFE7334880780007CA
:10F2D000000F002804D001282DD002284BD136E0A1
:10F2E0002C484078002800D050E02B48C0780028F7
:10F2F00003D101202749487003E02748C0782549F9
:10F3000088722448007891280BD02348007900287F
:10F3100003D101201F49087303E01F4800791D49EC
:10F32000087391201B49087000F0F2F81949087B16
:10F3300000F092F82AE017484078002800D025E035
:10F34000A12014490870032000F0A4F81EE0114821
:10F350004078002800D019E00E480078A02809D194
:10F360000F4908880821FFF781FD00F0D1F800203F
:10F37000084908700AE00A4908880521FFF776FD68
:10F3800000F0C6F800200349087000BF00BF00BFAE
:10F390007BE70000402C0020602B002014070000B9
:10F3A000DC2B002010B528480078802108408028F8
:10F3B00000D110BD24480078002805D023480088DB
:10F3C0002349884200D0F4E72048807A1F49897891
:10F3D0000907090F884203DD1C48807A082800D0FD
:10F3E000E7E71A4880780007000F002805D0174883
:10F3F00080780007000F072800DDDAE7134800884F
:10F4000014490880114880780007000F48800024C4
:10F4100007E00E48C01C015D0E48001D0155601C30
:10F42000C4B20C484088A042F3DC002006490870B2
:10F4300000F06EF807494A8808880023091DFFF785
:10F4400025FD00BFB5E70000402C0020602B002008
:10F4500014070000782B00207F2805DC7D21C900DF
:10F4600041430A4A91600DE0F12808DBF92806DCE7
:10F470000107090F64225143044A916002E00449E4
:10F48000024A91600221014A51737047502C0020BA
:10F4900018F0010000B5030011F0D6F90729050B9B
:10F4A00011171D2329000121144A117314495160B9
:10F4B00022E00221114A1173114951601CE003211D
:10F4C0000E4A11730F49516016E004210B4A117363
:10F4D0000D49516010E00521084A11730021516067
:10F4E0000AE00621054A11730849516004E0002131
:10F4F000024A1173516000BF00BF00BD502C0020B4
:10F50000A8610000F824010028230000F04902004F
:10F510000020014908737047502C002002490988D7
:10F520000918014A11807047502C002010B52E4850
:10F530000078102818D12D48408860280ADD2C4812
:10F54000807800090001801C294988702220264902
:10F55000087025E026488078000900012449887059
:10F560002020214908701BE01F480078112816D17F
:10F570001D48807A002800D010BD1B484078002824
:10F5800000D0F9E7082018498872194880780009E6
:10F5900000011749887020201349087000E0EBE74C
:10F5A00014481349088008468078F0218843303099
:10F5B0000F4988700846C0780020C8700846007956
:10F5C00014200871032088720220FFF763FF084AA5
:10F5D000917A1088921CFFF70BFC054908880021DE
:10F5E000FFF75CFB00BFC7E7402C0020782B002012
:10F5F0006C2B002094070000244A118852888A420C
:10F6000042D0224A52888A4204DA204A52888A1A10
:10F6100090B207E01D4A52880023DB439A1A521C1D
:10F62000521890B2194A5180127B002A10D0174A02
:10F630005268002A0CD0154A5268824205D9134AF2
:10F640005268121A114B5A6002E000220F4B5A60A6
:10F650000E4A527B022A17D10C4A9268002A0CD01B
:10F660000A4A9268824205D9084A9268121A074BE0
:10F670009A6002E00022054B9A60044A9268002AD0
:10F6800002D10122014B5A7370470000502C002018
:10F6900010B506F0E3F810BD00BF704710B5044682
:10F6A0008020204301460320400205F091FF10BD59
:10F6B00010B510210320400205F08AFF10BD0000A4
:10F6C00010B50224024805F0D3FF0446204610BDC1
:10F6D0000106000010B50021014805F079FF10BDBA
:10F6E0000106000010B50446802020430146024870
:10F6F00005F06EFF10BD00000106000010B51021DE
:10F70000014805F065FF10BD0106000030B5034655
:10F710000C46002101250D48834201D0002B01D168
:10F72000022030BD012A01D10120FAE7002108E0C2
:10F73000C8002058984202D100252846F1E7481C0D
:10F7400081B29142F4DB2846EBE70000FFFF0000A6
:10F75000002000BF14E00021C200134B9950C200EA
:10F76000D2189180C200114B9950C200D2189180DA
:10F77000C2000F4B9950C200D2189180411C88B230
:10F780004828E8DB0B490C4A11600C495160002104
:10F7900091600B4911610B49D16000210A4A118027
:10F7A0000A4A117070470000901F0020D0210020ED
:10F7B00010240020710C01007C1F00200D0D0100A1
:10F7C000B70D0100A90D0100BE000020C2000020FD
:10F7D000F0B585B00646674F384603900290002585
:10F7E000002400200190009063480068002803D0A6
:10F7F00061490868804707465F484068002803D091
:10F800005D494868804703905B488068002803D0C2
:10F81000594988688047029057480069002803D0FA
:10F8200055490869804700905348C068002803D0B4
:10F830005149C86880470546482D00DD4825009895
:10F84000002876D0002D74DD4C480088A8420BDAE1
:10F850002B463A4649494A48FAF746FF2B4647495C
:10F860004748039AFAF740FF44480088002833DDF0
:10F8700042480088A84202D1002040490880002464
:10F8800015E0E0003F490858E1003D4A51588842E0
:10F890000BD0E00011460858E1003A4A5050E00011
:10F8A00011460858E100384A5050601C84B2AC42FE
:10F8B000E7DB0120354908702C460BE00020E10011
:10F8C000314A5050E1002F4A5050E1002C4A50502C
:10F8D000601C84B2482CF1DB2B4800682549884223
:10F8E00046D0294880882A49884205DA26488088F7
:10F8F0008019254988803BE00020234988800846FC
:10F9000000680190012D33DD002408E0601CC00078
:10F910001D490858E1001C4A5050601C84B2681E02
:10F92000A042F3DC691EC900174A019850501FE03D
:10F93000FFE7002015490870002414E00020E100D2
:10F94000114A5050E10089188880E1000C4A50505B
:10F95000E10089188880E1000A4A5050E1008918C6
:10F960008880601C84B2482CE8DB002003490880B2
:10F9700005B0F0BDFFFF00007C1F0020BE0000208E
:10F98000D021002010240020901F0020C200002061
:10F99000881300002E480078401C2D4908702D481F
:10F9A0000078401C2B4908702B480078401C2A49DD
:10F9B00008702A480068401C28490860084600680A
:10F9C000FF219131884202D9002024490860204853
:10F9D0000078C82802D900201D4908701D48007809
:10F9E000842802D900201B4908701B480078502841
:10F9F00002D9002018490870194818490968405C64
:10FA000018490870184812490978405C174908706D
:10FA1000174810490978405C1649087016480E4985
:10FA20000978405C15490870154809490978405C17
:10FA300014490870144806490978405C1349087055
:10FA4000134803490978405C124908707047000068
:10FA50005707002058070020590700205C070020A6
:10FA6000AB1D0200500700203B1F02005107002081
:10FA700003200200520700204F21020054070020FB
:10FA800087200200530700209F2102005507002015
:10FA9000672202005607002010B58200054BD218DD
:10FAA000525C012A04D100228300024C1B195A54D3
:10FAB00010BD0000BC2A002010B50446204600F00E
:10FAC00055FA204600F002F810BD000010B50446BB
:10FAD000B348007800287DD1B2480088B2498842F6
:10FAE00078DAB248007800284FD0B1480078002872
:10FAF00003D0AC480088AF490880AF4800780028A0
:10FB000018D1A8480188AB4800880A30814206D342
:10FB10000120A9490870A3480088A6490880A14887
:10FB20000088A449098888421CDA9E480088A149B7
:10FB3000088017E09F4801889A4800880A3081426F
:10FB400006D300209C49087096480088994908808F
:10FB50009448008897490988884203DD91480088C5
:10FB60009449088094480078002858D19348007838
:10FB7000042803D08E480078002807D089480088E0
:10FB8000822803DA05208D490870A3E08B480078AD
:10FB9000032803D086480078002809D081480088CF
:10FBA000FF211931884203DA04208449087091E06A
:10FBB00082480078022803D07D48007800280AD0C7
:10FBC00078480088FF21AF31884204DA03207B495E
:10FBD00008707FE0E2E079480078012803D074489B
:10FBE0000078002809D06F480088AF21890088423A
:10FBF00003DA0220714908706CE070480078002830
:10FC000003D06B480078002864D066480088E12162
:10FC1000890088425EDA0120684908705AE0664827
:10FC20000078012856D165480078012803D0604843
:10FC30000078002809D05B480088E12189008842CB
:10FC400003DB00205D49087044E05C48007802282E
:10FC500003D057480078002809D052480088AF21C7
:10FC60008900884203DB01205449087032E0534880
:10FC70000078032803D04E480078002809D049486E
:10FC80000088FF21AF31884203DB02204B49087016
:10FC900020E04A480078042803D04548007800282E
:10FCA00009D040480088FF211931884203DB032036
:10FCB000424908700EE041480078052803D03C48CE
:10FCC0000078002806D037480088822802DB04200C
:10FCD0003A490870FCF7B2FE3349643988425DD373
:10FCE0003748006800193649086031480078002814
:10FCF00008D000202E490870314908602F4800784C
:10FD00003049087000F0A4FD00281FD12C4800687D
:10FD10002D49884239D300202949086029480078B4
:10FD200026490978884205DA26480078401C25498A
:10FD300008702AE02348007820490978884224DDA9
:10FD400020480078401E1F4908701EE01C480068CB
:10FD50001E49884219D300201949086019480078C3
:10FD600016490978884205DA16480078401C15497A
:10FD700008700AE01348007810490978884204DDC9
:10FD800010480078401E0F4908700E4800780B4953
:10FD90000978884202D100200949086010BD00009E
:10FDA0000B000020020000201C0C000012000020AC
:10FDB00008000020040000200A00002006000020A7
:10FDC0001800002007000020C05D0000407E0500F4
:10FDD00000200B4908700B49087001200A4908707F
:10FDE0000A49087000200A4908700A4908700A493F
:10FDF00008800A4908800A4908800A490870704743
:10FE00000600002007000020080000200900002054
:10FE10000A0000200B0000200C0000200E00002033
:10FE2000100000201200002000200B4908700B4930
:10FE3000087001200A4908700A49087000200A4920
:10FE400008700A4908700A4908800A4908800A4966
:10FE500008800A490870704706000020070000204B
:10FE600008000020090000200A0000200B000020EC
:10FE70000C0000200E0000201000002012000020C6
:10FE8000F8B50646002700240025002000903148E0
:10FE90000078002809D00320F9F766FB002804D079
:10FEA0000320F9F755FB2C4908802C4800880A28C4
:10FEB0004AD300202949088029480078282829D2D7
:10FEC0000320F9F745FB0746002407E060002549B9
:10FED000085AB84200DD05E0601CC4B22048007832
:10FEE0008442F3DB00BF1E48057808E0681E40002E
:10FEF0001C49085A69001B4A5052681EC5B2A542E7
:10FF0000F4DC600017490F5215480078401C144972
:10FF1000087019E0002000900F2407E060001149EC
:10FF2000095A009808180090601CC4B2192CF5D327
:10FF30000A210098F8F70AF90749088000200849C3
:10FF40000870012008490870044800888019034996
:10FF50000880F8BD090000200200002016000020E3
:10FF600000000020E807002012000020394909881D
:10FF70001E2928DA0021384A1180384A1180384970
:10FF80000988384A914207DC37490978002914D09A
:10FF900033490988914210DC0121344A1170002153
:10FFA000334A1170334A11702F4A11700121324ABD
:10FFB00011700021314A11704BE029490988091854
:10FFC000274A118045E023490988264A6432914234
:10FFD0002ADB0021224A1180204A11801E4909880B
:10FFE000204A914207DC20490978002916D01A4995
:10FFF0000988914212DC02211C4A117000211C4A1E
:020000040001F9
:10000000117005211B4A11700021174A117001213E
:10001000194A11700021194A11701AE00E49098815
:1000200009180D4A118014E000210D4A11800A4A76
:1000300011800A4909880B4A914205DD00210B4ACB
:100040001170094A117004E0044909880918034A2B
:100050001180704702000020100000200C000020DA
:100060000E000020B80B0000090000200B0000204B
:100070000600002007000020080000200A000020E1
:100080000148007870470000BC0900200148007A50
:1000900070470000BC0900200148807870470000CC
:1000A000BC09002001480088704700008000002043
:1000B000F8B50023002500950024002200BF94E03D
:1000C00001259D40ACB20D8825400095009DA542BC
:1000D0006FD11A468D79012D0DD1464D032636027A
:1000E000AD192D5C012696403543424E03273F0251
:1000F000F61935540CE03F4D03263602AD192D5C40
:1001000001269640B5433B4E03273F02F61935546E
:10011000CD78002D4ED1374D60352D5CCE78002E38
:1001200001D1012600E000269640B543314E6036ED
:1001300035548D78002D2ED12E4D19267601AD190E
:100140002D5C8E78002E01D1012600E0002696401D
:10015000B543284E19277F01F61935540D79002D26
:100160000ED1244D50352D5C0E79002E01D1012683
:1001700000E000269640B5431E4E5036355423E02D
:100180001C4D50352D5C0E7996403543EEB2194D1D
:1001900050352E5418E0174D19267601AD192D5CF7
:1001A0008E7896403543134E19277F01F619355442
:1001B0000AE018E00F4D60352D5CCE78964035434F
:1001C000EEB20C4D60352E544D79012D0AD1094DFA
:1001D00030352D5C012696403543EEB2054D303565
:1001E0002E5400E000BF5D1CABB2082B00DA67E7BD
:1001F000F8BD000000000440FFB5074615461E4646
:1002000000243846019900F01FF8002802D0012090
:1002100004B0F0BD00240CE00A2060430949085CEA
:10022000B04204D12946204600F05EF807E0601C89
:1002300084B20A2060430349085C0028ECD100BF67
:100240000020E5E7B00100200246002A03D1402942
:1002500001DD01207047032A03D1022901DD0120BD
:10026000F8E7042A03D1202901DD0120F2E7052A5D
:1002700003D1202901DD0120ECE70C2A03D110294C
:1002800001DD0120E6E70D2A05D1012903DD402922
:1002900001DA0120DEE70E2A03D1202901D1012055
:1002A000D8E70020D6E7000010B5064A03231B025A
:1002B000D218125C8A43034B032424021B191A54DC
:1002C00010BD00000000044010B5064A03231B02C5
:1002D000D218125C0A43034B032424021B191A543C
:1002E00010BD00000000044070B502460020B1E0DF
:1002F0000A2353435A4C1B195B1C440004191B1955
:100300009B788B427DD10A235343554C1B195B1CB0
:10031000440004191B195B78082B33D10A2353437B
:100320004F4C1B195B1C440004191B574D4C4E4D80
:100330006419E35C012423430A245443484D64199F
:10034000641C450045196457464D474EAD192B5561
:100350000A235343424C1B195B1C440004191B57CE
:10036000404C35466419E35C022423430A24544379
:100370003B4D6419641C450045196457394DAD194E
:100380002B5564E00A235343354C1B195B1C440076
:1003900004191B195B78092B34D10A235343304CC1
:1003A0001B195B1C440004191B572E4C2E4D64195D
:1003B000E35C402423430A245443294D6419641CFC
:1003C000450045196457274D274EAD192B550A2373
:1003D0005343234C1B195B1C440004191B57214C2D
:1003E00035466419E35C8024A3430A2454431C4D1E
:1003F0006419641C4500451964571A4DAD192B55F5
:1004000025E025E00A235343154C1B195B1C4400CF
:1004100004191B57134C144D6419E35C0A2454430C
:100420000F4D6419641C4500451964196578012451
:10043000AC402343DCB20A235343094D5B195B1CD8
:10044000450045195B57074D074EAD19EC5404E0C4
:10045000431CD8B2032800DA4AE700BF70BD000091
:10046000B00100200000044075080000F8B5002429
:10047000FCF7FEFA012861D100F0A2FB0446FF223E
:100480000721002003F0B8F8012C21D100F096FCE0
:1004900000280ED000F0A6FB054600F097FB0646AC
:1004A00001200346024629460090304605F010FC24
:1004B00050E000F097FB054600F088FB064601205F
:1004C0000023024629460090304605F001FC41E039
:1004D000022C21D100F072FC00280ED000F082FB2B
:1004E000054600F073FB06460120034602462946F6
:1004F0000090304605F0ECFB2CE000F073FB054665
:1005000000F064FB0646002001231A4629460090AD
:10051000304605F0DDFB1DE000F050FC054600F024
:1005200061FB064600F052FB0746012003462A46BF
:1005300031460090384605F0CBFB0BE00020034627
:1005400002460146009005F0C3FB00220721104639
:1005500003F052F8F8BD0000FEB500248148007891
:10056000012827D1FCF784FA012815D1FCF762F89D
:1005700000BF0EE0182C0AD0152C08D00D2C06D088
:100580001A2C04D0FF222146002003F035F8601C0D
:10059000C4B2242CEEDBE4E0FCF798F9002406E07A
:1005A00000222146104603F027F8601CC4B2242C18
:1005B000F6DBD6E0FCF75CFA01287BD1FCF73EFACB
:1005C0006949884278D300F007FB064600F01EFB1D
:1005D00007460A21F7F7BAFD0546324629460120AB
:1005E0000BF032F900F05CFD064600F0DDFC0A215C
:1005F0000290F7F7ABFD054600F0EEFA07463246EB
:10060000294609F0AFF8FFF731FF00F0C7FA0546B9
:100610002946012007F0ECFB00F0F2FA0646FF2124
:10062000F531F7F7A9FDC5B22946012006F00CFB0C
:10063000FFF726FD0546FFF735FD0646FFF72CFDC3
:1006400007462B4632463946012005F01BFE00F0D6
:1006500005F90546294601200BF09CFB00F0CAFC79
:10066000054600F0C3FB064600F0CAFC074600F052
:10067000C3FB00233A4601460096019502900120F3
:100680000AF0FEFDFF220321002002F0B5FFFF2249
:100690000421002002F0B0FF00F07AFC054600F0D3
:1006A00071FC064600F07AFC07462A46314607F000
:1006B000D3FD56E00DE0FFE7FF220321002002F00A
:1006C0009BFFFF220421002002F096FFFCF72CF88C
:1006D00047E0FCF7FBF800220321104602F08CFFF4
:1006E00000220421104602F087FF00222321104639
:1006F00002F082FF00222221104602F07DFF00223C
:100700000721104602F078FF00220821104602F06F
:1007100073FF00220921104602F06EFF00220A2119
:10072000104602F069FF00221321104602F064FF18
:1007300000221121104602F05FFF00221221104614
:1007400002F05AFF00220E21104602F055FF00224F
:100750000F21104602F050FF00221021104602F037
:100760004BFFFEBDE9000020B80B00000149086006
:10077000704700008407002002480068401C0149BF
:100780000860704780070020F3B581B0064600205E
:100790000E49086000F01EF8044600F01BF80546FC
:1007A0002F1B3046029903F0E5FE00900AE000F0AE
:1007B00011F805462F1B06480068002802D004489F
:1007C0000068804700988742F1D3FEBD8007002073
:1007D000840700200148006870470000800700205F
:1007E0000B490978012901D101200FE00849097856
:1007F000022901D1022009E005490978032901D124
:10080000042003E00121024A11700120704700001A
:100810001507002010B5094B1B8899B20A12C8B2FF
:10082000D3433133064C2370C343233363701346E1
:100830005633A37003467133E37010BD48070020A0
:100840001B0700200148008870470000200000209E
:1008500001480088704700003800002001480078F7
:1008600070470000950000200148007870470000A4
:100870009600002010B5002205210648FAF756FC24
:100880000402012205210348FAF750FC201880B227
:1008900010BD00005408002010B5062205210348B1
:1008A000FAF744FCC006C00F10BD00005408002039
:1008B00010B5042205210648FAF738FC0402052287
:1008C00011460348FAF732FC201880B210BD000030
:1008D0005408002010B5062205210248FAF726FC2C
:1008E000C01110BD5408002010B502220521024895
:1008F000FAF71CFC10BD00005408002010B50622B9
:1009000005210348FAF712FC8006C00F10BD000055
:100910005408002010B5042202210348FAF706FC0F
:10092000C007C00F10BD00005408002010B50522FC
:1009300002210348FAF7FAFBC007C00F10BD000000
:100940005408002010B5002204210348FAF7EEFBFA
:100950004006400F10BD00005408002010B50422CE
:1009600001210248FAF7E2FB801110BD5408002073
:1009700010B5002201210248FAF7D8FB10BD000093
:100980005408002010B5052201210348FAF7CEFBD8
:100990008007800F10BD00005408002010B5012210
:1009A00011460248FAF7C2FB10BD000054080020AF
:1009B00010B5002206210C48FAF7B8FB0402012208
:1009C00006210948FAF7B2FB201804020222062188
:1009D0000548FAF7ABFB201804020322062102485F
:1009E000FAF7A4FB201810BD5408002010B504220B
:1009F00006210C48FAF79AFB040205220621094851
:100A0000FAF794FB20180402062211460548FAF76B
:100A10008DFB20180402072206210248FAF786FB04
:100A2000201810BD5408002010B5022203210248EE
:100A3000FAF77CFB10BD00005408002010B503221B
:100A400000210248FAF772FB10BD00005408002094
:100A500010B5002211460248FAF768FB10BD0000ED
:100A60005408002010B5042200210248FAF75EFB6A
:100A700010BD00005408002010B5012200210248DA
:100A8000FAF754FB10BD00005408002010B50522F1
:100A900000210248FAF74AFB10BD0000540800206C
:100AA000322815DA3C498978012903DD01213A4AC7
:100AB000517070E038498978002905DD2F286ADCFB
:100AC0000021354A517066E00021334A517062E0DE
:100AD0003E2817DA322815DB2F498978022903DDF1
:100AE00002212D4A517056E02B498978012905DDF4
:100AF0003B2850DC0121284A51704CE00121264A54
:100B0000517048E0502817DA3E2815DB22498978D1
:100B1000032903DD0321204A51703CE01E498978F6
:100B2000022905DD4D2836DC02211B4A517032E0D6
:100B30000221194A51702EE0622817DA502815DB7D
:100B400015498978042903DD0421134A517022E0F4
:100B500011498978032905DD5F281CDC03210E4A31
:100B6000517018E003210C4A517014E073280FDA19
:100B700062280DDB08498978042905DD70280ADC24
:100B80000421054A517006E00421034A517002E035
:100B90000521014A51707047BC09002001480078C6
:100BA00070470000070000200148006870470000FF
:100BB000901F00200148007870470000DD000020F1
:100BC0000148007870470000DC00002001480078F0
:100BD00070470000E10000200148007970470000E4
:100BE000402800200148407870470000E1000020C4
:100BF0000148007A7047000040280020002070471C
:100C000001480088704700002200002010B5002431
:100C1000FFF7E2FF00280AD10A4800880A49884203
:100C200002DB0846074908800648048808E00548B2
:100C30000088FCF7F1FB84B20448844200DB0446E0
:100C4000204610BD3A000020C6070000CE04000078
:100C5000002005490988054A914202DB1146024AF3
:100C600011800149088870473A000020C60700003B
:100C7000F8B50027002500260024FFF7E9FE054609
:100C8000FFF7FAFE0646F020284000110A2805DB8F
:100C9000F02028400011C01C044303E0F02028404D
:100CA0000011044324022807000F0A2804DB280748
:100CB000000FC01C044302E02807000F0443240275
:100CC000F020304000110A2805DBF02030400011F0
:100CD000C01C044303E0F020304000110443240210
:100CE0003007000F0A2804DB3007000FC01C044344
:100CF00002E03007000F0443002C01D10248F8BD88
:100D000027463846FBE70000FFFF0000F8B5002744
:100D1000002500260024FFF7A5FE0546FFF7B6FED6
:100D20000646F020284000110A2805DBF020284064
:100D30000011C01C044303E0F020284000110443CC
:100D400024022807000F0A2804DB2807000FC01C14
:100D5000044302E02807000F04432402F02030403F
:100D600000110A2805DBF02030400011C01C0443AC
:100D700003E0F02030400011044324023007000F4C
:100D80000A2804DB3007000FC01C044302E03007D0
:100D9000000F0443002C01D10248F8BD2746384615
:100DA000FBE70000FFFF000010B50024FFF746FE40
:100DB0000446204610BD012070470000014800781D
:100DC000704700005107002001480078704700007C
:100DD000530700200148C07B70470000C80900206D
:100DE0000148C07C70470000C80900200148007A13
:100DF00070470000C809002010B50024054800888D
:100E0000323084B264212046F7F7B6F984B2204626
:100E100010BD0000C809002070B50024074908680B
:100E2000FBF746FF05466421F7F790F984B20448C2
:100E3000844200DD0446204670BD0000C809002041
:100E4000DE03000010B5002400F014F8012800D1E2
:100E50000CE000F00FF8022802D1FF24373405E03F
:100E60000A2103480088F7F787F984B2204610BDAD
:100E70000200002001480078704700000B000020AD
:100E8000002005490968002903D00349096808685A
:100E900000E0024870470000640100203075000047
:100EA00010B50024044804F0E3FB002801D001241D
:100EB00000E00024204610BD0407000010B5002407
:100EC000044804F0D5FB002801D0012400E00024F0
:100ED000204610BD0507000010B50024044804F0AA
:100EE000C7FB002801D0012400E00024204610BDEB
:100EF0000707000010B50024062004F0B9FB002805
:100F000001D0012400E00024204610BD10B50024CB
:100F1000052004F0ADFB002801D0012400E00024EE
:100F2000204610BD10B50024044804F0A1FB0028A1
:100F300001D0012400E00024204610BD0607000077
:100F400010B50024044804F093FB002801D00124CC
:100F500000E00024204610BD0305000010B5002469
:100F6000044804F085FB002801D0012400E000249F
:100F7000204610BD040500000148807A704700003B
:100F8000C80900200148807870470000600A0020EE
:100F90000148406870470000600A0020014840781E
:100FA00070470000600A002070B50024FFF714FEAF
:100FB000002803D1FCF744FC04460DE0FFF70CFECB
:100FC000012806D1FCF73CFC0546FCF725FA04464F
:100FD00002E0FCF735FC0446204670BD0148007C69
:100FE00070470000C80900200148007D70470000DC
:100FF000C80900200148407A70470000C809002055
:1010000010B5002405488088323084B2642120461F
:10101000F7F7B2F884B2204610BD0000C8090020DE
:1010200070B5002407494868FBF742FE0546642175
:10103000F7F78CF884B20448844200DD0446204669
:1010400070BD0000C8090020DE03000070B50BF081
:10105000AFF905460BF0ACF904490860002D01D149
:10106000012400E00024204670BD00007001002033
:101070000148007B70470000C80900200148407B00
:1010800070470000C80900200148807B70470000BD
:10109000C80900200148007870470000E0000020E7
:1010A00070B50024FFF798FD002803D1FCF7EAFB98
:1010B00004460FE0FFF790FD012807D10020FCF760
:1010C000E1FB0546FCF7A8F9044603E00020FCF725
:1010D000D9FB0446204670BD0148007870470000E7
:1010E0004200002070B505460024032D00D170BDDC
:1010F000002D01D0012D1BD181210320800204F09D
:1011000067FA8021134804F063FA32211248FFF78E
:101110003BFB002409E0A200104BD2189178A200FA
:10112000985A04F055FA601CC4B23B2CF3DB0FE074
:10113000022D0DD1002409E0A200094BD2189178AC
:10114000A200985A04F044FA601CC4B23B2CF3DBB2
:1011500000BFCCE702060000A0860100E4130200F5
:10116000D0140200F8B5002100240023002200BFA3
:101170000AE001258D40ABB205881D402C469C42FB
:1011800000D10A464D1CA9B21029F2DB0588FF2DBB
:101190001FDC284D6D7E0688B543264E7576354694
:1011A0002D7E0688B543234E357635466D7E86788E
:1011B000F607F60F964035431E4E757635462D7E62
:1011C000867802273E40760896403543194E35769C
:1011D00022E0184DED7E0688B543164EF57635466D
:1011E000AD7E0688B543134EB5768578ED07ED0FD5
:1011F0001646083EB5400F4EF67E35430D4EF57649
:101200008578022635406D081646083EB540094EE1
:10121000B67E3543074EB5760025009505E000BF44
:101220006D462D786D1CEEB200966D462D78012D21
:10123000F5D9F8BD206B0440C107C90F002905D0BE
:101240000021394A1171002238490A7102210140F6
:10125000002905D00021344A1172002233490A7254
:1012600004210140002905D000212F4A11730022DA
:101270002E490A7308210140002905D000212A4A7D
:101280001174002229490A7410210140002905D057
:101290000021254A1175002224490A7520210140A8
:1012A000002905D00021204A117600221F490A7624
:1012B00040210140002904D000221B494A711B49EA
:1012C0004A7180210140002904D0002216494A7247
:1012D00016494A72FF2101310140002904D0002241
:1012E00011494A7311494A730121490201400029F9
:1012F00004D000220C494A740C494A740121890225
:101300000140002904D0002207494A7507494A755F
:101310000121C9020140002904D0002202494A7675
:1013200002494A76704700000060004000610040BA
:10133000C107C90F002905D001223C490A710021CB
:101340003B4A117102210140002905D00122374991
:101350000A720021364A117204210140002905D089
:10136000012232490A730021314A117308210140D8
:10137000002905D001222D490A7400212C4A11743C
:1013800010210140002905D0012228490A750021B9
:10139000274A117520210140002905D00122234947
:1013A0000A760021224A117640210140002905D009
:1013B00001221E494A7100221D494A7180210140C3
:1013C000002905D0012219494A72002218494A729F
:1013D000FF2101310140002905D0012213494A7340
:1013E000002213494A73012149020140002905D016
:1013F00001220E494A7400220D494A7401218902D2
:101400000140002905D0012208494A7500220849F7
:101410004A750121C9020140002905D00122034972
:101420004A76002202494A76704700000061004077
:101430000060004010B50C480078002803D00B4A2B
:1014400050689168884708484078002803D0084AC7
:1014500050689168884704488078002803D0054A7E
:1014600050689168884710BD00600040000300206C
:10147000800400200006002010B5084800790028EC
:1014800003D0074A10695169884704484079002809
:1014900003D0044A50689168884710BD006000403E
:1014A000000300208C04002010B50848007A0028B2
:1014B00003D0074AD069116A88470448407A002857
:1014C00003D0044A50689168884710BD006000400E
:1014D000000300209804002010B50848007B002875
:1014E00003D0074A906AD16A88470448407B0028A5
:1014F00003D0044A50689168884710BD00600040DE
:1015000000030020A404002010B50848007C002837
:1015100003D0074A506B916B88470448407C0028F1
:1015200003D0044A50689168884710BD00600040AD
:1015300000030020B004002010B50848007D0028FA
:1015400003D0074A106C516C88470448407D00283E
:1015500003D0044A50689168884710BD006000407D
:1015600000030020BC04002010B50848007E0028BD
:1015700003D0074AD06C116D88470448407E00288C
:1015800003D0044A50689168884710BD006000404D
:1015900000030020C804002010B50848407F002840
:1015A00003D0074A5068916888470448007F0028A4
:1015B00003D0044A906DD16D884710BD0060004093
:1015C000D40400200003002010B50848407800280B
:1015D00003D0074A5068916888470448007800287B
:1015E00003D0044A506E916E884710BD20600040C1
:1015F000E00400200003002010B50948007900280D
:1016000003D0084A106F516F88470548001D407885
:10161000002803D0044A50689168884710BD000034
:101620002060004000030020EC04002010B5034AB5
:10163000D06F78329168884710BD00000003002009
:1016400010B5024A50689168884710BD8403002095
:1016500010B50948007C002803D0084A50689168FA
:101660008847054810304078002803D0044A506865
:101670009168884710BD0000206000409003002062
:101680001005002010B5024A50689168884710BDC7
:101690009C03002010B5024A50689168884710BD2D
:1016A000A803002010B50948007F002803D0084A8D
:1016B00050689168884705481C304078002803D05E
:1016C000044A50689168884710BD000020600040BF
:1016D000B40300203405002010B50C480078002821
:1016E00003D00B4A50689168884708484078002822
:1016F00003D0084A506891688847044880780028D9
:1017000003D0054A50689168884710BD406000408A
:10171000C003002040050020C006002010B50D4881
:101720000079002803D00C4A50689168884709481E
:10173000001D4078002803D0084A50689168884707
:101740000448001D8078002803D0054A506891683D
:10175000884710BD40600040CC0300204C050020AD
:10176000CC06002010B50D48007A002803D00C4AA2
:10177000506891688847094808304078002803D0AD
:10178000084A5068916888470448083080780028E3
:1017900003D0054A50689168884710BD40600040FA
:1017A000D803002058050020D806002010B50D48A9
:1017B000007B002803D00C4A50689168884709488C
:1017C0000C304078002803D0084A50689168884758
:1017D00004480C308078002803D0054A506891688E
:1017E000884710BD40600040E403002064050020ED
:1017F000E406002010B50D48007C002803D00C4AF8
:10180000506891688847094810304078002803D014
:10181000084A50689168884704481030807800284A
:1018200003D0054A50689168884710BD4060004069
:10183000F003002070050020F006002010B5024AD9
:1018400050689168884710BDFC03002010B5094816
:10185000007E002803D0084A5068916888470548F0
:1018600018304078002803D0044A506891688847AF
:1018700010BD0000406000400804002088050020E2
:1018800010B50948007F002803D0084A50689168C5
:10189000884705481C304078002803D0044A506827
:1018A0009168884710BD000040600040140400208B
:1018B0009405002010B508480078002803D0074A96
:1018C00050689168884704484078002803D0044A4B
:1018D00050689168884710BD606000402004002077
:1018E000A005002010B509480079002803D0084A57
:1018F0005068916888470548001D4078002803D04B
:10190000044A50689168884710BD0000606000403C
:101910002C040020AC05002010B50948007A0028EE
:1019200003D0084A506891688847054808304078D5
:10193000002803D0044A50689168884710BD000011
:101940006060004038040020B805002010B5024A4D
:1019500050689168884710BD4404002010B5024AC1
:1019600050689168884710BD5004002010B50948A0
:10197000007D002803D0084A5068916888470548D0
:1019800014304078002803D0044A50689168884792
:1019900010BD0000606000405C040020DC050020F9
:1019A00010B50948007E002803D0084A50689168A5
:1019B0008847054818304078002803D0044A50680A
:1019C0009168884710BD00006060004068040020F6
:1019D000E805002010B50948007F002803D0084A18
:1019E00050689168884705481C304078002803D02B
:1019F000044A50689168884710BD0000606000404C
:101A000074040020F405002010B5FE4800688079B9
:101A1000002806D001286ED002286DD003286CD192
:101A200004E2F8480068407903000EF00DFF0A0652
:101A300014BC2BBC47BC67BC9BBC0AF05FFF0020FA
:101A4000F0490968C873EF4800684079401CED49C7
:101A500009684871AEE0EC490969EA4A1268D27A2D
:101A6000885C0AF0C3FFE74800684079401CE549FC
:101A700009684871E34800684079401CE1490968F9
:101A8000487197E001F020FF002810D10AF0AEFF66
:101A9000DC4800684079401CDA4909684871D94837
:101AA00000684079401CD7490968487105E00AF090
:101AB0004FFF0020D349096848717BE001F004FF23
:101AC000002811D101200AF091FFCE48006840792A
:101AD000401CCC4909684871CA4800684079401CDC
:101AE000C8490968487105E00AF032FF0020C5497D
:101AF000096848715EE05FE0FEE0A3E101F0E4FE0A
:101B0000002828D1BF490968C97A24225143BF4A15
:101B100012688918BB4A1268D27B885C0AF066FF9B
:101B2000B8480068C07B401CB6490968C873B5480E
:101B30000068C07B242814D3B24800684079401C58
:101B4000B04909684871AF4800684079401CAD4908
:101B50000968487105E00AF0FBFE0020A949096800
:101B6000487127E001F0B0FE002815D1A5480068B3
:101B7000C07A401CA3490968C872A2480068C07AAC
:101B8000A1490978884207DB00209E490968C8728C
:101B900001209C49096888710AF0DAFE0020994901
:101BA0000968487106E00AF0D3FE002095490968EB
:101BB000487100BF00BF4FE19248006840790300C0
:101BC0000EF042FE080513912A91479170910AF098
:101BD00095FE00208B490968C8738A4800684079DF
:101BE000401C88490968487184E087490969854A29
:101BF0001268D27A885C0AF0F9FE8248006840795F
:101C0000401C8049096848717E4800684079401C42
:101C10007C49096848716DE001F056FE002811D139
:101C200026200AF0E3FE774800684079401C754999
:101C300009684871734800684079401C7149096817
:101C4000487105E00AF084FE00206E490968487179
:101C500050E001F039FE00281DD101200AF0C6FE37
:101C600068480068C07B401C66490968C8736548BD
:101C70000068C07B242814D3624800684079401C67
:101C80006049096848715F4800684079401C5D49B7
:101C90000968487105E00AF05BFE002059490968AF
:101CA000487127E001F010FE002815D15548006862
:101CB000C07A401C53490968C87252480068C07A0B
:101CC00051490978884207DB00204E490968C872EB
:101CD00002204C49096888710AF03AFE00204949FF
:101CE0000968487106E00AF033FE0020454909689A
:101CF000487100BF00BFAFE0424800684079030070
:101D00000EF0A2FD0805138B2A8B478B638B0AF01C
:101D1000F5FD00203B490968C8733A4800684079DE
:101D2000401C3849096848717EE037490969354ADD
:101D30001268D27A885C0AF059FE3248006840790D
:101D4000401C3049096848712E4800684079401CA1
:101D50002C490968487167E001F0B6FD002811D1EF
:101D600025200AF043FE274800684079401C254999
:101D700009684871234800684079401C2149096876
:101D8000487105E00AF0E4FD00201E490968487129
:101D90004AE001F099FD002810D10AF027FE194809
:101DA00000684079401C1749096848711548006867
:101DB0004079401C13490968487105E00AF0C8FDE4
:101DC00000201049096848712EE001F07DFD0028CF
:101DD00015D10C480068C07A401C0A490968C872CD
:101DE00008480068C07A08490978884207DB002063
:101DF00004490968C87203200249096888710AF019
:101E0000A7FD05E0D40700203C2F0020D0070020CC
:101E1000002012490968487106E00AF099FD002087
:101E20000E490968487100BF00BF15E000200B494A
:101E300009688871094909684871062007490968D5
:101E4000C87009E00AF084FD00200449096848715F
:101E500002490968887100BF00BF10BDD407002087
:101E600010B56A480068407903000EF0EDFC0906E1
:101E700010C627C644C6608EC6000AF03FFD634800
:101E800000684079401C614909684871BCE06049BC
:101E900009695E4A1268D27A885C0AF0A7FD5B483D
:101EA00000684079401C59490968487157480068E2
:101EB0004079401C554909684871A5E001F004FDCE
:101EC000002811D14F200AF091FD50480068407958
:101ED000401C4E49096848714C4800684079401CD4
:101EE0004A490968487105E00AF032FD0020474977
:101EF0000968487188E001F0E7FC002810D10AF079
:101F000075FD424800684079401C404909684871A5
:101F10003E4800684079401C3C490968487105E02A
:101F20000AF016FD00203949096848716CE001F09B
:101F3000CBFC002822D135480068C07A401C3349C8
:101F40000968C87231480068C07A31490978884206
:101F50000FDB00202D490968C8722C4800684079C1
:101F6000401C2A49096848710020284909684862CC
:101F700008E0002025490968487103E00020234952
:101F8000096848710AF0E4FC3EE020480068407CA3
:101F9000002816D01E48C068002803D01C48C1681D
:101FA00019208847002019490968486217490968BB
:101FB0004871164909688871052014490968C87074
:101FC0001AE012480068406A282807D20F480068C3
:101FD000406A401C0D49096848620DE000200B4929
:101FE000096848620949096848710849096888719F
:101FF000052006490968C87006E00AF0A9FC00201F
:1020000002490968487100BF00BF10BDD407002015
:102010003C2F002010B50024F7480068807A012882
:102020007ED1F5480068C07900287AD0F24800686F
:102030008079002804D0012874D0022873D191E15E
:10204000ED480068007B24286ED2EB480068C07918
:1020500001287AD1002475E0E7480068C07A24217D
:102060004843E64909684018E3490968097B415C2F
:10207000E1480068C07A24225043E14A126880187F
:10208000DD4A1268127B805C814229D0DA48006800
:10209000C07A24214843DA4909684018D6490968BA
:1020A000097B415CD4480068C07A24225043D34A5B
:1020B00012688018D04A1268127B8154CE4800689A
:1020C000407B242805D3CC480068007BCA490968B6
:1020D0004873C9480068007BC7490968887308E0ED
:1020E000C5480068407B242803D20120C249096802
:1020F0008871C1480068007B401CBF4909680873AB
:10210000BD480068007B242808D3BB480068407B9A
:10211000242803D20120B84909688871B64805E02F
:10212000D3E1CDE169E0BAE138E00EE00068007B80
:10213000242804D2B04800688079012800D103E047
:10214000601CC4B2242C87D356E0002413E0AA48B4
:102150000068C07A24214843A94909684018015DF4
:10216000A5480068C07A24225043A44A1268801807
:102170000155601CC4B2242CE9D300209E49096893
:10218000487323209C490968887301209A4909688B
:10219000887124209849096808732DE00020964929
:1021A0000968087394480068C07A401C924909681D
:1021B000C87291480068C07A92490978884217DB52
:1021C0008D480068007C012804D102208A490968F2
:1021D000887106E000208849096888718649096885
:1021E000C871002084490968C87283490968087465
:1021F000002081490968487161E17F4800684079A1
:1022000003000EF021FB080513A62AA651A68EA6F0
:1022100001207949096808740AF070FB7648006863
:102220004079401C74490968487199E07549096909
:10223000714A1268D27A885C0AF0D8FB6E4800684E
:102240004079401C6C49096848716B4800684079C6
:10225000401C69490968487182E001F035FB00289B
:102260001BD165490968497B491CC8B20AF0BEFB0D
:1022700061480068407B60490968C8735E4800682F
:102280004079401C5C49096848715B4800684079A6
:10229000401C59490968487105E00AF059FB0020C3
:1022A0005549096848715BE001F00EFB00282BD10D
:1022B00051490968C97A24225143504A1268891841
:1022C0004D4A1268D27B885C0AF090FB4A4800684D
:1022D000C07B401C48490968C87347480068C07BF8
:1022E00045490968897B88421ADD4348006840797E
:1022F000401C4149096848713F4800684079401CCA
:102300003D49096848710BE00AF022FB3A48006831
:10231000407B39490968C87300203749096848710A
:102320001EE001F0D1FA00280CD133490968887108
:10233000242031490968C8732F49096848732E4918
:10234000096888730AF004FB00202B49096848716A
:1023500006E00AF0FDFA002027490968487100BF2D
:1023600000BFACE024480068407903000EF06CFA2E
:1023700008050F8E268E4C8E688E0AF0BFFA1E4816
:1023800000684079401C1C490968487185E01D4976
:102390000969194A1268D27A885C0AF027FB164844
:1023A00000684079401C1449096848711248006867
:1023B0004079401C1049096848716EE001F084FAC8
:1023C000002811D125200AF011FB0B480068407944
:1023D000401C094909684871074800684079401C59
:1023E00005490968487105E00AF0B2FA002002497F
:1023F0000968487151E00000D4070020D007002090
:10240000CC0700203C2F002001F05EFA002810D1FC
:102410000AF0ECFA644800684079401C6249096897
:102420004871614800684079401C5F4909684871FB
:1024300005E00AF08DFA00205B49096848712CE03C
:1024400001F042FA00281AD157480068C07A401CAF
:1024500055490968C87254480068C07A53490978D8
:1024600088420CDB002050490968C8724E4909684F
:1024700088714D49096848714B490968C8710AF06B
:1024800067FA002048490968487106E00AF060FAD6
:10249000002045490968487100BF00BF0FE00AF0FD
:1024A00057FA00204049096848713F490968887116
:1024B0003D49096808733C490968C87200BF71E06A
:1024C00000203949096888726CE037480068807AD2
:1024D000022867D134480068007A00285ED032486C
:1024E00000684079002804D001280CD0032846D188
:1024F0001BE00AF003FA2C4800684079401C2A4986
:102500000968487149E000200AF070FA264800681E
:102510004079401C24490968487123480068407983
:10252000401C21490968487137E00AF0B1F90028D8
:1025300012D11D4800684078401C1B49096848704A
:10254000194800684078032812D301F05DFA002092
:102550001549096848700BE00020134909680872A2
:10256000AA2011490968887000200F49096848703D
:102570000AF0EEF900200C49096848710DE00AF0F4
:10258000E7F9002008490968487107490968487057
:10259000AA2005490968887000BF03E000200249AD
:1025A0000968887210BD0000D40700203C2F00206D
:1025B000F8B504460D4600260C2060431D49085C12
:1025C000002801D00120F8BD0C20604319494018B3
:1025D00085600C20604340188068002801D10120EC
:1025E000F1E701210C206043124A115400222046D9
:1025F000E317DB0E1B185B115B01E31A9B000E4F08
:10260000DB19E717FF0E3F197F11DA550EF04EF96F
:1026100000222046E317DB0E1B185B115B01E31A57
:102620009F00064BFB18E717FF0E3F197F11DA5585
:102630003046C8E700030020006000400061004011
:1026400000BFFEE709480088401C0849088008468A
:1026500000880749884208DD06480078002804D031
:10266000084602490880012088707047D800002081
:10267000DC050000DC00002010B51548807801283A
:1026800024D11448007801280CD11348007801287F
:1026900008D1002011498870084602F0B7FD0020DB
:1026A0000D4908700B48007802280CD10C480078BE
:1026B000012808D1002009498870084602F0A6FDCB
:1026C00000200749087000200249087010BD000072
:1026D000D8000020DC000020DE000020E100002007
:1026E000DF0000207047000010B500F05DFE0128FB
:1026F00003D1002001490880887010BDD800002057
:10270000F0B505460E46174600243A46314628469F
:1027100000F058FE00BF42E000202101394A126853
:1027200050522101374A126889184880002120013F
:10273000344A1268801881802001324A1268801859
:10274000C18020012F4A12688018017220012D4A91
:1027500012688018417220012A4A1268801881721A
:102760002001284A12688018C17200202101254AE0
:1027700012688918087300212001224A1268801803
:102780004173002021011F4A1268891888730021B3
:1027900020011C4A12688018C173601CC4B21A4818
:1027A0004078A042B8DC64201849096808807D2080
:1027B000C00016490968488015481449096888808E
:1027C0007D20000111490968C88010490968088105
:1027D00010480E49096848810F480C4909688881EA
:1027E00040000A490968C8813220084909680882FE
:1027F000FF20F53005490968488204490968888244
:10280000F0BD0000940700208807002090070020FA
:102810004C040000102700003075000038B500247B
:1028200004E0002013490855601C84B2282CF8D31A
:1028300001216846417001706A460F490D48FFF753
:102840005FFF7D21C900322000F0ACF90B490C4834
:1028500000F0C6F90948643000F058F90748C8305C
:1028600000F064F9074800F077F9074800F08AF9AA
:1028700038BD0000502800209C19020028230000C9
:10288000B80B0000542400001027000010B52448A5
:102890000078002803D10120214908703EE020483B
:1028A0000078012810D11F480078012808D10020A5
:1028B0001D498870084602F0A9FC002019490870DB
:1028C00002201749087029E015480078022810D125
:1028D00016480078012808D100201349887008465E
:1028E00002F094FC00201149087003200C49087084
:1028F00014E00B480078032803D10520084908702C
:102900000CE007480078052803D005480078062821
:1029100004D10020024908700549087010BD00006C
:10292000DC000020DE000020E1000020DF000020AD
:10293000E0000020F8B50024002500263548007886
:1029400000281ED134480078002803D101203249E4
:10295000087016E030480078012803D102202E4983
:1029600008700EE02C480078022803D103202A4981
:10297000087006E028480078032802D10020264984
:1029800008702448007801280ED10124172500265C
:1029900022480123324629460090204601F048FE95
:1029A00001201F49087034E01A48007802280FD12E
:1029B00001243B2500261948401C012332462946A4
:1029C0000090204601F034FE01201649087020E0F6
:1029D0001048007803280DD1FEF7FEF8002803D137
:1029E00001201149087102E000200F4908710DF023
:1029F000FDFE0EE007480078052803D106200549B2
:102A0000087006E003480078062802D10520014935
:102A10000870F8BDDC000020DD000020E10000208F
:102A2000DE000020DF0000204028002010B5044612
:102A300023000DF009FF095B060E16171819595AE5
:102A40005E00F9F7FBFF2C49884201D3FFF772FFC4
:102A500050E0F9F7F3FF2849884201D3FFF716FF4A
:102A600048E047E046E045E0F9F7E8FF22498842C0
:102A700039D301F08DFD21480078032814D1204876
:102A80000078002810D1FEF7B3F8002806D1012005
:102A90001C4988608868FAF75BFF05E00020194947
:102AA00088608868FAF754FF14480078012805D137
:102AB00013480078002801D1FAF752F9104800783D
:102AC000052803D10120104908700AE00C4800785D
:102AD000062803D102200C49087002E000200A49B0
:102AE00008700BF023FC05E004E003E0FFF7AAFD0B
:102AF00000E000BF00BF10BDB80B0000DD000020EB
:102B0000DC00002040280020E000002001460020DA
:102B1000054A126852898A4201DC012002E0024A19
:102B200012681181704700009007002001460020C4
:102B3000084A126812898A4201DB012009E0054A2D
:102B4000126892898A4201DC012002E0014A12687F
:102B5000518170479007002001460020084A126802
:102B600052898A4201DB012009E0054A1268D289B4
:102B70008A4201DC012002E0014A1268918170471B
:102B80009007002001460020054A126892898A4277
:102B900001DB012002E0024A1268D1817047000087
:102BA00090070020024600200C4B1B681B8A9342B2
:102BB00001DD012010E08A4201DB01200CE0074B1F
:102BC0001B689B888B4201DC012005E0034B1B68DE
:102BD0001A80024B1B685980704700009007002044
:102BE000024600200C4B1B681B8A934201DD01202A
:102BF00010E08A4201DB01200CE0074B1B685B8878
:102C0000934201DB012005E0034B1B689A80024BD5
:102C10001B68D980704700009007002070B50446FB
:102C200000250C206043FE490968401840680028D0
:102C300007D00C216143FA4A126889184868804716
:102C400005460C206043F6490968085C002873D1EA
:102C50000C206043F249096840188068002874D04D
:102C60002001F04909684018C07A02280AD1032DD2
:102C700008D10C206043EA4A12688018816801205C
:102C8000884762E02001E74909684018C07A0228B5
:102C90000AD1042D08D10C206043E14A1268801843
:102CA00081680220884750E02001DE490968401809
:102CB000C07A02280AD1052D08D10C206043D84AD9
:102CC000126880188168032088473EE02001D549BA
:102CD00009684018C07A02280AD1062D08D10C20B4
:102CE0006043CF4A126880188168042088472CE02E
:102CF0002001CC4909684018C07A02280AD1072D62
:102D000008D10C206043C64A1268801881680520EB
:102D100088471AE02001C34909684018C07A022890
:102D20000BD1082D09D10C206043BD4A12688018D0
:102D300081680620884708E00DE00C206043B84A0F
:102D4000126880188168002088472001B549096809
:102D50004018C5720CE30C206043B1490968085C57
:102D6000012873D10C206043AD4909684018806880
:102D7000002874D02001AB4909684018C07A0328A4
:102D80000AD1022D08D10C206043A54A1268801890
:102D900081680120884762E02001A2490968401843
:102DA000C07A04280AD1022D08D10C2060439C4A25
:102DB0001268801881680220884750E020019949F4
:102DC00009684018C07A05280AD1022D08D10C20C4
:102DD0006043934A126880188168032088473EE068
:102DE0002001904909684018C07A06280AD1022DAE
:102DF00008D10C2060438A4A126880188168042038
:102E000088472CE02001874909684018C07A0728C4
:102E10000AD1022D08D10C206043814A1268801823
:102E20008168052088471AE020017E49096840181A
:102E3000C07A08280BD1022D09D10C206043784AB2
:102E40001268801881680620884708E00DE00C2091
:102E50006043734A12688018816800208847200107
:102E6000704909684018C57282E20C2060436C49C1
:102E70000968085C0228F7D1002D7DD1200169493D
:102E80000968085A68490968098A884275DA200180
:102E900064490968085A0A3081B22001614A1268FF
:102EA000115220015F490968085A5F490968098A77
:102EB000884231DB20015B490968401840885A4943
:102EC00009680988884227DB2001564909684018AB
:102ED000408855490968498888421DDC0020210145
:102EE000504A12688918488020014E4909684018E4
:102EF000807A0028B8D10C206043494909684018FD
:102F000080680028B0D00C206043454A12688018C1
:102F10008168012088472BE2200142490968085A4C
:102F200041490968098A88429EDB20013D490968B8
:102F3000401840883C4909688988884294DB200110
:102F4000384909684018408837490968C988884263
:102F50008ADC00202101334A126889184880200148
:102F6000304909684018807A0028D4D10C20604389
:102F70002B490968401801E063E00BE080680028F5
:102F8000C9D00C206043264A12688018816802204C
:102F90008847EDE100202101224A12688918488003
:102FA0002101204A12688918C872002120011D4A97
:102FB00012688018C18020011A4A12688018417274
:102FC0002001184A1268801881721848017820017F
:102FD000144A12688018017200202101114A1268F7
:102FE0008918888021010F4A126889180873210105
:102FF0000C4A12688918487321010A4A1268891814
:10300000887300212001074A12688018C1730C20C0
:10301000604303490968401880680028B9D007E078
:103020008C070020940700209007002088070020CC
:103030000C206043CF4A12688018816800208847BE
:1030400096E1012DA5D12001CB4909684018C07A2D
:10305000A84225D000212001C74A1268801841806B
:1030600000202101C44A12688918C8802001C24981
:1030700009684018C572C14800782101BE4A12682B
:103080008918487200202101BB4A1268891888807B
:10309000BA4801782001B84A12688018017267E1C5
:1030A0002001B54909684018007AB4490978884276
:1030B00020D0B24800782101AF4A126889180872FE
:1030C0002001AD4909684018407AAC490978884226
:1030D00009D02001A8490968401880882101A64A22
:1030E00012688918C88000212001A34A126880183C
:1030F000818012E02001A049096840188088A04919
:1031000088420AD220019C490968401880880A3008
:103110002101994A12688918888020019649096816
:1031200040184088964988420AD22001924909688D
:10313000401840880A3021018F4A12688918488057
:1031400020018D4909684018407A8C4909788842E5
:1031500005D001202101884A12688918887220014F
:103160008549096840184088864909680988884265
:1031700004DB00212001804A1268115220017E499F
:1031800009684018807A00287ED10C206043794974
:10319000096840188068002877D0200176490968BE
:1031A00040184088774909680989884214DB200162
:1031B000714909684018007B00280DD10C2060433C
:1031C0006C4A126880188168032088470120210119
:1031D000694A12688918087320016749096840180C
:1031E0004088684909684989884214DB200162499E
:1031F00009684018407B00280DD10C2060435D4ACF
:1032000012688018816804208847012021015A4AE9
:103210001268891848732001574909684018408886
:10322000584909688989884214DB20015249096894
:103230004018807B00280DD10C2060434D4A126855
:103240008018816805208847012021014A4A1268B8
:1032500089188873200148490968401840884949FD
:103260000968C989884210DB200143490968401870
:10327000C07B00287CD10C2060433E4A1268801835
:1032800081680620884701E007E03BE0012021013A
:10329000394A12688918C8736AE0200136490968FA
:1032A0004018407A01282ED13448007802282AD1CB
:1032B0002001314909684018C08832490968498AA3
:1032C000884255DB20012C490968401880882D4927
:1032D0000968898A88424BDB0C20604325490968CC
:1032E00040188068002843D00C206043214A1268AF
:1032F0008018816807208847002021011E4A126833
:103300008918487234E020011B4909684018407A46
:1033100002282DD119480078012829D12001164909
:1033200009684018C08817490968898A88421FDBE4
:103330002001114909684018808812490968498AA2
:10334000884215DB0C2060430A49096840188068F0
:1033500000280DD00C206043064A1268801881684E
:103360000820884700202101034A12688918487202
:1033700070BD00008C070020940700208807002003
:10338000F0FF00009007002010B5002400BF04E00B
:103390002046FFF743FC601CC4B202484078A042BC
:1033A000F6DC10BD8807002010B50024044802F0A8
:1033B0005FF9002800D000E00124204610BD000085
:1033C0000304000010B5074B14781C7054785C702F
:1033D000054B1960054B186003461833044C2360F5
:1033E00010BD0000880700208C07002090070020F7
:1033F0009407002010B50446012C09D1FF220C21AE
:10340000002000F0F9F80121022004F05FFE08E03E
:1034100000220C21104600F0EFF80021022004F0F9
:1034200055FE10BD10B5002404210848F7F790FEA2
:10343000552801D1012407E0042001F01BF80028E1
:1034400001D0002400E00124204610BD54080020D3
:1034500010B50446012C09D1FF221C21002000F0E8
:10346000CBF80121062004F031FE08E000221C21E7
:10347000104600F0C1F80021062004F027FE10BD20
:1034800010B50024062000F0F5FF002801D001242B
:1034900000E00024204610BD10B50446012C09D1DF
:1034A000FF221721002000F0A7F80121042004F0DA
:1034B0000DFE08E000221721104600F09DF80021C3
:1034C000042004F003FE10BD00200449097A0029FD
:1034D00001D0012000E0002070470000600A0020B9
:1034E00010B50446022C1CD100220D21104600F01C
:1034F00083F8FDF763FC002809D0FF220B21002090
:1035000000F07AF801210D2004F0E0FD58E00022DF
:103510000B21104600F070F800210D2004F0D6FDBC
:103520004EE0032C1CD100220B21104600F064F861
:10353000FDF744FC002809D0FF220D21002000F0F7
:103540005BF801210D2004F0C1FD39E000220D21BE
:10355000104600F051F800210D2004F0B7FD2FE0D7
:10356000042C0ED1FF220D21002000F045F800228E
:103570000B21104600F040F801210D2004F0A6FDBB
:103580001EE0012C0ED100220D21104600F034F86F
:10359000FF220B21002000F02FF801210D2004F064
:1035A00095FD0DE000220D21104600F025F80022C7
:1035B0000B21104600F020F800210D2004F086FDBC
:1035C00010BD000010B500240A480078012801D180
:1035D00001240CE0FCF75AFD012801D1032406E088
:1035E000FCF754FD022801D1022400E00424204607
:1035F00010BD0000E900002010B5064B1B78834287
:1036000007DD242905D224234343034C24681B19D6
:103610005A5410BD3C2F0020CC07002010B5744830
:103620000068407903000DF00FF90B0711D325D383
:103630005A6D77D38DA8D30009F060F96C48006803
:103640004079401C6A4909684871CFE06949496975
:10365000087809F0CBF9664800684079401C644955
:1036600009684871624800684079401C60490968EF
:103670004871BBE000F028F9002811D17F2009F043
:10368000B5F95B4800684079401C594909684871A0
:10369000574800684079401C5549096848711DE049
:1036A000534800684078401C5149096848705048A8
:1036B0000068407803280BD300204D490968487002
:1036C000AA204B4909688870032049490968C870D5
:1036D00009F03EF9002046490968487186E000F08B
:1036E000F3F8002807D1424800684079401C40495F
:1036F0000968487103E000203D490968487109F0F4
:1037000027F973E009F0FAF8394800684079401C5D
:1037100037490968487169E0364949690978491C9F
:10372000C8B209F063F9324800684079401C30495A
:10373000096848712E4800684079401C2C49096886
:10374000487153E000F0C0F800280FD109F0A8F844
:10375000274909688870012009F01CF9244800688D
:103760004079401C22490968487105E009F0F0F8E9
:1037700000201F490968487138E01D4800688078BA
:1037800018280CD102201A4909680870002018492D
:1037900009684870042016490968C87011E0144887
:1037A00000684078401C1249096848701048006859
:1037B0004078032805D300F027F900200C49096858
:1037C000487009F0C5F800200949096848710DE002
:1037D00009F0BEF8002006490968487104490968E3
:1037E0004870AA2002490968887000BF00BF10BD58
:1037F000D40700203C2F002010B5314800684079E4
:10380000002804D001280CD0032848D11DE009F07D
:1038100075F82B4800684079401C294909684871AF
:103820004BE028490969087809F0E0F82448006865
:103830004079401C22490968487121480068407954
:10384000401C1F490968487137E000F03DF8002826
:103850000CD101201A49096808700020184909682C
:103860004870042016490968C87011E014480068BF
:103870004078401C12490968487011480068407837
:10388000032805D300F0C0F800200D4909684870EE
:1038900009F05EF800200A49096848710DE009F056
:1038A00057F80020064909684871054909684870B9
:1038B000AA2003490968887000BF00BF10BD00003E
:1038C000D40700203C2F002010B508F0E1FF04468B
:1038D0001F4800680078002838D01D480068C0786C
:1038E000042833D3002C09D1002119480068C07A7C
:1038F0008200174800681430815027E0144800689F
:10390000C07A81001248006814304058114988423A
:1039100011D20F480068C07A81000D480068143049
:103920004058401C0A490968C97A8A000849096850
:10393000143188500AE000F067F80021044800685C
:10394000C07A82000248006814308150204610BDC1
:10395000D4070020B80B000000B587B001206946ED
:1039600008710848029008480390084804900848E5
:1039700005900848069001A9074800F00FF807B025
:1039800000BD0000C13C01005D580100D5090200E6
:10399000091A0200081A0200B8280020F8B50646E5
:1039A0000F46002400253946304600F0EFF900BFED
:1039B00014E000250EE00021242060430B4A126829
:1039C0008018415524206043094A126880184155E7
:1039D000681CC5B2242DEED3601CC4B20548007823
:1039E000A042E6DC00F010F8F8BD0000CC07002093
:1039F000D00700203C2F00200120024909680871EF
:103A000070470000D407002010B500F073F90020C3
:103A100003490968087002490968C87010BD0000B0
:103A2000D407002007480068C078062808D1054858
:103A30000068C079002803D1012002490968C871D3
:103A400070470000D407002010B555480068C078C2
:103A500003000CF0F9FE08671D1A1714110E056615
:103A600050484068002803D04E48416800208847ED
:103A700093E000F0E5F890E000F0C6F88DE000F08B
:103A8000D1F88AE0FFF7B8FE87E0FFF7C7FD84E0D2
:103A900044484068002803D04248416801208847D4
:103AA0003F480068407C00281AD03E48C068002883
:103AB00003D03C48C168C8208847002038490968BD
:103AC0004862374800680078002804D00420344950
:103AD0000968C87024E0022031490968C8701FE0F5
:103AE0002F480068406A401C2D49096848622C48EC
:103AF0000068406A7D21C900884211D3002028490E
:103B000009684862264800680078002804D004202C
:103B100023490968C87003E0022021490968C87078
:103B20003BE000BF1F484068002803D01D484168A3
:103B3000002088471A480068407C002813D01948A4
:103B4000C068002803D01748C168C82088470020F3
:103B500013490968486212480068C078401C10493F
:103B60000968C87018E00E480068406A401C0C499B
:103B7000096848620A480068406A7D21C900884295
:103B80000AD3002006490968486205480068C078E1
:103B9000401C03490968C87000BF00BF10BD000089
:103BA000D40700203C2F002010B515480068C078CD
:103BB000072824D0012012490968487408E01148F8
:103BC0008068002802D00F4988688047FFF73CFFD3
:103BD0000B480068C0780628F1D109480068007ACF
:103BE0000028ECD106480068C0790028E7D10448D5
:103BF0000068807A0028E2D101490968487410BD44
:103C0000D40700203C2F002010B50548006800783C
:103C1000012802D1FDF7F8FE01E0F5F76FFD10BDB8
:103C2000D407002010B5054800680078012802D1AB
:103C3000FEF716F901E0F6F73FF910BDD4070020B2
:103C400010B51D480068807A002829D11A480068FC
:103C5000007A002803D002201749096888721648A4
:103C60000068C079002803D00120134909688872D0
:103C7000114800680079012812D100200E49096816
:103C800008710D490968887207200B490968C870D6
:103C90000A484068002803D0084841680020884747
:103CA000054800680078012802D1FEF7B3F901E069
:103CB000F6F7DCF910BD0000D40700203C2F0020EF
:103CC00010B504462146084801F0EEFC074800788C
:103CD000002805D1002C03D032210548FCF754FD03
:103CE0000248047010BD000001030000EA0000203B
:103CF00050C300000020244909684870AA202249C6
:103D00000968887000202049096848621E490968CE
:103D100008711D49096848711B49096888711A4969
:103D20000968C871184909680872174909688872D2
:103D300015490968C8721449096808732420124992
:103D4000096848731049096888730F490968C8737E
:103D500000200D49096808740B49096848740A492C
:103D60000968887408490968C8740749096848617E
:103D7000002105480068816103480068C16102486C
:103D80000068016270470000D407002010B50A786F
:103D90000D4B1860034628330C4C236024235343F7
:103DA000044628341B190A4C23600A4C4B68636094
:103DB0008B68A360CB68E3604B6963610B69236127
:103DC0000B78237010BD0000D4070020CC07002022
:103DD000D00700203C2F002007480068C078062844
:103DE00008D105480068007A002803D10120024963
:103DF0000968087270470000D407002010B5044617
:103E0000012C09D1FF2220210020FFF7F5FB012121
:103E1000084604F05BF908E0002220211046FFF775
:103E2000EBFB0021012004F051F910BD10B5002476
:103E3000032000F01FFB002801D0012400E0002433
:103E4000204610BD10B50446032C0ED1FF221521CB
:103E50000020FFF7D1FB002214211046FFF7CCFB16
:103E600001210E2004F032F939E0022C1CD1FCF7BC
:103E7000A5FF002809D0FF2214210020FFF7BCFB7A
:103E800001210E2004F022F908E00022142110463E
:103E9000FFF7B2FB00210E2004F018F900221521D3
:103EA0001046FFF7A9FB1AE0012C0ED1FF221421C6
:103EB0000020FFF7A1FB01210E2004F007F90022EA
:103EC00015211046FFF798FB09E000221521104646
:103ED000FFF792FB002214211046FFF78DFB10BD67
:103EE00010B50024F8F7AAFD094988420DD3FCF764
:103EF000C1FF002807D1FCF751FE012801DD032492
:103F000004E0022402E0022400E00124204610BD67
:103F1000B80B000010B50446012C09D1FF221D2169
:103F20000020FFF769FB0121002004F0CFF808E032
:103F300000221D211046FFF75FFB0021084604F018
:103F4000C5F810BD10B50024022000F093FA002837
:103F500001D0012400E00024204610BD10B5044625
:103F6000012C09D1FF221E210020FFF745FB012172
:103F7000092004F0ABF808E000221E211046FFF7EC
:103F80003BFB0021092004F0A1F810BD70B500240E
:103F900000250026FCF7BEFC0546FCF7C7FC0646DC
:103FA00002210848F7F7D4F8552800D108E0012E7F
:103FB00001D1002404E0012D01D1012400E00024FE
:103FC000204670BD5408002010B50446012C09D1CC
:103FD000FF221F210020FFF70FFB0121082004F022
:103FE00075F808E000221F211046FFF705FB0021AD
:103FF000082004F06BF810BD70B500240025FCF714
:1040000013FD054603211A48F7F7A2F8552806D1F3
:1040100001201849088000201749088023E016482D
:104020000088012811D114490880FCF717FC762874
:1040300003DA01200F49088015E0FCF70FFC78280F
:1040400011DB00200B4908800DE001200A4908809F
:10405000FCF704FC762803DA01200649088002E018
:1040600000200449088003480488204670BD0000F1
:1040700054080020060100200801002010B5044665
:10408000012C09D1FF2221210020FFF7B5FA0121DF
:10409000072004F01BF808E0002221211046FFF75A
:1040A000ABFA0021072004F011F810BD10B5002470
:1040B000FCF7CCFF012801D1012400E000242046B8
:1040C00010BD10B50446012C09D1FF221621002095
:1040D000FFF792FA0121032003F0F8FF08E0002225
:1040E00016211046FFF788FA0021032003F0EEFFA7
:1040F00010BD10B50024052000F0BCF9002801D047
:10410000012400E00024204610BD10B50446012C17
:1041100009D1FF2219210020FFF76EFA01210520A5
:1041200003F0D4FF3CE0022C17D1FCF747FE002837
:1041300009D0FF2219210020FFF75EFA0121052096
:1041400003F0C4FF2CE0002219211046FFF754FAB7
:104150000021052003F0BAFF22E0032C17D1FCF761
:1041600033FE002809D0FF2219210020FFF744FA6E
:104170000121052003F0AAFF12E0002219211046B8
:10418000FFF73AFA0021052003F0A0FF08E0002223
:1041900019211046FFF730FA0021052003F096FFA1
:1041A00010BD000010B50024FCF722FD01282FD11E
:1041B00004211948F6F7CCFF552801D1012428E045
:1041C000FCF7C0FB01280BD0FCF7BCFB022807D092
:1041D000FCF7B8FB032803D0FCF7B4FB052801D19A
:1041E000012416E0FCF7AEFB042801D1022410E004
:1041F000FCF7A8FB062801D103240AE0FCF7A2FB88
:10420000002803D0FCF79EFB072802D1002400E021
:104210000024204610BD00005408002010B50446BC
:10422000012C0ED1FF221B210020FFF7E5F900220F
:104230001A211046FFF7E0F901210A2003F046FF9A
:104240001EE0022C0ED1FF221A210020FFF7D4F924
:1042500000221B211046FFF7CFF901210A2003F0AD
:1042600035FF0DE000221A211046FFF7C5F90022A4
:104270001B211046FFF7C0F900210A2003F026FF9A
:1042800010BD000010B5002410480078012801D1AD
:10429000012418E0FCF79EFD022803D0FCF79EFEE7
:1042A00002280FD1FCF768FE012809D1FCF798FD20
:1042B000012803D0FCF798FE012801D1012402E077
:1042C000022400E00224204610BD0000E900002086
:1042D00010B5F8F7CDFB0446204610BD10B5034BD2
:1042E00008220349034800F013F910BDD142010030
:1042F000A81902007828002070B506465C4880683E
:10430000002804D05A4988688047054600E0002507
:104310000024A6E0564841680C20604308184088F5
:10432000A84207D0524841680C20604308184088D2
:1043300002287DD14E4841680C20604308188068EF
:1043400000280CD04A494A680C21614351188868FA
:10435000804747490968E2008918487009E04448E5
:1043600041680C206043095C41480068E200801805
:1043700041703F480068E100401840783C490968B6
:10438000E200895C88420FD039480068E10040189B
:10439000417837480068E2008154002034490968B8
:1043A000E200891848605AE031480068E10040188E
:1043B00041782F4842680C206043101840788142B1
:1043C0001FD12B480068E100401841682848426826
:1043D0000C2060431018808881420BD82448006864
:1043E000E10040184068801921490968E2008918F5
:1043F000486034E001201E490968E20089184880BD
:104400002DE01B480068E1004018416818484268E8
:104410000C2060431018C08881420DD814480068F1
:10442000E10040184068811911480068E20000E08E
:1044300009E08018416012E000200D490968E2009F
:10444000891848800BE0002009490968E2008918B2
:104450004880002106480068E20080184160601C26
:1044600084B203488089A04200DD53E770BD00009C
:10447000F42E00200146064A92898A4205DD044A4C
:104480001268CB00D218508800E00020704700006E
:10449000F42E0020002000BF14E00D494A680C21D2
:1044A00041435118498801290AD10021084A12685C
:1044B000C300D2185180064A1268C300D218516056
:1044C000411C88B2024989898142E6DC70470000BC
:1044D000F42E0020002000BF13E00C494A680C2194
:1044E000414351184988002909D1084A1268C3007C
:1044F000D2185180054A1268C300D2185160411C7D
:1045000088B2024989898142E7DC7047F42E002095
:10451000F0B504460020164DAB6069602C60AA819E
:1045200000BF1FE0124D6E680C254543755D104EAF
:104530003668C700F61975700D4D6E680C25454339
:10454000755D0B4E3668C700F5550025084E366878
:10455000C700F6197580064E3668C700F6197560F3
:10456000451CA8B2024DAD898542DBDCF0BD0000E0
:10457000F42E002070B505460E46002E05D03146BB
:104580002846F3F7E3FD044600E02C46204670BDC4
:1045900010B5FCF75BFD012817D10C480078012805
:1045A00013D00A48007803280FD009480078002863
:1045B0000BD1FCF765FC0749884202D108F075F879
:1045C00003E07D20000108F077F810BDDD00002039
:1045D000DC0000208813000008B5002000900122B4
:1045E00069460520F9F7E8FD054900988860002034
:1045F00004490870044908700449087008BD0000A7
:1046000040280020DC000020DE000020DF00002029
:1046100008B500200090012269460520F9F7CCFD7D
:104620000020024908710098886008BD40280020D9
:1046300070B5049C2578914216DD01280AD18D427F
:1046400006DAFF26F61AAE420ED3EE18F5B20BE0EC
:10465000154609E0022807D1954204DD9D4203DB9F
:10466000EE1AF5B200E00D46257070BD0D4A4168A6
:10467000516081699161C168D160416A5162016A8A
:104680001162016811604169516181689160C1697D
:10469000D16101691161816A91620021024A117040
:1046A00070470000102F0020C807002010B5FFF74A
:1046B000F1FEF8F723F800210148F6F753FE10BD8C
:1046C0006008002010B5F8F719F8FFF703FF0AF0AB
:1046D000A1F80AF03DF9FBF77BFBFAF7A9F8FFF721
:1046E0007BFFF8F745FCF6F739FCF9F73DF9552162
:1046F0000548F6F737FEF8F773FAF9F7B3F8FBF762
:1047000027F8F6F725FE10BD600800201CB5002034
:104710003349087008F0A2F80020FCF7E3FC0CF025
:10472000BBFBF7F78FF9F8F75BFAF9F79BF8F6F7A9
:1047300007F8F6F785FAE12040020BF0EFFF00F0F2
:1047400079FAF6F70BFC08F069FAF7F7D7FFF9F7F3
:10475000B5FEF8F79DFCF8F717FCFFF7BFFDFEF775
:104760005DF8FFF7F9F8FFF71FFAF9F7ADFDFBF772
:104770005BFBFAF75DF81B4AFF21913101200AF03B
:10478000ADF90022114601200AF0ECF807F0D4FF41
:104790000AF026F80AF0DCF8FFF73AFFF9F71CF9FF
:1047A0000020114988714871087101208870487093
:1047B0001420087007226846F3F75FFD01990098FE
:1047C00000F0C2FF0221012000F09AFEFAF7C0FFBC
:1047D000F6F7BEFD55210548F6F7C4FD1CBD0000E7
:1047E000E90000200090D003FA00002060080020BB
:1047F0007047000010B50446552C03D1054948699F
:10480000804702E003490868804700200249087099
:1048100010BD0000102F0020C807002010B546482A
:10482000007803000CF010F80A06111B26303B46F6
:104830005051738141484068002802D03F49486880
:10484000804701203C49087000BF3C488068002830
:1048500004D03A49886880473749087069E037488A
:10486000C068002802D03549C86880470320324913
:10487000087000BF31480069002804D02F4908693A
:1048800080472D49087054E02C484069002802D028
:104890002A494869804700202749087049E027488D
:1048A0008069002802D0254988698047062022496E
:1048B000087000BF2148C069002804D01F49C8699A
:1048C00080471D49087034E000BF1B480078072866
:1048D0000AD11A48006A002802D01849086A80479D
:1048E00009201549087011E01348007808280AD1FA
:1048F0001248406A002802D01049486A80470920BF
:104900000D49087002E000200B49087000BF0A48FA
:104910000078002808D00948806A002804D0074998
:10492000886A80470449087003E000200249087043
:1049300000BF00BF10BD0000C8070020102F0020DE
:104940007047000010B500200CF062FB09F040F841
:1049500009F094F809F0AAF800F0C6FCF6F706FA98
:104960000220FCF7BFFB002007490870FFF71CF985
:10497000FFF742F8FFF768F8F6F752F810200AF050
:10498000C3FC00F0B1FD10BD9C01002010B5012456
:1049900008F0ECFB012801D1052407E0F8F748F8FE
:1049A0000349884201D2012400E00224204610BDC0
:1049B000204E000010B5062408F0D8FB002800D1D6
:1049C000002408F0D9FB012803D008F0D5FB072804
:1049D00000D90924204610BD10B5F6F7C7F900220A
:1049E000114601200AF0F0F800213C48F6F7BAFC25
:1049F00000203B490880002400BF00F02FFF322137
:104A00007D200001FBF7C0FE0020364908700AE057
:104A10000022344801781046FEF7EEFD3148007858
:104A2000401C304908702F4800782428F0DB002013
:104A30002D49087009E000212B48007809F0D8FCC6
:104A400029480078401C28490870274800780D281C
:104A5000F1DBFEF7F9FFF5F7B9FE08F0D9FA2348C4
:104A60000078401C2149087008460078052812D3B8
:104A700000200870FEF7D6FF1D4800780A2805D3ED
:104A800000201B490870FFF7A7F904E018480078D8
:104A9000401C1749087008F06FFB0128ADD908F0D9
:104AA0006BFB0728A9D200200F49087008E00E48C8
:104AB000007809F0B7FC0C480078401C0A490870DF
:104AC000094800780D28F2DBF6F7BAF855210348BB
:104AD000F6F748FCF7F782FF204610BD600800207B
:104AE0007C000020030100200101002002010020C1
:104AF0000401002010B5032408E000F0AFFE0120FF
:104B000000F0B6FD002801D0042400E0F5E700BF66
:104B1000204610BD10B500202A49086007F09EFE0F
:104B20000120FCF7DFFAF6F78DFF55212648F6F74E
:104B300019FCF8F755F8F8F795FE0CF0ADF9F5F714
:104B4000FFFDF9F783FCF6F77BF808F071FAF9F747
:104B5000B5FCF9F751FEF8F79BFAFFF7BFFBFDF73D
:104B60005DFEFFF7B7FCFFF737FDFEF7F5FEFFF739
:104B70001BF800F05FF8E12040020BF0CFFDF6F7E4
:104B8000EDF9FBF751F9F9F753FE104AFF21913186
:104B9000012009F0A3FF00221146012009F0E2FEE6
:104BA00009F01EFE09F0D4FEF8F7DEFE0221012016
:104BB00000F0A6FCFAF7CCFD07F0E0FDF6F7C8FB25
:104BC00010BD000050000020600800200090D003BD
:104BD00070B506460D4614460E4806600E48056040
:104BE0000E49206808600E49606808600D49A06899
:104BF00008600D49206908600C49E06808600C49AC
:104C00006069086005480068002802D00348006811
:104C1000804770BDB0000020B80000209800002040
:104C20009C000020A0000020A4000020A80000207C
:104C3000AC00002000B587B00C4801900C480290F1
:104C40000C4803900020049005900B48069000202B
:104C50000A49086048600A490860486001AA0121C1
:104C6000C9020848FFF7B4FF07B000BD894C010036
:104C70002D500100B54F0100E14E010074120020DB
:104C80006C0A00207C17002001207047F3B5C3B0E8
:104C90000446449E0020009057E002E0641C761E0B
:104CA00000BF022E05D32078EB28F7D1607890283A
:104CB000F4D1072E00D24AE0A778FD1CB54200D9F6
:104CC00045E0A81E205C0002691E615C084342901A
:104CD000042D38D9291FA01C0CF0F8F842998842FD
:104CE00026D11D480068002804D0B91EE01C1A4ACD
:104CF0001268904719480068002824D0E178684677
:104D00000171207981116846417120798106890EEF
:104D100068468171381FC1B26846C171C279611D90
:104D200002A8F3F7AAFA01A80C49096888470AE023
:104D30000020009002E00098401C00900098A842DB
:104D4000F9D3002000906419761B072EA5D200BF6E
:104D50004498801B45B0F0BDA4000020AC000020AA
:104D6000F7B5C0B0154600260027E81DFF21013128
:104D7000884202DD002043B0F0BDEB21684601709F
:104D800090214170281DC1B2684681700021C17018
:104D90004098C1B2684601710524002605E041989B
:104DA000805D69460855641C761CAE42F7DBA11E87
:104DB00000A802300CF08AF80746381269460855F8
:104DC000641C0F55641C06480068002805D0214665
:104DD0006846034A12689047CDE70020CBE7000001
:104DE0009C00002070B50024002500261B48406868
:104DF0001A490968884200D170BD184840681749AF
:104E00000968884205D91548406814490968451A57
:104E100007E01248006811494968401A01218902D7
:104E20000D1AFF2D01D9FF2600E02E4600240DE0CB
:104E30000A4801680830405C09490855074800885D
:104E4000401C8005800D05490860641CB442EFD306
:104E5000B1B203480BF0BEFC00BFCDE774120020D6
:104E60007C16002070B500251A480068002830D054
:104E7000194A1288FF230133991A184A1268164BEF
:104E80001B88D018134A126890470546002D20D081
:104E900011480088401910490880084601880F48C9
:104EA0000068FFF7F3FE0446002C0DDD0A48008879
:104EB000844209DA08480088021B08480068011982
:104EC00006480068F3F7D9F903480088001B024937
:104ED000088070BDA0000020B4000020B0000020B9
:104EE00038B5044600200090A07810280CD1207915
:104EF0002D49087008460078012853D10022114638
:104F00002020FFF72DFF4DE0A078122803D1207953
:104F10002549087246E0A078052803D12079224966
:104F200088723FE0A07802281DD120791E4948727E
:104F30000846407A012806D10090012269460420E3
:104F4000FFF70EFF2EE01848407A02282AD100BF52
:104F5000BFF34F8F15481649C860BFF34F8F00BF8E
:104F600000BF00BFFDE7A07801281BD120793328BE
:104F700003D101200C49487005E02079352802D181
:104F8000002009494870607907498870607A0006F6
:104F9000217A09040843E17909020843A179084309
:104FA0000149486038BD0000600A00200400FA058D
:104FB00000ED00E070B503460022002400251A48E9
:104FC0004068194E3668B04201D1002070BD1648C5
:104FD0004068154E3668B04205D913484068124EF5
:104FE0003668841B07E0104800680F4E7668801B07
:104FF0000126F602341AA14201D9254600E00D46E9
:1050000000220CE0084806680830805D9854064885
:105010000088401C4005400D034E3060521CAA42DF
:10502000F0D32846D2E700006C0A002070B5034692
:105030000022002415484068144D2D68A84208D36A
:1050400012484068114D2D68401B0125AD022C1AF5
:1050500004E00E4800680D4D6D68441BA14201D963
:10506000012070BD00220CE09D5C084846680830B5
:10507000855508388088401C8005800D034D686088
:10508000521C8A42F0D30020EBE70000741200208B
:1050900010B50248FFF7EAFA10BD0000901A0200AE
:1050A0000021014A1175704740600040014600BF71
:1050B000F020084000110A23584302460807000F59
:1050C0008018C0B270470146002204E0501CC2B2F2
:1050D00008460A38C1B20A29F8DA1007000E084358
:1050E0007047000010B5044601218020F6F7BCF996
:1050F000607A012805D14248C07810210843404910
:10510000C870607AA22805D13E48007F80210843FC
:105110003C490877607A3B49087700203A4948774C
:105120000846407F2178084337494877E07B0028CC
:1051300005D00846407F202108433349487732484C
:10514000407FC008C000A17A08432F49487708462D
:10515000807FF72108402C498877E078FFF7B3FF7C
:1051600029498874A078FFF7AEFF2749C874607892
:10517000FFF7A9FF244908752078002805D10846C3
:10518000007D2179084320490875E079FFF79BFFEE
:105190001D4988756079FFF796FF1B494875A0790E
:1051A000FFF791FF1849C875207AFFF78CFF164961
:1051B00008760846807F4006400E8877E07A00280F
:1051C00006D00846807F402108430F49887703E0D6
:1051D0000D48807F0C498877A07BFFF774FF0A4950
:1051E0008876607BFFF76FFF0749C876207B0877DA
:1051F0000846807F102188430349887710BD00004E
:105200002004024060040440404F044010B50446AE
:105210001B48807F01210843194988772078FFF7D0
:1052200052FF174908756078FFF74DFF1449C8749D
:10523000A078FFF748FF1249887420780C2806DD13
:105240000846407F082108430D49487709E00C488B
:10525000407F0B4948770846007DE17808430849BC
:1052600008750748807F400840000549887700BFDF
:105270000348807F022108400028F9D110BD0000BA
:10528000404F044010B500201449087616200BF05A
:1052900001FB0021124801761248407F802108431B
:1052A000104948770846807F012108430D498877D7
:1052B00000BF0C48807F022108400028F9D009482F
:1052C000807F400840000749887700BF0548807FFD
:1052D000022108400028F9D110BD000040600040C4
:1052E00040610040404F044010B50020074908705D
:1052F00000212020F6F7B8F80121054801750020AB
:105300000449087515200BF0ADFA10BD005004409B
:10531000406100404060004070B504460D46002CDE
:1053200014D0002D12D0042D10D800F013F800284E
:105330000CD1002608E00649885D22460121F4F7D9
:105340001BF8A41C701CC6B2AE42F4DB70BD00009A
:105350000C1A020000200549897DC907C90F0029E0
:1053600001D0012000E00020704700000050044000
:1053700030B585B005460C4600200390049000909F
:1053800001900290072C0BDC0120A04081B26846FE
:1053900081810121C17303A90220FAF789FE3EE051
:1053A000082C01D0092C0BD10120A04081B2684605
:1053B00081810121C17303A90120FAF779FE2EE052
:1053C0000A2C03D00B2C01D00D2C0BD10120A040B6
:1053D00081B2684681810121C17303A90020FAF7D7
:1053E00067FE1CE00C2C01D00F2C0BD10120A0403B
:1053F00081B2684681810121C17303A90E20FAF7A9
:1054000057FE0CE00E2C0AD10120A04081B2684664
:1054100081810121C17303A90C20FAF749FE002103
:1054200068460170C17041700121817000210171D5
:10543000C1720D218172FF21017200214172F3F7C7
:10544000FBFF03491520FDF7B3F805B030BD0000A0
:10545000A150010010B500201049087515200BF06F
:1054600001FA00210E4801751520002809DB00BF54
:1054700000BFC206D20E012191400A4A116000BF4E
:1054800000BF00BF084880798011032805D0064876
:105490000078802108430449087010BD4060004036
:1054A0004061004000E100E00050044010B5F4F716
:1054B000BDF810BD10B501231A4600211846F5F7B6
:1054C0008FFF012211461046F5F7EEFFF2F7FAFDC5
:1054D00003480BF0D3FC02480249086010BD0000ED
:1054E0000090D0034C07002000BF0448006904214D
:1054F00008430249086130BF00BF704700ED00E07B
:10550000F3B585B00546002400270026002003904F
:105510000490EEB22804070E0F2F54DA082E52DA48
:10552000002009E00C214143284A515AA94201D1E7
:10553000044603E0411CC8B21728F3D300BF012082
:10554000B04086B20C20604320494018C3780C203C
:10555000604340188278F8B231460190FAF74CFE69
:1055600068468681012181730021C1730221417443
:10557000F8B203A9FAF79CFD0C216143134A89187C
:10558000C888FBF7D5FE0C20604310494018C1883D
:105590006846018169460698887202A8FBF7E2FD19
:1055A0000C226243094BD21891680C226243D21834
:1055B00004201056FCF7FCFF0C216143034A8918B4
:1055C000C888FBF739FE07B0F0BD0000281C0200B8
:1055D000FEB505460C460020C0430290EFB22804F9
:1055E000060E0F2E42DA082F40DA0120B840694635
:1055F000088080202040002816D101208870A00754
:10560000800F022801D1487109E0A007800F01280E
:1056100002D16946487102E0002069464871F0B243
:105620006946FAF745FD1FE00020694688700E20A4
:105630002040002800D000BF10202040002802D1C8
:105640006946087102E0012069460871E007C00F51
:10565000002802D16946887102E0012069468871FC
:10566000F0B26946FAF724FD002002900298FEBDD0
:1056700030B50146CAB20C04230E00200F2B0FDAFE
:10568000082A0DDA01249440A2B2064C03252D020B
:105690006419E45C1440002C01D0012000E00020DB
:1056A00030BD000000000440F8B504460F4600205D
:1056B000C0430090E6B22004050E0F2D11DA082E2B
:1056C0000FDA0120B04086B2002F04D1E8B2314693
:1056D000FAF7EAFD03E0E8B23146FAF7F5FD0020FB
:1056E00000900098F8BD00001649897F01221143FF
:1056F000144A917700BF1349897F02221140002983
:10570000F9D01049897C81700E49C97C41700D49DE
:10571000097D01700B498A7D8271497D01710949BA
:10572000CA7D42710A7EC271897F49084900054AD3
:10573000917700BF0349897F022211400029F9D1E6
:1057400070470000404F044003B585B00020019031
:10575000029003900490002168464173817E01A865
:10576000C1706846417E01A881706846017E417122
:10577000002101A80171082168460171817D01A8FD
:10578000C1716846C17D4172417D01A88171684641
:10579000017D01A80172002168468173C17301A8CF
:1057A00081730C2141734121684601740021C17449
:1057B00001A8FFF797FC1D200449888204491620A0
:1057C000FCF7F6FE00F006F807B000BD204F0440DD
:1057D000C90F020010B5FFF755FD10BD70B50446A6
:1057E0000D46601E0D49884200D90124002C00D1CD
:1057F000012440200A49087008460078604309499E
:1058000048610321081F0BF05DF8002005498861FD
:10581000072008610448056070BD0000FFFFFF001D
:105820007801002000E000E0740100200020C04367
:10583000002809DBC206D20E01219140054A116001
:10584000BFF34F8FBFF36F8F00BF00200249086185
:105850008861704780E100E000E000E010B50AF0E8
:10586000D7FF10BD1A20084908722B2048723C202F
:1058700088724D20C8727F20044909680860AC20F6
:105880000349487070470000000402407C0100207A
:105890000010024010B51C480078012812D11B48A6
:1058A0000078642809DB022019494871087100203A
:1058B000164908701449087004E014480078401C28
:1058C000124908701348007801281CD1124800784A
:1058D000012804D1002010490870104908700F48B1
:1058E000007832280ADBF7F7C3F900210C48F5F7F6
:1058F000E9FC55210B48F5F735FD04E00748007831
:10590000401C0649087010BD190700201807002028
:1059100008070020120700201407002013070020AA
:105920005408002060080020F8B504460D46002702
:105930000020009003200003204000130090102C52
:1059400004D0122C02D01148844217D122202840C2
:10595000222806D127073F0F39460098F4F7DCFECE
:1059600006461220284012280ED12007000F471C9F
:1059700039460098F4F7D0FE064605E02107090FE6
:105980000098F4F7C9FE06463046F8BD1010000036
:10599000F8B504460D4600260027012000032040EC
:1059A0000713102C04D0122C02D00F48844215D1BA
:1059B00022202840222805D12607360F31463846B6
:1059C000FAF76AF81220284012280CD12007000F9D
:1059D000461C31463846FAF75FF804E02107090F04
:1059E0003846FAF759F8F8BD10100000FFB58BB033
:1059F0001C4600200790069005903848049010211E
:105A00000B980840002801D0022707E040210B989E
:105A10000840002801D0012700E00027002C04D016
:105A2000149804700120089001E0102008900025CF
:105A300048E0002C08D025466000294A115A0C98ED
:105A4000F2F784FB079006E06800254A115A0C988B
:105A5000F2F77CFB07903E4630E0711C0798F2F7A6
:105A600075FB400806900D98F2F7C6FC03900D9A5E
:105A70000699881AF2F7C0FC18490190F2F741FC28
:105A800002900399F2F77AFC05900598F2F7BBFCB7
:105A900049004908039102900498F2F7B4FC4900C8
:105AA000490801910090039B029AF2F7C1FC03D2CE
:105AB0000A95099605980490701CC6B27F2ECCDD1D
:105AC000681CC5B208988542B3DB14990A9808701F
:105AD00014990998487004980FB0F0BD0000C842AE
:105AE0003C1D02000246412A2ED010DC212A2AD079
:105AF00006DC102A45D0122A4BD0202A59D11CE0AE
:105B0000222A26D0232A2AD0402A52D116E08123E5
:105B10005B01D01A9A4228D008DC422A1AD0432AC4
:105B20001ED025481018002843D13AE0012822D081
:105B300020281BD021283CD11EE000BF1F4803892C
:105B40000B43038136E000BF1C4843890B4343816C
:105B500030E000BF194883890B4383812AE000BFEE
:105B60001648C3890B43C38124E000BF14488388CF
:105B70000B4383801EE000BF1148C3880B43C380E2
:105B800018E00E4843890B43438103890B4303818B
:105B900010E00A48C3890B43C38183890B43838187
:105BA00008E00748C3880B43C38083880B43838086
:105BB00000E000BF00BF7047F0EFFFFF001104409E
:105BC00000140440F0B505460E46412D30D010DCDF
:105BD000212D2CD006DC102D51D0122D56D0202D89
:105BE00062D11CE0222D2AD0232D30D0402D5BD154
:105BF00016E081214901681A8D4230D008DC422D1F
:105C00001ED0432D24D02A48281800284CD144E027
:105C100001282CD0202823D0212845D128E000BFFE
:105C2000244F3888314600F049F804463DE000BF73
:105C3000204F7888314600F041F8044635E000BF37
:105C40001C4FB888314600F039F804462DE000BFFB
:105C5000184FF888314600F031F8044625E000BFBF
:105C6000154F3888314600F029F804461DE000BF82
:105C7000114F7888314600F021F8044615E00D4FA9
:105C80007888314600F01AF804460EE0094FF8888B
:105C9000314600F013F8044607E0074F7888314694
:105CA00000F00CF8044600E000BF00BF2046F0BD45
:105CB000F0EFFFFF001104400014044002460020F2
:105CC00013460B40002B01D0012000E0002070475C
:105CD000FFB581B00E461746012F07D1F748407D2A
:105CE00000090001C01DF549487505E0F348407DF5
:105CF00000090001F1494875049801287ED10A2164
:105D00000198F2F723FA0546ED48445DE007C00F1D
:105D1000002807D0E948007C00090001C01DE749C0
:105D2000087405E0E548007C00090001E3490874B7
:105D300002202040002807D0E048C07BF0218843A3
:105D40007030DE49C87305E0DC48C07BF021884331
:105D5000DA49C87304202040002807D0D748807C47
:105D600000090001C01DD549887405E0D348807C36
:105D700000090001D149887408202040002807D07C
:105D8000CE48407CF02188437030CC49487405E00F
:105D9000CA48407CF0218843C849487410202040FC
:105DA000002807D0C548407C00090001C01DC34938
:105DB000487405E0C148407C00090001BF494874AF
:105DC00020202040002807D0BC48007CF0218843D8
:105DD0007030BA49087405E0B848007CF021884367
:105DE000B649087440202040002808D0B348807C81
:105DF000F02188437030B149887406E08BE0AF48E9
:105E0000807CF0218843AD4988740A210198F2F71B
:105E10009DF90D46AA48445DE007C00F002807D051
:105E2000A648807BF02188437030A449887305E040
:105E3000A248807BF0218843A0498873022020403B
:105E4000002807D09D48807B00090001C01D9B49A8
:105E5000887305E09948807B0009000197498873A1
:105E600004202040002807D09448007DF02188437A
:105E700070309249087505E09048007DF021884314
:105E80008E49087508202040002807D08B48007DE7
:105E900000090001C01D8949087505E08748007D9B
:105EA000000900018549087510202040002807D00E
:105EB0008248C07CF021884370308049C87405E076
:105EC0007E48C07CF02188437C49C8742020204053
:105ED000002807D07948C07B00090001C01D774920
:105EE000C87305E07548C07B000900017349C87399
:105EF00040202040002807D07048C07C00090001E5
:105F0000C01D6E49C87454E06C48C07C0009000193
:105F10006A49C8744DE06948007C0009000167497E
:105F200008740846C07BF02188436449C87308465A
:105F3000807C0009000188740846407CF021884379
:105F40005E4948740846407C0009000148740846D0
:105F5000007CF0218843594908740846807CF02170
:105F60008843564988740846807BF021884353490A
:105F700088730846807B0009000188730846007D0D
:105F8000F02188434D4908750846007D000900014D
:105F900008750846C07CF02188434849C874084603
:105FA000C07B00090001C8730846C07C00090001DD
:105FB000C8740A9801287DD10A213046F2F7C6F844
:105FC00005463F48445DE007C00F002807D03B4826
:105FD000407B00090001C01D3849487305E037487F
:105FE000407B000900013549487302202040002809
:105FF00007D03248007BF021884370302F49087366
:1060000005E02E48007BF02188432C4908730420CA
:106010002040002807D02948807DF0218843703037
:106020002649887505E02548807DF021884323496D
:10603000887508202040002807D02048807D00096E
:106040000001C01D1D49887505E01C48807D0009C0
:1060500000011A49887510202040002807D01748F1
:10606000407DF021884370301449487505E013489D
:10607000407DF021884311494875202020400028A8
:1060800007D00E48407BF021884370300B4948739D
:1060900005E00A48407BF0218843084948734020C6
:1060A000204000280ED00548C07D00090001C01D19
:1060B000024900E092E0C8750AE000005026002086
:1060C0007C1702006D48C07D000900016B49C8754E
:1060D0000A213046F2F73AF80D466948445DE00778
:1060E000C00F002807D06548C07AF021884370307F
:1060F0006249C87205E06148C07AF02188435F496F
:10610000C87202202040002807D05C48C07A0009ED
:106110000001C01D5949C87205E05848C07A0009FD
:1061200000015649C87204202040002807D0534877
:10613000407E00090001C01D5049487605E04F48E7
:10614000407E000900014D49487608202040002883
:1061500007D04A48007EF0218843703047490876CE
:1061600005E04648007EF021884344490876102027
:106170002040002807D04148007E00090001C01DD2
:106180003E49087605E03D48007E000900013B4994
:10619000087620202040002807D03848007B0009DE
:1061A0000001C01D3549087305E03448007B000933
:1061B00000013249087340202040002807D02F48B2
:1061C000C07DF021884370302C49C87554E02B48BD
:1061D000C07DF02188432949C8754DE02748407BA0
:1061E00000090001254948730846007BF0218843D7
:1061F000224908730846807DF02188431F4988752D
:106200000846807D0009000188750846407DF02120
:1062100088431A4948750846407BF021884317494E
:1062200048730846C07D00090001C8750846C07A59
:10623000F02188431149C8720846C07A000900015C
:10624000C8720846407E0009000148760846007E74
:10625000F0218843094908760846007E00090001BC
:1062600008760846007B0009000108730846C07DD7
:10627000F02188430149C87505B0F0BD50260020C3
:106280007C170200FFB581B00E4617460198012821
:106290007ED10498002826D1FA480078012822D01F
:1062A000F6F7CCFBF84988421DD3FAF787FD0028A2
:1062B0000DD0F648807DF02188437030F349887511
:1062C0000846C07C00090001C01DC87418E0EF48F2
:1062D000807DF0218843ED4988750846C07C00091F
:1062E0000001C8740CE0E948807DF02188437030DB
:1062F000E64988750846C07C00090001C01DC874C5
:10630000E248C07CF02188437030E049C8740846F8
:10631000007EF02188437030DC4908760846807D95
:1063200000090001401C88750846407DF021884323
:106330001030D64948750846407D00090001401CD0
:1063400048750846007DF02188431030CF49087514
:106350000846007D00090001401C087533000AF062
:1063600073FA062E261E140C042FC848007D00095F
:106370000001C01DC549087500BFC448007DF0215B
:1063800088437030C149087500BFC048407D00E0B7
:10639000ADE100090001C01DBC49487500BFBB4804
:1063A000407DF02188437030B849487500BFB74838
:1063B000807D00090001C01DB449887500BF00E060
:1063C00000BF00BF049800285ED1AE4800780128C5
:1063D0005AD0F6F733FBAC49884255D3AB48C07F5F
:1063E000F0218843A949C8770846807F0009000149
:1063F00088770846407FF0218843A44948770846BB
:10640000007FF0218843A14908770846C07DF0212C
:1064100088439E49C8750846C07F00090001C877B7
:106420000846807FF0218843984988770846407F56
:1064300000090001C01D48770846807EF02188438E
:10644000924988760846807E0009000188760846D1
:10645000407E0009000148760846007E00090001E0
:1064600008760846007F0009000108770846C07ECC
:10647000F02188438549C8760846407EF02188434C
:10648000703082494876B8E164213846F1F75EFE03
:106490000546012D07D17D48C07FF021884370302B
:1064A0007A49C87705E07948C07FF0218843774969
:1064B000C8770A213846F1F749FE0A210090F1F722
:1064C00045FE0D46642F02D37148445D01E07148DA
:1064D000445DE007C00F002807D06C48807F0009AA
:1064E0000001C01D6949887705E06848807F000980
:1064F00000016649887702202040002807D06348C1
:10650000407FF021884370306049487705E05F485C
:10651000407FF02188435D494877042020400028CF
:1065200007D05A48007FF0218843703057490877D8
:1065300005E05648007FF021884354490877082039
:106540002040002807D05148C07DF021884370309A
:106550004E49C87505E04D48C07DF02188434B4940
:10656000C87510202040002807D04848C07F000987
:106570000001C01D4549C87705E04448C07F0009B7
:1065800000014249C87720202040002807D03F481A
:10659000807FF021884370303C49887705E03B4894
:1065A000807FF021884339498877402020400028A7
:1065B00007D03648407F00090001C01D33494877A5
:1065C00005E03248407F00090001304948770A2140
:1065D0003846F1F7BBFD0D462D48445DE007C00F7E
:1065E000002807D02948807EF02188437030274951
:1065F000887605E02548807EF02188432349887607
:1066000002202040002807D02048807E0009000199
:10661000C01D1E49887605E01C48807E00090001E7
:106620001A49887604202040002807D01748407E69
:1066300000090001C01D1549487605E01348407E59
:10664000000900011149487608202040002807D0A1
:106650000E48007E00090001C01D0C49087605E0C7
:106660000A48007E000900010849087610202040F1
:10667000002811D00548007F00090001C01D034912
:1066800008770FE0E9000020B80B00002427002065
:106690007C1702008F1702005948007F0009000193
:1066A0005749087720202040002807D05448C07E52
:1066B000F021884370305249C87605E05048C07ECA
:1066C000F02188434E49C87640202040002807D05A
:1066D0004B48407EF02188437030494948768CE031
:1066E0004748407EF02188434549487685E0444844
:1066F000807D00090001424988750846407DF021EF
:1067000088433F4948750846407D000900014875A7
:106710000846007DF0218843394908750846007D08
:106720000009000108750846C07C00090001C87412
:106730000846807DF0218843314988750846C07C31
:10674000F02188432E49C8740846007EF021884312
:106750002B4908760846C07FF02188432849C8772E
:106760000846807F0009000188770846407FF021B5
:106770008843234948770846007FF0218843204911
:1067800008770846C07DF02188431D49C875084632
:10679000C07F00090001C8770846807FF021884348
:1067A000174988770846407F000900014877084666
:1067B000807EF0218843124988760846807E000951
:1067C000000188760846407E0009000148760846A8
:1067D000007E0009000108760846007F00090001DC
:1067E00008770846C07EF02188430549C8760846E8
:1067F000407EF02188430249487605B0F0BD000094
:106800002427002010B50146002200200A0EFE4B6E
:10681000985CC307DB0F002B07D0FC4BDB7FF02419
:10682000A3437033F94CE37705E0F84BDB7FF024AA
:10683000A343F64CE37702230340002B07D0F34B2E
:10684000DB7F1B091B01DB1DF04CE37705E0EF4B01
:10685000DB7F1B091B01ED4CE37704230340002B76
:1068600007D0EA4B9B7F1B091B01DB1DE74CA3777D
:1068700005E0E64B9B7F1B091B01E44CA377082333
:106880000340002B09D0E14B20335B781B091B012F
:10689000DB1DDE4C2034637007E0DC4B20335B787B
:1068A0001B091B01D94C2034637010230340002BBB
:1068B00009D0D64B20331B78F024A3437033D34C3C
:1068C0002034237007E0D14B20331B78F024A343FE
:1068D000CE4C2034237020230340002B09D0CB4B17
:1068E00020331B781B091B01DB1DC84C203423708F
:1068F00007E0C64B20331B781B091B01C34C203417
:10690000237040230340002B07D0C04B9B7FF02413
:10691000A3437033BD4CA37705E0BC4B9B7FF024B1
:10692000A343BA4CA377FF231B040B401A0CB64BAE
:10693000985CC307DB0F002B07D0B44B1B7F1B09F0
:106940001B01DB1DB14C237705E0B04B1B7F1B09FE
:106950001B01AE4C237702230340002B07D0AB4B27
:10696000DB7EF024A3437033A84CE37605E0A74B0D
:10697000DB7EF024A343A54CE37604230340002BE5
:1069800007D0A24B9B7EF024A34370339F4CA37689
:1069900005E09E4B9B7EF024A3439C4CA3760823EA
:1069A0000340002B07D0994B5B7FF024A343703347
:1069B000964C637705E0954B5B7FF024A343934CA3
:1069C000637710230340002B07D0904B5B7F1B099C
:1069D0001B01DB1D8D4C637705E08C4B5B7F1B0936
:1069E0001B018A4C637720230340002B07D0874B81
:1069F0001B7FF024A3437033844C237705E0834B43
:106A00001B7FF024A343814C237740230340002BBA
:106A100007D07E4BDB7E1B091B01DB1D7B4CE37625
:106A200005E07A4BDB7E1B091B01784CE376FF23E4
:106A30001B020B401A0A744B985CC307DB0F002B38
:106A400007D0724B1B7EF024A34370336F4C237628
:106A500005E06E4B1B7EF024A3436C4C237602238F
:106A60000340002B07D0694B1B7E1B091B01DB1D5C
:106A7000664C237605E0654B1B7E1B091B01634CAE
:106A8000237604230340002B07D0604BDB7D1B09DA
:106A90001B01DB1D5D4CE37505E05C4BDB7D1B09D9
:106AA0001B015A4CE37508230340002B07D0574BBA
:106AB0009B7E1B091B01DB1D544CA37605E0534B49
:106AC0009B7E1B091B01514CA37610230340002B16
:106AD00007D04E4B5B7EF024A34370334B4C637660
:106AE00005E04A4B5B7EF024A343484C63762023A9
:106AF0000340002B07D0454B5B7E1B091B01DB1DB0
:106B0000424C637605E0414B5B7E1B091B013F4C09
:106B1000637640230340002B07D03C4BDB7DF02401
:106B2000A3437033394CE37505E0384BDB7DF0242B
:106B3000A343364CE375CAB2334B985CC307DB0FF3
:106B4000002B07D0314B1B7DF024A34370332F4C17
:106B5000237505E02D4B1B7DF024A3432B4C23759F
:106B600002230340002B07D0284B1B7D1B091B0170
:106B7000DB1D264C237505E0244B1B7D1B091B01E7
:106B8000224C237504230340002B07D01F4BDB7CD2
:106B90001B091B01DB1D1D4CE37405E01B4BDB7C5B
:106BA0001B091B01194CE37408230340002B07D079
:106BB000164B9B7CF024A3437033144CA37405E064
:106BC000124B9B7CF024A343104CA374102303406E
:106BD000002B07D00D4B5B7DF024A34370330B4C8F
:106BE000637505E0094B5B7DF024A343074C637597
:106BF00020230340002B0BD0044B5B7D1B091B01A2
:106C0000DB1D024C637509E07C170200042700209D
:106C10000C4B5B7D1B091B010A4C63754023034031
:106C2000002B07D0074BDB7CF024A3437033054CCB
:106C3000E37405E0034BDB7CF024A343014CE374D5
:106C400010BD00000427002000B501287ED1FE4AB7
:106C5000D278F0239A437032FB4BDA701A461279DD
:106C600012091201D21D1A711A461279F0239A43A1
:106C70007032F54B1A711A46527912091201D21D5F
:106C80005A711A465279F0239A437032EE4B5A7178
:106C90001A46D27912091201D21DDA711A46D27936
:106CA000F0239A437032E84BDA711A46527A12098D
:106CB0001201D21D5A721A46527AF0239A43703248
:106CC000E14B5A721A46927AF0239A437032DE4BA5
:106CD0009A721A469278F0239A437032DA4B9A707D
:106CE0001A46D27A12091201D21DDA721A46527865
:106CF00012091201D21D5A701A46D27AF0239A4311
:106D00007032D14BDA721A46203AD27FF0239A437E
:106D10007032CD4B203BDA77CB4A127B120912013D
:106D2000D21D20331A731A46203A927F120912019B
:106D3000D21D203B9A77C44A127BF0239A437032CB
:106D4000C14B1A731A46203A127F00E0F2E1F02399
:106D50009A437032BC4B203B1A77BB4A527B1209D4
:106D60001201D21D20335A731A46203AD27E1209DC
:106D70001201D21D203BDA76B44AD278F0239A432E
:106D80007032B24BDA701A46127B12091201D21D10
:106D90001A731A46127912091201D21D1A711A4673
:106DA000927AF0239A437032A84B9A721A4612795B
:106DB000F0239A437032A54B1A711A465279120980
:106DC0001201D21D5A711A46927912091201D21D6E
:106DD0009A711A46127A12091201D21D1A721A46B3
:106DE000127AF0239A437032984B1A721A46527AEA
:106DF00012091201D21D5A72934A92791209120194
:106E0000521C914B9A711A469279F0239A43103290
:106E10008D4B9A711A46127A12091201521C1A727B
:106E20001A46127AF0239A431032874B1A721A4686
:106E3000927A12091201521C9A721A46D2781209D9
:106E40001201521CDA701A46927812091201521C71
:106E50009A701A465278F0239A4310327A4B5A703D
:106E60001A461278F0239A431032774B1A701A465A
:106E7000127812091201521C1A701A46203AD27F57
:106E800012091201521C203BDA771A46927FF02336
:106E90009A4310326C4B203B9A771A46527FF0236C
:106EA0009A431032684B203B5A771A46527F120998
:106EB0001201521C5A771A46127F12091201521CF3
:106EC0001A771A46D27EF0239A4310325E4B203B4B
:106ED000DA761A46927EF0239A4310325A4B203BC0
:106EE0009A765A4A127BF0239A431032574B1A7300
:106EF0001A46D27AF0239A431032544BDA721A4669
:106F0000D27A12091201521CDA721A46927A1209C6
:106F10001201521C9A721A46527AF0239A43103286
:106F20004A4B5A721A465279F0239A431032474B11
:106F30005A711A46D279F0239A431032434BDA71D0
:106F40000B0009F081FC19F3E9DFD5CBC1B7ADA384
:106F5000998F87786E645A50463E362E261E160E3E
:106F6000F5003A4AD279F0239A437032374BDA71FE
:106F700000BF364A5279F0239A437032334B5A712C
:106F800000BF324A527AF0239A4370322F4B5A7222
:106F900000BF2E4A927A12091201D21D2B4B9A720F
:106FA00000BF2A4AD27A12091201D21D274BDA7287
:106FB00000BF264AD27AF0239A437032234BDA720A
:106FC00000BF224A127BF0239A4370321F4B1A7380
:106FD00000BF1D4A203A927EF0239A4370321A4B2A
:106FE000203B9A7600BF184A203AD27EF0239A437B
:106FF0007032154B203BDA7600BF134A203A127FDD
:1070000012091201D21D104B203B1A7700BF0E4A05
:10701000203A527F12091201D21D0B4B203B5A77A6
:1070200000BF094A203A527FF0239A437032064B40
:10703000203B5A7700BF044A203A927FF0239A43BC
:107040007032014B203B03E07026002044270020D3
:107050009A7700BFDC4AD27F12091201D21DDA4BA7
:10706000DA7700BFD84A2032127812091201D21DF5
:10707000D54B20331A7000BFD34A20321278F02348
:107080009A437032D04B20331A7000BFCE4A203260
:107090005278F0239A437032CB4B20335A7000BFA2
:1070A000C94A2032927812091201D21DC64B2033F0
:1070B0009A7000BFC44A2032D27812091201D21D40
:1070C000C14B2033DA7000BFBF4A2032927A1209D6
:1070D0001201D21DBC4B20339A7200BFBA4A203233
:1070E000127AF0239A437032B74B20331A7200BFE2
:1070F000B54A2032127A12091201D21DB24B203346
:107100001A7200BFB04A20329279F0239A4370324B
:10711000AD4B20339A7100BFAB4A203292791209ED
:107120001201D21DA84B20339A7100BF01E0FFE786
:1071300000BF47E1A44A2032D278F0239A43A24B01
:107140002033DA701A461279120912011A711A469E
:107150001279F0239A439C4B20331A711A465279C4
:10716000120912015A711A465279F0239A43964B2A
:1071700020335A711A46D27912091201DA711A466D
:10718000D279F0239A43904B2033DA711A46527A1F
:10719000120912015A721A46527AF0239A438A4B04
:1071A00020335A721A46927AF0239A43864B203340
:1071B0009A721A469278F0239A43834B20339A703E
:1071C0001A46D27A12091201DA721A465278120954
:1071D00012015A701A46D27AF0239A437A4B20331E
:1071E000DA72794AD27FF0239A43774BDA771A46DC
:1071F0002032127B1209120120331A73724A927FD5
:1072000012091201203B9A771A462032127BF02392
:107210009A436D4B20331A736B4A127FF0239A43C3
:10722000694B1A771A462032527B12091201203319
:107230005A73654AD27E12091201203BDA76634AFC
:10724000D278F0239A43614BDA701A46127B120906
:1072500012011A731A461279120912011A711A468A
:10726000927AF0239A43594B9A721A461279F02374
:107270009A43564B1A711A465279120912015A71E1
:107280001A469279120912019A711A46127A120953
:1072900012011A721A46127AF0239A434B4B1A7251
:1072A0001A46527A120912015A72474A20329279CA
:1072B00012091201444B20339A711A469279F02335
:1072C0009A43414B20339A711A46127A12091201DD
:1072D0001A721A46127AF0239A433B4B20331A72E1
:1072E0001A46927A120912019A721A46D278120933
:1072F0001201DA701A469278120912019A701A462F
:107300005278F0239A43304B20335A701A46127841
:10731000F0239A432C4B20331A701A461278120924
:1073200012011A70284AD27F12091201203BDA7723
:107330001A46927FF0239A43234B9A771A46527F3C
:10734000F0239A43204B5A771A46527F12091201B2
:107350005A771A46127F120912011A771A46D27EFC
:10736000F0239A43184BDA761A46927EF0239A431A
:10737000154B9A76154A127BF0239A43134B1A73D6
:107380001A46D27AF0239A43104BDA721A46D27A0E
:1073900012091201DA721A46927A120912019A72CD
:1073A0001A46527AF0239A43084B5A721A46527977
:1073B000F0239A43054B5A711A46D279F0239A4327
:1073C000024BDA7100BD0000502600204427002047
:1073D000F7B582B006461746002500200190002E22
:1073E0007ED1F9F7EDFB05285FD1F9F7E7FC00281E
:1073F0000DD0FA484079F02188437030F749487140
:107400000846807800090001C01D88700AE0F34832
:107410004079F0218843F149487108468078000995
:1074200000018870ED48C07900090001EB49C8717E
:1074300008468079000900018871084640790009F2
:10744000000148710846007AF0218843E349087238
:107450000846007A0009000108720846C079F02148
:107460008843DE49C8710846C07800090001C87029
:1074700008468078F0218843D849887008464078CB
:10748000F0218843D549487008464078000900013A
:107490004870084600790009000108710846C07864
:1074A000F0218843CD49C87029E2CC484079F021C9
:1074B00088437030C9494871084680780009000146
:1074C000C01D88700846C07900090001C8710846CF
:1074D000807900090001887108464079000900E0C0
:1074E00034E0000148710846007AF0218843BB4926
:1074F00008720846007A0009000108720846C0793F
:10750000F0218843B549C8710846C07800090001D8
:10751000C87008468078F0218843B04988700846D2
:107520004078F0218843AD4948700846407800090A
:1075300000014870084600790009000108710846FA
:10754000C078F0218843A549C870ADE7012E5FD10E
:10755000F9F734FC00280DD0A0484079F021884389
:1075600070309E4948710846807800090001C01DAE
:1075700088700AE099484079F0218843974948711A
:10758000084680780009000188709448C079000995
:1075900000019249C871084680790009000188718C
:1075A000084640790009000148710846007AF02138
:1075B00088438A4908720846007A00090001087267
:1075C0000846C079F02188438449C8710846C078CC
:1075D00000090001C87008468078F02188437F497F
:1075E000887008464078F02188437C4948700846F6
:1075F0004078000900014870084600790009000140
:1076000008710846C078F02188437449C870EAE3DD
:10761000022E7DD1F9F7D4FA05287AD1F9F7CEFBFD
:10762000002877D0012F76D10A210398F0F78EFD3C
:107630000546F9F7E3FA002802D16948445D01E004
:107640006848445DE007C00F002807D06348C07950
:1076500000090001C01D6149C87105E05F48C0799B
:10766000000900015D49C87102202040002807D0B0
:107670005A48807900090001C01D5849887105E009
:10768000564880790009000154498871042020403F
:10769000002807D05148407900090001C01D4F491A
:1076A000487105E04D484079000900014B49487197
:1076B00008202040002807D04848007AF02188435D
:1076C00070304649087205E04448007AF02188434A
:1076D0004249087210202040002807D03F48007A15
:1076E00000090001C01D3D49087205E03B48007AD1
:1076F00000090001394908722020204000280BD0E1
:107700003648C079F021884370303449C87109E0A7
:10771000AEE242E1F4E0A4E03048C079F0218843D1
:107720002E49C87140202040002807D02B484079BE
:10773000F021884370302949487105E02748407995
:10774000F0218843254948710A210398F0F7FEFC8F
:107750000D462348445DE007C00F002807D01F48AE
:10776000C07800090001C01D1C49C87005E01B4815
:10777000C078000900011949C87002202040002883
:1077800007D016488078F0218843703013498870FC
:1077900005E012488078F021884310498870042061
:1077A0002040002807D00D484078F02188437030F1
:1077B0000A49487005E009484078F02188430749A4
:1077C00048700820204000280ED004484078000966
:1077D0000001C01D014948700CE000009026002007
:1077E0007C1702008F170200FE4840780009000154
:1077F000FC49487010202040002807D0F948007943
:1078000000090001C01DF749087105E0F54800793D
:1078100000090001F349087120202040002807D00A
:10782000F048C078F02188437030EE49C87005E018
:10783000EC48C078F0218843EA49C87040202040D5
:10784000002807D0E748807800090001C01DE549FD
:107850008870C8E2E348807800090001E149887037
:10786000C1E2E0484079F02188437030DD49487139
:107870000846807800090001C01D88700846C0795C
:1078800000090001C871084680790009000188716B
:10789000084640790009000148710846007AF02145
:1078A0008843D04908720846007A0009000108722E
:1078B0000846C079F0218843CA49C8710846C07893
:1078C00000090001C87008468078F0218843C54946
:1078D000887008464078F0218843C24948700846BD
:1078E000407800090001487008460079000900014D
:1078F00008710846C078F0218843BA49C87072E21E
:10790000B8484079F0218843B649487108468078E4
:107910000009000188700846C07900090001C8719B
:1079200008468079000900018871084640790009FD
:10793000000148710846007AF0218843A94908727D
:107940000846007A0009000108720846C079F02153
:107950008843A449C8710846C07800090001C8706E
:1079600008468078F02188439E4988700846407810
:10797000F02188439B49487008464078000900017F
:107980004870084600790009000108710846C0786F
:10799000F02188439349C87025E2012F73D10A2151
:1079A0000398F0F7D3FB0546F9F728F9002802D130
:1079B0008D48445D01E08D48445DE007C00F00281C
:1079C00007D08848C07900090001C01D8549C871E9
:1079D00005E08448C079000900018249C87102208D
:1079E0002040002807D07F48807900090001C01D91
:1079F0007C49887105E07B4880790009000179495C
:107A0000887104202040002807D07648407900097A
:107A10000001C01D7349487105E0724840790009B2
:107A200000017049487108202040002807D06D48A7
:107A3000007AF021884370306A49087205E069488D
:107A4000007AF021884367490872102020400028FE
:107A500007D06448007A00090001C01D614908721E
:107A600005E06048007A000900015E4908722020A4
:107A70002040002808D05B48C079F021884370304E
:107A80005849C87106E09DE05648C079F021884306
:107A90005449C87140202040002807D051484079FF
:107AA000F021884370304F49487105E04D484079D6
:107AB000F02188434B4948710A210398F0F746FBAF
:107AC0000D464948445DE007C00F002807D04548EF
:107AD000C07800090001C01D4249C87005E0414856
:107AE000C078000900013F49C870022020400028EA
:107AF00007D03C488078F02188437030394988703D
:107B000005E038488078F0218843364988700420A1
:107B10002040002807D033484078F0218843703057
:107B20003049487005E02F484078F02188432D49BE
:107B3000487008202040002807D02A4840780009D3
:107B40000001C01D2749487005E02648407800091B
:107B500000012449487010202040002807D0214807
:107B6000007900090001C01D1E49087105E01D488B
:107B70000079000900011B490871202020400028DD
:107B800007D01848C078F021884370301549C87074
:107B900005E01448C078F02188431249C87040209D
:107BA0002040002807D00F48807800090001C01D40
:107BB0000C49887017E10B488078000900010949D9
:107BC000887010E107484079F021884370300549FA
:107BD00048710846807800090001C01D8870084679
:107BE000C07905E0902600207C1702008F17020064
:107BF00000090001C87108468079000900018871F8
:107C0000084640790009000148710846007AF021D1
:107C10008843764908720846007A00090001087214
:107C20000846C079F02188437049C8710846C07879
:107C300000090001C87008468078F02188436B492C
:107C4000887008464078F0218843684948700846A3
:107C500040780009000148700846007900090001D9
:107C600008710846C078F02188436049C870BAE0BE
:107C7000032E9FD1F8F7A4FF05285FD1F9F79EF8EE
:107C800000280DD059484079F02188437030574979
:107C900048710846807800090001C01D88700AE01C
:107CA00052484079F021884350494871084680780D
:107CB0000009000188704D48C079000900014B4956
:107CC000C87108468079000900018871084640792A
:107CD0000009000148710846007AF02188434349B1
:107CE00008720846007A0009000108720846C07947
:107CF000F02188433D49C8710846C0780009000159
:107D0000C87008468078F021884338498870084652
:107D10004078F0218843354948700846407800098A
:107D20000001487008460079000900010871084602
:107D3000C078F02188432D49C87054E02B48007961
:107D4000F021884370302949087108464079F021B4
:107D50008843703025494871084680780009000141
:107D6000C01D88700846C07900090001C871084626
:107D700080790009000188710846407900090001F6
:107D800048710846007AF02188431849087208466D
:107D9000007A0009000108720846C079F021884382
:107DA0001249C8710846C07800090001C870084629
:107DB0008078F02188430D49887008464078F0218A
:107DC00088430A4948700846407800090001487015
:107DD000084600790009000108710846C078F021C2
:107DE00088430249C87005B0F0BD0000902600200D
:107DF00070B505460C46012D7ED1B148407D000985
:107E00000001C01DAE4948750846007DF021884339
:107E10001030AB4908750846007D00090001401C80
:107E200008750846C07CF02188431030A449C87406
:107E30000846807CF02188431030A14988740846A8
:107E4000807C00090001401C8874F9F713F80228AF
:107E500003D0F9F70FF801286CD19A48007801286F
:107E600068D0F4F7EBFD9849884263D3F8F7A6FF92
:107E700000282FD09248007DF0218843703090492F
:107E800008750846007D00090001C01D08750846F8
:107E9000C07CF021884370308949C8740846807CD2
:107EA000F02188437030864988740846807C000938
:107EB0000001C01D88740846407DF0218843703061
:107EC0007F4948750846407CF021884370307C49E2
:107ED0004874F4E07A48007DF021884310307849F6
:107EE00008750846007D00090001401C0875084619
:107EF000C07CF021884300E0B4E010307049C874C1
:107F00000846807CF021884310306D49887408460B
:107F1000807C00090001401C88740846407DF021E7
:107F20008843674948750846407CF0218843644986
:107F30004874C4E0F8F732FE002824D1F4F77EFD3F
:107F4000614988421FD3F8F739FF00280ED05C48FA
:107F5000407DF02188437030594948750846407C7F
:107F6000F02188437030564948741AE05448407DE7
:107F7000F0218843524948750846407CF0218843E7
:107F80004F4948740DE04E48407DF02188437030E1
:107F90004B4948750846407CF02188437030484979
:107FA0004874F8F7FBFD01282AD1464800780128DB
:107FB00026D0F4F743FD4449884221D34048407D10
:107FC000F021884370303E4948750846407CF021D6
:107FD000884370303A494874F8F7F0FE002807D01B
:107FE0003748007DF021884370303549087566E0D8
:107FF0003348007DF02188431030314908755EE038
:10800000230008F021FC062C241C140C042D2C4801
:10801000807C00090001C01D2949887400BF2848E0
:10802000807CF021884370302549887400BF244843
:10803000C07CF021884370302149C87400BF2048BB
:10804000007D00090001C01D1D49087500BF1C48C6
:10805000007DF021884370301949087500BF00E0A9
:1080600000BF2CE01648407DF02188431449487534
:108070000846007DF0218843114908750846007DB7
:108080000009000108750846C07CF02188430C49AE
:10809000C8740846807CF0218843094988740846E2
:1080A000807C0009000188740846407D00090001B9
:1080B00048750846407CF02188430149487470BDEA
:1080C00070260020E9000020B80B000030B5024601
:1080D000002901D1002000E00720130008F0B4FBC4
:1080E0000F09141F2B3743505D67727C88929FA93C
:1080F000B500574B5B7EF024A3430401F0252C40D0
:108100002343534C6376A1E0524B9B79F024A34365
:108110000401F0252C4023434E4CA37196E04D4BB7
:108120002033DB791B091B010407240F2343494C2F
:108130002034E3718AE0464B2033DB7C1B091B01B2
:108140000407240F2343424C2034E3747EE0404B69
:1081500040331B781B091B010407240F23433C4CAD
:108160004034237072E03A4B2033DB7FF024A3438A
:108170000401F0252C402343354C2034E37765E09F
:10818000334B20335B7BF024A3430401F0252C40C8
:1081900023432F4C2034637358E02E4B9B791B09EB
:1081A0001B010407240F23432A4CA3714EE0294BE3
:1081B0009B7CF024A3430401F0252C402343254C51
:1081C000A37443E0234BDB7E1B091B010407240F30
:1081D0002343204CE37639E01D4B2033DB7F1B0922
:1081E0001B010407240F2343194C2034E3772DE0AF
:1081F000174B9B7E1B091B010407240F2343144CC0
:10820000A37623E0134B20339B79F024A34304018E
:10821000F0252C4023430F4C2034A37116E00D4B66
:10822000DB7D1B091B010407240F2343094CE37565
:108230000CE0074B20335B7C1B091B010407240F58
:108240002343034C2034637400E000BF00BF30BD03
:108250005026002024270020F7B582B00746154697
:1082600000260024FE480078012804D0F4F7E6FB3D
:10827000FC49884279D2FC48407CF0218843703028
:10828000F94948740846807C00090001C01D8874C3
:108290000846007D00090001C01D08750846007DE4
:1082A000F02188437030F04908750846807CF02141
:1082B00088437030EC4988740846C07C000900018E
:1082C000C01DC8740846C07CF02188437030E64960
:1082D000C8740846407C00090001C01D4874084667
:1082E000407D00090001C01D48750846407DF02111
:1082F00088437030DC4948750846007CF02188438B
:108300007030D94908740846007C00090001C01D7E
:1083100008740846C07BF02188437030D249C87386
:10832000FF220A210020FBF767F9FF22132100201A
:10833000FBF762F9FF2211210020FBF75DF9FF2214
:1083400012210020FBF758F9FF220E210020FBF735
:1083500053F9FF220F210020FBF74EF9FF221021D5
:108360000020FBF749F9F4E3FFE7039836283DD0F6
:1083700019DC08287ED007DC801E030008F064FAB0
:108380000635A8FCFBFAF97E102874D006DC092813
:1083900072D00D2871D00E2870D1FDE333286ED035
:1083A0003428F9D170E13F286AD00FDC373808282B
:1083B00064D243007B449B885B009F448A00970201
:1083C000FF025F005F006503CB0318004E287BD0DF
:1083D00006DC402879D0412878D04D28DCD1BBE19B
:1083E0004F2874D05028D7D14FE100BF00BF9E481E
:1083F000407CF02188439C4948740846807C0009F1
:10840000000188740846007D00090001C01D087540
:108410000846007DF021884370309349087508466E
:10842000807CF0218843904988740846C07C00090C
:108430000001C01DC8740846C07CF02188438A49E9
:10844000C8740846407C0009000148740846407D15
:108450000009000148750846407DF02188438249A3
:1084600048750846007CF02188437F490874084617
:10847000007C06E0A1E2FDE337E2D2E3FBE394E017
:1084800028E00009000108740846C07BF0218843F9
:108490007549C873FF220A210020FBF7ADF8FF22BF
:1084A00013210020FBF7A8F800220E211046FBF74D
:1084B000A3F800220F211046FBF79EF8002210219E
:1084C0001046FBF799F877E2ABE110E2DDE26DE0F0
:1084D00000BF00BF6448407CF02188436249487473
:1084E0000846807C0009000188740846007D000968
:1084F0000001C01D08750846007DF02188437030DA
:10850000594908750846807CF0218843564988748B
:108510000846C07C00090001C8740846C07CF021F0
:1085200088435149C8740846407C000900014874DA
:108530000846407D00090001C01D48750846407D81
:10854000F0218843484948750846007CF02188435B
:10855000454908740846007C000900010874084673
:10856000C07BF02188434049C873FF220A210020C4
:1085700003E055E1EFE086E016E0FBF73DF8FF226F
:1085800013210020FBF738F800220E211046FBF7DC
:1085900033F800220F211046FBF72EF8002210219D
:1085A0001046FBF729F88EE700BF00BF2E48407C3D
:1085B000F02188432C4948740846807C000900015A
:1085C000C01D88740846007D00090001C01D0875A3
:1085D0000846007DF021884370302349087508461D
:1085E000807CF021884370301F4988740846C07C25
:1085F00000090001C8740846C07CF02188431A496C
:10860000C8740846407C0009000148740846407D53
:108610000009000148750846407DF0218843124951
:1086200048750846007CF02188430F4908740846C5
:10863000007C0009000108740846C07BF0218843D3
:108640000949C873FF220A210020FAF7D5FFFF224B
:1086500013210020FAF7D0FF00220E21104605E07A
:10866000E9000020B80B000090260020FAF7C4FFB4
:1086700000220F211046FAF7BFFF002210211046FA
:10868000FAF7BAFF1FE700BF00BFFE48407CF021A9
:108690008843FC4948740846807C00090001C01DDD
:1086A00088740846007D00090001C01D0875084651
:1086B000007DF02188437030F24908750846807CBF
:1086C000F0218843EF4988740846C07C0009000106
:1086D000C8740846C07CF0218843EA49C87408463B
:1086E000407C00090001C01D48740846407D000917
:1086F000000148750846407DF0218843E1494875EE
:108700000846007CF0218843DE4908740846007C56
:108710000009000108740846C07BF0218843D9494C
:10872000C873FF220A210020FAF766FFFF221321F7
:108730000020FAF761FF00220E211046FAF75CFFD5
:1087400000220F211046FAF757FF00221021104691
:10875000FAF752FFF6E300BFCA48407CF021884395
:10876000C84948740846807C00090001887408469E
:10877000007D0009000108750846007DF02188434E
:108780007030C04908750846807CF0218843BD4997
:1087900088740846C07C00090001C8740846C07C83
:1087A000F02188437030B749C8740846407C0009FE
:1087B000000148740846407D0009000148750846DC
:1087C000407DF0218843AF4948750846007CF02180
:1087D0008843AC4908740846007C0009000108740D
:1087E0000846C07BF0218843A649C873FF220A21AE
:1087F0000020FAF701FFFF2213210020FAF7FCFE08
:1088000000220E211046FAF7F7FE00220F21104633
:10881000FAF7F2FE002210211046FAF7EDFE91E37E
:1088200000BF9848407CF021884396494874084628
:10883000807C0009000188740846007D0009000161
:1088400008750846007DF021884370308D49087511
:108850000846807CF02188438A4988740846C07C99
:1088600000090001C8740846C07CF021884385498E
:10887000C8740846407C0009000148740846407DE1
:108880000009000148750846407DF021884370309A
:108890007C4948750846007CF02188437949087472
:1088A0000846007C0009000108740846C07BF021DE
:1088B00088437449C873FF220A210020FAF79CFEFE
:1088C000FF2213210020FAF797FE00220E21104606
:1088D000FAF792FE00220F211046FAF78DFE0022D1
:1088E00010211046FAF788FE2CE300BF00BF654850
:1088F000407CF02188437030624948740846807C8F
:1089000000090001C01D88740846007D00090001AF
:10891000C01D08750846007DF02188437030594914
:1089200008750846807CF0218843564988740846BB
:10893000C07C00090001C8740846C07CF02188434F
:108940005049C8740846407C000900014874084634
:10895000407D0009000148750846407DF0218843AC
:10896000484948750846007CF02188434549087409
:108970000846007C0009000108740846C07BF0210D
:1089800088434049C873FF220A210020FAF734FEC9
:10899000FF2213210020FAF72FFE00220E2110469D
:1089A000FAF72AFE00220F211046FAF725FE0022D0
:1089B00010211046FAF720FEC4E200BF3148407C87
:1089C000F02188432F4948740846807C0009000143
:1089D00088740846007D0009000108750846007D7E
:1089E000F02188437030274908750846807CF021C3
:1089F0008843244988740846C07C00090001C87473
:108A00000846C07CF021884370301E49C87408466F
:108A1000407C0009000148740846407D00090001BF
:108A200048750846407DF021884316494875084638
:108A3000007CF0218843134908740846007C000933
:108A4000000108740846C07BF02188430D49C873B3
:108A5000FF220A210020FAF7CFFDFF221321002078
:108A6000FAF7CAFD00220E211046FAF7C5FD0022D2
:108A70000F211046FAF7C0FD002210211046FAF728
:108A8000BBFD5FE29026002000BFFC48407CF02147
:108A90008843FA4948740846807C000900018874BC
:108AA0000846007D0009000108750846007DF02198
:108AB00088437030F14908750846807CF02188436E
:108AC000EE4988740846C07C00090001C874084655
:108AD000C07CF0218843E949C8740846407C0009FD
:108AE000000148740846407D0009000148750846A9
:108AF000407DF02188437030E04948750846007C8D
:108B0000F0218843DD4908740846007C0009000113
:108B100008740846C07BF0218843D849C873FF22F7
:108B20000A210020FAF768FDFF2213210020FAF73E
:108B300063FD00220E211046FAF75EFD00220F2190
:108B40001046FAF759FD002210211046FAF754FD9D
:108B5000F8E1F8E1C948407CF02188437030C7490A
:108B600048740846807C00090001C01D88740846CE
:108B7000007D00090001C01D08750846007DF02138
:108B80008843BE4908750846807CF0218843BB496C
:108B900088740846C07C00E0A9E000090001C874A0
:108BA0000846C07CF0218843B449C8740846407C1C
:108BB0000009000148740846407D0009000148751D
:108BC0000846407DF0218843AC4948750846007C42
:108BD000F0218843A94908740846007C0009000177
:108BE00008740846C07BF0218843A449C873FF225B
:108BF0000A210020FAF700FDFF2213210020FAF7D6
:108C0000FBFC00220E211046FAF7F6FC00220F2191
:108C10001046FAF7F1FC002210211046FAF7ECFC9E
:108C200090E19648407CF021884394494874084676
:108C3000807C0009000188740846007D000900015D
:108C400008750846007DF02188438C490875084660
:108C5000807CF0218843894988740846C07C0009DB
:108C60000001C8740846C07CF02188438349C87459
:108C7000084601E09EE003E1407C000900014874E1
:108C80000846407D0009000148750846407DF021F6
:108C900088437A4948750846007CF0218843774923
:108CA00008740846007C0009000108740846C07B6F
:108CB000F021884370307149C87300220A211046A0
:108CC000FAF79AFC002213211046FAF795FCFF22CE
:108CD0000E210020FAF790FC00220F211046FAF72F
:108CE0008BFC002210211046FAF786FC2AE163482B
:108CF000407CF0218843614948740846807C000923
:108D0000000188740846007D0009000108750846C6
:108D1000007DF0218843594908750846807CF02180
:108D20008843564988740846C07C00090001C8740D
:108D30000846C07CF02188435049C8740846407CEE
:108D40000009000148740846407D0009000148758B
:108D50000846407DF0218843484948750846007C14
:108D6000F0218843454908740846007C0009000149
:108D7000C01D08740846C07BF02188433F49C87372
:108D800000220A211046FAF737FC00221321104670
:108D9000FAF732FC00220E211046FAF72DFCFF22D2
:108DA0000F210020FAF728FC002210211046FAF7C4
:108DB00023FCC7E03148407CF02188432F494874A8
:108DC0000846807C0009000188740846007D00097F
:108DD000000108750846007DF02188432749087581
:108DE0000846807CF0218843244988740846C07C6A
:108DF00000090001C8740846C07CF02188431F495F
:108E0000C8740846407C0009000148740846407D4B
:108E10000009000148750846407DF0218843174944
:108E200048750846007CF021884370301349087467
:108E30000846007C0009000108740846C07BF02148
:108E400088430E49C87300220A211046FAF7D4FB62
:108E5000002213211046FAF7CFFB00220E21104604
:108E6000FAF7CAFB00220F211046FAF7C5FBFF22D2
:108E700010210020FAF7C0FB64E0000090260020DB
:108E8000FD48407CF0218843FB4948740846807CBB
:108E90000009000188740846007D0009000108757A
:108EA0000846007DF0218843F34908750846807C18
:108EB000F0218843F04988740846C07C000900010D
:108EC000C8740846C07CF0218843EB49C874084642
:108ED000407C0009000148740846407D00090001FB
:108EE00048750846407DF0218843E34948750846A7
:108EF000007CF0218843E04908740846007C0009A2
:108F0000000108740846C07BF0218843DA49C87321
:108F100000220A211046FAF76FFB002213211046A7
:108F2000FAF76AFB00220E211046FAF765FB0022D1
:108F30000F211046FAF760FB002210211046FAF7C5
:108F40005BFB00BF00BF002F03D0CC48007A002895
:108F500008D1F3F773FDCA49884203D3C9480078A2
:108F6000012872D1FF2211210020FAF745FBFF22D0
:108F700012210020FAF740FBC2480078012804D0F3
:108F8000F3F75CFDBE49884216D2BF48807BF021D2
:108F900088437030BC498873084640300078F0211F
:108FA00088437030B849403108700846007800099D
:108FB0000001C01D08702DE07D20C000854214D244
:108FC000B148807BF0218843AF4988730846403020
:108FD0000078F02188437030AB4940310870084672
:108FE000007800090001087014E0A748807BF02198
:108FF00088437030A4498873084640300078F021D7
:109000008843A149403108700846007800090001F2
:10901000C01D08707D20C000854205D2014628464B
:10902000EFF794F8064604E098492846EFF78EF8E3
:10903000064694480078012804D0F3F7FFFC9049D5
:10904000884203D29248845D02E0A0E29148845DA8
:10905000E007C00F002809D08B484030C0780009D5
:109060000001C01D88494031C87007E08648403083
:10907000C0780009000184494031C87002202040B6
:10908000002807D08048C07900090001C01D7E4932
:10909000C87105E07C48C079000900017A49C871AF
:1090A00004202040002807D077488079000900017B
:1090B000C01D7549887105E0734880790009000179
:1090C0007149887108202040002807D06E484079F7
:1090D000F021884370306C49487105E06A48407956
:1090E000F02188436849487110202040002807D0AB
:1090F0006548407900090001C01D6349487105E0D9
:1091000061484079000900015F49487120202040F2
:10911000002807D05C480079F021884370305A4914
:10912000087105E058480079F021884356490871D4
:1091300040202040002807D053488079F021884300
:1091400070305149887105E04F488079F02188439B
:109150004D4988717D20C000854213D26421284684
:10916000EEF7F4FF064647480078012804D0F3F7ED
:1091700065FC4349884202D24548845D23E0454866
:10918000845D20E0642128463230EEF7DFFF7D2148
:10919000C9000090EEF7DAFF019164210198EEF723
:1091A000D5FF06463C48854208D23648007801285B
:1091B00004D0F3F743FC3249884202D23448845D3C
:1091C00001E03448845DE007C00F002809D02E4834
:1091D00040308078F021884370302B4940318870CE
:1091E00007E0294840308078F02188432649403103
:1091F000887002202040002807D02348807A000988
:109200000001C01D2049887205E01F48807A0009CE
:1092100000011D49887204202040002807D01A4808
:10922000407A00090001C01D1749487205E0164840
:10923000407A0009000114494872082020400028A3
:1092400007D01148007AF021884370300E49087227
:1092500005E00D48007AF02188430B490872102080
:10926000204000281AD00848007A00090001C01DDB
:109270000549087218E0000090260020600A0020CE
:10928000B80B0000E900002004270020A0860100A0
:109290007C1702008F17020010270000FE48007A9A
:1092A00000090001FC49087220202040002807D056
:1092B000F948C079F02188437030F749C87105E05A
:1092C000F548C079F0218843F349C8714020204017
:1092D000002807D0F048407AF02188437030EE49EA
:1092E000487205E0EC48407AF0218843EA49487228
:1092F0007D20C000854219D20A212846EEF726FFBC
:109300000A210190EEF722FF0E460A2D08D2E3480B
:109310000078012804D0F3F791FBE149884202D29A
:10932000E048845D12E0E048845D0FE06421284657
:109330003230EEF70BFF0A210090EEF707FF0A210B
:109340000190EEF703FF0E46D6498C5DE007C00F93
:10935000002809D0D0484030807800090001C01DA5
:10936000CD494031887007E0CB4840308078000913
:109370000001C9494031887002202040002807D0F0
:10938000C548807B00090001C01DC349887305E002
:10939000C148807B00090001BF4988730420204038
:1093A000002807D0BC48407B00090001C01DBA4915
:1093B000487305E0B848407B00090001B64948738E
:1093C00008202040002807D0B348007BF0218843C4
:1093D0007030B149087305E0AF48007BF021884345
:1093E000AD49087310202040002807D0AA48C07A51
:1093F00000090001C01DA849C87205E0A648C07A4E
:1094000000090001A449C87220202040002807D08C
:10941000A148807AF021884370309F49887205E026
:109420009D48807AF02188439B49887240202040E3
:10943000002807D09848407BF02188437030964937
:10944000487305E09448407BF02188439249487373
:109450007D20C000854207D20A212846EEF776FE1D
:109460000E469048845D0BE0642128463230EEF7CA
:109470006DFE0A210190EEF769FE0E4689498C5D6A
:10948000E007C00F002809D0834840304078F02121
:109490008843703080494031487007E07E48403052
:1094A0004078F02188437C494031487002202040B8
:1094B000002809D078484030407800090001C01DDC
:1094C00075494031487007E07348403040780009E2
:1094D000000171494031487004202040002807D025
:1094E0006D48007CF021884370306B49087405E0BA
:1094F0006948007CF02188436749087408202040AF
:10950000002807D06448007C00090001C01D6249A2
:10951000087405E06048007C000900015E49087499
:1095200010202040002807D05B48C07BF0218843F2
:1095300070305949C87305E05748C07BF021884313
:109540005549C87320202040002807D05248C07BCE
:1095500000090001C01D5049C87305E04E48C07B9A
:10956000000900014C49C87340202040002807D062
:109570004948407C00090001C01D47494874ECE09F
:109580004548407C0009000143494874E5E0002259
:109590000A211046FAF730F8002213211046FAF794
:1095A0002BF8002211211046FAF726F8002212218A
:1095B0001046FAF721F800220E211046FAF71CF89F
:1095C00000220F211046FAF717F80022102110464A
:1095D000FAF712F830484030C078000900012E49EF
:1095E0004031C8702C48C079000900014039C87169
:1095F0000846807900090001887108464079F02109
:10960000884325494871084640790009000148719E
:1096100008460079F02188431F490871084680797F
:10962000F02188431C498871084640308078F02139
:1096300088431949403188701748807A0009000131
:10964000403988720846407A00090001487208468D
:10965000007AF0218843104908720846007A000910
:10966000000108720846C079F02188430A49C87190
:109670000846407AF021884307494872084640303E
:10968000807800090001403188700348807B000920
:1096900000014039887309E004270020E900002018
:1096A000B80B00007C1702008F1702000846407BB1
:1096B0000009000148730846007BF02188432849CF
:1096C00008730846C07A00090001C8720846807A0B
:1096D000F0218843224988720846407BF021884364
:1096E0001F494873084640304078F02188431C49A0
:1096F0004031487008464078000900014870184819
:10970000007CF0218843164908740846007C000953
:10971000000108740846C07BF02188431049C873D3
:109720000846C07B00090001C8730846407C000958
:10973000000148740846807BF021884308498873FB
:10974000084640300078F0218843054940310870D0
:109750000846007800090001087005B0F0BD00005F
:1097600004270020F7B582B007460E460121FF20EE
:109770000830FBF799FF0121FC48FBF795FFFC48F7
:10978000007801287ED0F3F759F9FA49884279D355
:10979000F7F716FA032843D1F7F70CFA002803D09D
:1097A000F7F708FA01283BD1002F1CD1F7F706FB89
:1097B00000280CD0F048407CF0218843EE494874E2
:1097C0000846807C00090001C01D8874EEE0EA486C
:1097D000407CF0218843E84948740846807C0009B1
:1097E00000018874E2E0F7F7E9FA00280CD0E248BB
:1097F000407CF02188437030DF4948740846807C03
:10980000000900018874D1E0DB48407CF0218843E6
:10981000D94948740846807C000900018874C5E075
:10982000F7F7C8F9002803D0F7F7C4F9012865D184
:10983000002F0CD1D048407CF0218843CE49487499
:109840000846807C00090001C01D88740BE0CA48EE
:10985000407CF02188437030C74948740846807CBA
:10986000000900018874F7F7A5F9002821D1C24842
:109870002030C078F02188437030BF492031C87053
:10988000BD4800E064E0807D000900012039887552
:109890000846807DF0218843B7498875FF2223213F
:1098A0000020F9F7A9FE002222211046F9F7A4FEB4
:1098B0007CE0F7F77FF9012878D1AF482030C078F5
:1098C000F0218843AC492031C870AB48807D000945
:1098D0000001C01D203988750846807DF02188432D
:1098E0007030A5498875002223211046F9F784FEBF
:1098F000FF2222210020F9F77FFE57E09E48407C9E
:10990000F02188439C4948740846807C0009000186
:10991000887408462030C078F02188439649203169
:10992000C8709548807D0009000120398875084677
:10993000807DF021884390498875002223211046BC
:10994000F9F75AFE002222211046F9F755FE2DE0C4
:109950008948407CF0218843703087494874084624
:10996000807C00090001C01D887408462030C07842
:10997000F0218843703080492031C8707E48807D56
:1099800000090001C01D203988750846807DF0213E
:109990008843703078498875FF2223210020F9F729
:1099A0002BFEFF2222210020F9F726FEF7F702F90D
:1099B000002808D06E480078012804D0F3F73EF85C
:1099C0006C49884276D26D48864209D96A4820306F
:1099D0004079F0218843703067492031487107E0B1
:1099E000654820304079F02188436349203148712F
:1099F00063493046EEF7AAFB0A210190EEF7A6FB79
:109A00000D465E48401C864202D35E48445D01E03C
:109A10005D48445DE007C00F002809D0564820305B
:109A2000C07800090001C01D53492031C87007E00B
:109A300051482030C078000900014F492031C870DA
:109A400002202040002809D04B4820308078F021A7
:109A50008843703048492031887007E046482030FC
:109A60008078F021884344492031887004202040C8
:109A7000002809D0404820304078F02188437030D9
:109A80003D492031487007E03B4820304078F021C4
:109A900088433949203148700820204000280AD0E6
:109AA00035482030407900090001C01D324920317D
:109AB000487108E0A1E230482030407900090001F7
:109AC0002D492031487110202040002809D02A4813
:109AD00020300079F0218843703027492031087107
:109AE00007E0254820300079F021884322492031C1
:109AF000087120202040002809D01F48203000791C
:109B000000090001C01D1C492031087107E01A48F6
:109B100020300079000900011749203108714020E8
:109B20002040002809D01448203080780009000126
:109B3000C01D11492031887007E00F48203080781F
:109B4000000900010C49203188707D21C900304690
:109B5000EEF7FCFA0A210190EEF7F8FA0D460848F4
:109B6000864213D30748445D12E00000050500005B
:109B7000E9000020B80B0000042700209F860100A8
:109B8000102700007C1702008F170200F948445D7F
